Component: ARM Compiler 5.06 update 6 (build 750) Tool: armlink [4d35ed]

==============================================================================

Section Cross References

    main.o(i.advertising_init) refers to memseta.o(.text) for __aeabi_memclr4
    main.o(i.advertising_init) refers to ble_advdata.o(i.ble_advdata_set) for ble_advdata_set
    main.o(i.advertising_init) refers to app_error.o(i.app_error_handler_bare) for app_error_handler_bare
    main.o(i.advertising_init) refers to main.o(.data) for .data
    main.o(i.advertising_init) refers to main.o(.bss) for .bss
    main.o(i.advertising_start) refers to app_error.o(i.app_error_handler_bare) for app_error_handler_bare
    main.o(i.advertising_start) refers to bsp.o(i.bsp_indication_set) for bsp_indication_set
    main.o(i.advertising_start) refers to main.o(.bss) for .bss
    main.o(i.assert_nrf_callback) refers to app_error.o(i.app_error_handler) for app_error_handler
    main.o(i.ble_stack_init) refers to softdevice_handler.o(i.softdevice_handler_init) for softdevice_handler_init
    main.o(i.ble_stack_init) refers to app_error.o(i.app_error_handler_bare) for app_error_handler_bare
    main.o(i.ble_stack_init) refers to softdevice_handler.o(i.softdevice_app_ram_start_get) for softdevice_app_ram_start_get
    main.o(i.ble_stack_init) refers to softdevice_handler.o(i.softdevice_enable) for softdevice_enable
    main.o(i.ble_stack_init) refers to main.o(.constdata) for .constdata
    main.o(i.ble_stack_init) refers to main.o(.bss) for .bss
    main.o(i.log_init) refers to nrf_log_frontend.o(i.nrf_log_init) for nrf_log_init
    main.o(i.log_init) refers to app_error.o(i.app_error_handler_bare) for app_error_handler_bare
    main.o(i.main) refers to main.o(i.log_init) for log_init
    main.o(i.main) refers to nrf_log_frontend.o(i.nrf_log_frontend_std_0) for nrf_log_frontend_std_0
    main.o(i.main) refers to main.o(i.timers_init) for timers_init
    main.o(i.main) refers to main.o(i.ble_stack_init) for ble_stack_init
    main.o(i.main) refers to main.o(i.advertising_init) for advertising_init
    main.o(i.main) refers to main.o(i.advertising_start) for advertising_start
    main.o(i.main) refers to twi_slave_tiny_unwrap.o(i.twi_slave_tiny_main_unwrap) for twi_slave_tiny_main_unwrap
    main.o(i.main) refers to main.o(i.power_manage) for power_manage
    main.o(i.power_manage) refers to app_error.o(i.app_error_handler_bare) for app_error_handler_bare
    main.o(i.timers_init) refers to app_timer.o(i.app_timer_init) for app_timer_init
    main.o(i.timers_init) refers to app_error.o(i.app_error_handler_bare) for app_error_handler_bare
    twi_slave_tiny_unwrap.o(i.read_reg) refers to app_twi.o(i.app_twi_perform) for app_twi_perform
    twi_slave_tiny_unwrap.o(i.read_reg) refers to app_error.o(i.app_error_handler_bare) for app_error_handler_bare
    twi_slave_tiny_unwrap.o(i.read_reg) refers to twi_slave_tiny_unwrap.o(.data) for .data
    twi_slave_tiny_unwrap.o(i.read_reg) refers to twi_slave_tiny_unwrap.o(.constdata) for .constdata
    twi_slave_tiny_unwrap.o(i.test_case) refers to twi_slave_tiny_unwrap.o(i.write_reg) for write_reg
    twi_slave_tiny_unwrap.o(i.test_case) refers to twi_slave_tiny_unwrap.o(i.read_reg) for read_reg
    twi_slave_tiny_unwrap.o(i.test_case) refers to nrf_log_frontend.o(i.nrf_log_frontend_hexdump) for nrf_log_frontend_hexdump
    twi_slave_tiny_unwrap.o(i.twi_init) refers to app_twi.o(i.app_twi_init) for app_twi_init
    twi_slave_tiny_unwrap.o(i.twi_init) refers to app_error.o(i.app_error_handler_bare) for app_error_handler_bare
    twi_slave_tiny_unwrap.o(i.twi_init) refers to twi_slave_tiny_unwrap.o(.constdata) for .constdata
    twi_slave_tiny_unwrap.o(i.twi_slave_tiny_main_unwrap) refers to twi_slave_tiny_unwrap.o(i.twi_init) for twi_init
    twi_slave_tiny_unwrap.o(i.twi_slave_tiny_main_unwrap) refers to app_error.o(i.app_error_handler_bare) for app_error_handler_bare
    twi_slave_tiny_unwrap.o(i.twi_slave_tiny_main_unwrap) refers to twi_slave_tiny_unwrap.o(i.test_case) for test_case
    twi_slave_tiny_unwrap.o(i.write_reg) refers to memcpya.o(.text) for __aeabi_memcpy
    twi_slave_tiny_unwrap.o(i.write_reg) refers to app_twi.o(i.app_twi_perform) for app_twi_perform
    twi_slave_tiny_unwrap.o(i.write_reg) refers to app_error.o(i.app_error_handler_bare) for app_error_handler_bare
    twi_slave_tiny_unwrap.o(i.write_reg) refers to twi_slave_tiny_unwrap.o(.constdata) for .constdata
    twi_slave_tiny_unwrap.o(.constdata) refers to twi_slave_tiny_unwrap.o(.bss) for m_app_twi_queue_nrf_queue_cb
    twi_slave_tiny_unwrap.o(.constdata) refers to twi_slave_tiny_unwrap.o(.bss) for m_app_twi_queue_nrf_queue_buffer
    twi_slave_tiny_unwrap.o(.constdata) refers to twi_slave_tiny_unwrap.o(.bss) for m_app_twi_cb
    twi_slave_tiny_unwrap.o(.constdata) refers to twi_slave_tiny_unwrap.o(.constdata) for m_app_twi_queue
    twi_slave_tiny_unwrap.o(.constdata) refers to twi_slave_tiny_unwrap.o(.data) for tx_buff
    boards.o(i.bsp_board_button_idx_to_pin) refers to boards.o(.constdata) for .constdata
    boards.o(i.bsp_board_button_state_get) refers to boards.o(.constdata) for .constdata
    boards.o(i.bsp_board_buttons_init) refers to boards.o(i.nrf_gpio_cfg) for nrf_gpio_cfg
    boards.o(i.bsp_board_buttons_init) refers to boards.o(.constdata) for .constdata
    boards.o(i.bsp_board_led_idx_to_pin) refers to boards.o(.constdata) for .constdata
    boards.o(i.bsp_board_led_invert) refers to boards.o(.constdata) for .constdata
    boards.o(i.bsp_board_led_off) refers to boards.o(i.nrf_gpio_pin_write) for nrf_gpio_pin_write
    boards.o(i.bsp_board_led_off) refers to boards.o(.constdata) for .constdata
    boards.o(i.bsp_board_led_on) refers to boards.o(i.nrf_gpio_pin_write) for nrf_gpio_pin_write
    boards.o(i.bsp_board_led_on) refers to boards.o(.constdata) for .constdata
    boards.o(i.bsp_board_led_state_get) refers to boards.o(.constdata) for .constdata
    boards.o(i.bsp_board_leds_init) refers to boards.o(i.nrf_gpio_cfg) for nrf_gpio_cfg
    boards.o(i.bsp_board_leds_init) refers to boards.o(i.bsp_board_leds_off) for bsp_board_leds_off
    boards.o(i.bsp_board_leds_init) refers to boards.o(.constdata) for .constdata
    boards.o(i.bsp_board_leds_off) refers to boards.o(i.bsp_board_led_off) for bsp_board_led_off
    boards.o(i.bsp_board_leds_on) refers to boards.o(i.bsp_board_led_on) for bsp_board_led_on
    boards.o(i.bsp_board_pin_to_button_idx) refers to boards.o(.constdata) for .constdata
    boards.o(i.bsp_board_pin_to_led_idx) refers to boards.o(.constdata) for .constdata
    bsp.o(i.bsp_button_is_pressed) refers to boards.o(i.bsp_board_button_state_get) for bsp_board_button_state_get
    bsp.o(i.bsp_init) refers to boards.o(i.bsp_board_buttons_init) for bsp_board_buttons_init
    ble_advdata.o(i.adv_data_encode) refers to ble_advdata.o(i.ble_device_addr_encode) for ble_device_addr_encode
    ble_advdata.o(i.adv_data_encode) refers to ble_advdata.o(i.appearance_encode) for appearance_encode
    ble_advdata.o(i.adv_data_encode) refers to ble_advdata.o(i.flags_encode) for flags_encode
    ble_advdata.o(i.adv_data_encode) refers to ble_advdata.o(i.tx_power_level_encode) for tx_power_level_encode
    ble_advdata.o(i.adv_data_encode) refers to ble_advdata.o(i.uuid_list_encode) for uuid_list_encode
    ble_advdata.o(i.adv_data_encode) refers to ble_advdata.o(i.conn_int_encode) for conn_int_encode
    ble_advdata.o(i.adv_data_encode) refers to ble_advdata.o(i.manuf_specific_data_encode) for manuf_specific_data_encode
    ble_advdata.o(i.adv_data_encode) refers to ble_advdata.o(i.service_data_encode) for service_data_encode
    ble_advdata.o(i.adv_data_encode) refers to ble_advdata.o(i.name_encode) for name_encode
    ble_advdata.o(i.appearance_encode) refers to ble_advdata.o(i.uint16_encode) for uint16_encode
    ble_advdata.o(i.ble_advdata_set) refers to ble_advdata.o(i.advdata_check) for advdata_check
    ble_advdata.o(i.ble_advdata_set) refers to ble_advdata.o(i.adv_data_encode) for adv_data_encode
    ble_advdata.o(i.ble_advdata_set) refers to ble_advdata.o(i.srdata_check) for srdata_check
    ble_advdata.o(i.conn_int_encode) refers to ble_advdata.o(i.conn_int_check) for conn_int_check
    ble_advdata.o(i.conn_int_encode) refers to ble_advdata.o(i.uint16_encode) for uint16_encode
    ble_advdata.o(i.manuf_specific_data_encode) refers to ble_advdata.o(i.uint16_encode) for uint16_encode
    ble_advdata.o(i.manuf_specific_data_encode) refers to memcpya.o(.text) for __aeabi_memcpy
    ble_advdata.o(i.service_data_encode) refers to ble_advdata.o(i.uint16_encode) for uint16_encode
    ble_advdata.o(i.service_data_encode) refers to memcpya.o(.text) for __aeabi_memcpy
    ble_advdata.o(i.uuid_list_encode) refers to ble_advdata.o(i.uuid_list_sized_encode) for uuid_list_sized_encode
    ble_conn_params.o(i.ble_conn_params_change_conn_params) refers to ble_conn_params.o(i.is_conn_params_ok) for is_conn_params_ok
    ble_conn_params.o(i.ble_conn_params_change_conn_params) refers to ble_conn_params.o(.data) for .data
    ble_conn_params.o(i.ble_conn_params_change_conn_params) refers to ble_conn_params.o(.bss) for .bss
    ble_conn_params.o(i.ble_conn_params_init) refers to memcpya.o(.text) for __aeabi_memcpy4
    ble_conn_params.o(i.ble_conn_params_init) refers to app_timer.o(i.app_timer_create) for app_timer_create
    ble_conn_params.o(i.ble_conn_params_init) refers to ble_conn_params.o(.bss) for .bss
    ble_conn_params.o(i.ble_conn_params_init) refers to ble_conn_params.o(.data) for .data
    ble_conn_params.o(i.ble_conn_params_init) refers to ble_conn_params.o(i.update_timeout_handler) for update_timeout_handler
    ble_conn_params.o(i.ble_conn_params_init) refers to ble_conn_params.o(.constdata) for .constdata
    ble_conn_params.o(i.ble_conn_params_on_ble_evt) refers to ble_conn_params.o(i.on_write) for on_write
    ble_conn_params.o(i.ble_conn_params_on_ble_evt) refers to ble_conn_params.o(i.on_connect) for on_connect
    ble_conn_params.o(i.ble_conn_params_on_ble_evt) refers to ble_conn_params.o(i.on_disconnect) for on_disconnect
    ble_conn_params.o(i.ble_conn_params_on_ble_evt) refers to ble_conn_params.o(i.on_conn_params_update) for on_conn_params_update
    ble_conn_params.o(i.ble_conn_params_stop) refers to app_timer.o(i.app_timer_stop) for app_timer_stop
    ble_conn_params.o(i.ble_conn_params_stop) refers to ble_conn_params.o(.constdata) for .constdata
    ble_conn_params.o(i.conn_params_negotiation) refers to ble_conn_params.o(i.is_conn_params_ok) for is_conn_params_ok
    ble_conn_params.o(i.conn_params_negotiation) refers to app_timer.o(i.app_timer_start) for app_timer_start
    ble_conn_params.o(i.conn_params_negotiation) refers to ble_conn_params.o(.data) for .data
    ble_conn_params.o(i.conn_params_negotiation) refers to ble_conn_params.o(.bss) for .bss
    ble_conn_params.o(i.conn_params_negotiation) refers to ble_conn_params.o(.constdata) for .constdata
    ble_conn_params.o(i.is_conn_params_ok) refers to ble_conn_params.o(.data) for .data
    ble_conn_params.o(i.on_conn_params_update) refers to ble_conn_params.o(i.conn_params_negotiation) for conn_params_negotiation
    ble_conn_params.o(i.on_conn_params_update) refers to ble_conn_params.o(.data) for .data
    ble_conn_params.o(i.on_connect) refers to ble_conn_params.o(i.conn_params_negotiation) for conn_params_negotiation
    ble_conn_params.o(i.on_connect) refers to ble_conn_params.o(.data) for .data
    ble_conn_params.o(i.on_connect) refers to ble_conn_params.o(.bss) for .bss
    ble_conn_params.o(i.on_disconnect) refers to app_timer.o(i.app_timer_stop) for app_timer_stop
    ble_conn_params.o(i.on_disconnect) refers to ble_conn_params.o(.data) for .data
    ble_conn_params.o(i.on_disconnect) refers to ble_conn_params.o(.constdata) for .constdata
    ble_conn_params.o(i.on_disconnect) refers to ble_conn_params.o(.bss) for .bss
    ble_conn_params.o(i.on_write) refers to ble_srv_common.o(i.ble_srv_is_notification_enabled) for ble_srv_is_notification_enabled
    ble_conn_params.o(i.on_write) refers to ble_conn_params.o(i.conn_params_negotiation) for conn_params_negotiation
    ble_conn_params.o(i.on_write) refers to app_timer.o(i.app_timer_stop) for app_timer_stop
    ble_conn_params.o(i.on_write) refers to ble_conn_params.o(.bss) for .bss
    ble_conn_params.o(i.on_write) refers to ble_conn_params.o(.constdata) for .constdata
    ble_conn_params.o(i.update_timeout_handler) refers to ble_conn_params.o(.data) for .data
    ble_conn_params.o(i.update_timeout_handler) refers to ble_conn_params.o(.bss) for .bss
    ble_conn_params.o(.constdata) refers to ble_conn_params.o(.bss) for m_conn_params_timer_id_data
    ble_srv_common.o(i.ble_srv_ascii_to_utf8) refers to strlen.o(.text) for strlen
    ble_srv_common.o(i.characteristic_add) refers to ble_srv_common.o(i.set_security_req) for set_security_req
    ble_srv_common.o(i.characteristic_add) refers to memseta.o(.text) for __aeabi_memclr4
    ble_srv_common.o(i.descriptor_add) refers to memseta.o(.text) for __aeabi_memclr4
    ble_srv_common.o(i.descriptor_add) refers to ble_srv_common.o(i.set_security_req) for set_security_req
    nrf_drv_clock.o(i.POWER_CLOCK_IRQHandler) refers to nrf_drv_clock.o(i.nrf_clock_event_check) for nrf_clock_event_check
    nrf_drv_clock.o(i.POWER_CLOCK_IRQHandler) refers to nrf_drv_clock.o(i.nrf_clock_event_clear) for nrf_clock_event_clear
    nrf_drv_clock.o(i.POWER_CLOCK_IRQHandler) refers to nrf_drv_clock.o(i.clock_clk_started_notify) for clock_clk_started_notify
    nrf_drv_clock.o(i.POWER_CLOCK_IRQHandler) refers to nrf_drv_clock.o(.bss) for .bss
    nrf_drv_clock.o(i.clock_clk_started_notify) refers to nrf_drv_clock.o(i.item_dequeue) for item_dequeue
    nrf_drv_clock.o(i.clock_clk_started_notify) refers to nrf_drv_clock.o(.bss) for .bss
    nrf_drv_clock.o(i.hfclk_start) refers to softdevice_handler.o(i.softdevice_handler_is_enabled) for softdevice_handler_is_enabled
    nrf_drv_clock.o(i.hfclk_start) refers to nrf_drv_clock.o(i.nrf_clock_event_clear) for nrf_clock_event_clear
    nrf_drv_clock.o(i.hfclk_stop) refers to softdevice_handler.o(i.softdevice_handler_is_enabled) for softdevice_handler_is_enabled
    nrf_drv_clock.o(i.hfclk_stop) refers to nrf_drv_clock.o(i.nrf_clock_hf_is_running) for nrf_clock_hf_is_running
    nrf_drv_clock.o(i.hfclk_stop) refers to nrf_drv_clock.o(.bss) for .bss
    nrf_drv_clock.o(i.lfclk_start) refers to nrf_drv_clock.o(i.nrf_clock_event_clear) for nrf_clock_event_clear
    nrf_drv_clock.o(i.lfclk_stop) refers to nrf_drv_clock.o(.bss) for .bss
    nrf_drv_clock.o(i.nrf_drv_clock_hfclk_is_running) refers to softdevice_handler.o(i.softdevice_handler_is_enabled) for softdevice_handler_is_enabled
    nrf_drv_clock.o(i.nrf_drv_clock_hfclk_is_running) refers to nrf_drv_clock.o(i.nrf_clock_hf_is_running) for nrf_clock_hf_is_running
    nrf_drv_clock.o(i.nrf_drv_clock_hfclk_release) refers to app_util_platform.o(i.app_util_critical_region_enter) for app_util_critical_region_enter
    nrf_drv_clock.o(i.nrf_drv_clock_hfclk_release) refers to nrf_drv_clock.o(i.hfclk_stop) for hfclk_stop
    nrf_drv_clock.o(i.nrf_drv_clock_hfclk_release) refers to app_util_platform.o(i.app_util_critical_region_exit) for app_util_critical_region_exit
    nrf_drv_clock.o(i.nrf_drv_clock_hfclk_release) refers to nrf_drv_clock.o(.bss) for .bss
    nrf_drv_clock.o(i.nrf_drv_clock_hfclk_request) refers to app_util_platform.o(i.app_util_critical_region_enter) for app_util_critical_region_enter
    nrf_drv_clock.o(i.nrf_drv_clock_hfclk_request) refers to app_util_platform.o(i.app_util_critical_region_exit) for app_util_critical_region_exit
    nrf_drv_clock.o(i.nrf_drv_clock_hfclk_request) refers to nrf_drv_clock.o(i.item_enqueue) for item_enqueue
    nrf_drv_clock.o(i.nrf_drv_clock_hfclk_request) refers to nrf_drv_clock.o(i.hfclk_start) for hfclk_start
    nrf_drv_clock.o(i.nrf_drv_clock_hfclk_request) refers to nrf_drv_clock.o(.bss) for .bss
    nrf_drv_clock.o(i.nrf_drv_clock_init) refers to nrf_drv_common.o(i.nrf_drv_common_irq_enable) for nrf_drv_common_irq_enable
    nrf_drv_clock.o(i.nrf_drv_clock_init) refers to softdevice_handler.o(i.softdevice_handler_is_enabled) for softdevice_handler_is_enabled
    nrf_drv_clock.o(i.nrf_drv_clock_init) refers to nrf_drv_clock.o(.bss) for .bss
    nrf_drv_clock.o(i.nrf_drv_clock_init_check) refers to nrf_drv_clock.o(.bss) for .bss
    nrf_drv_clock.o(i.nrf_drv_clock_lfclk_is_running) refers to softdevice_handler.o(i.softdevice_handler_is_enabled) for softdevice_handler_is_enabled
    nrf_drv_clock.o(i.nrf_drv_clock_lfclk_release) refers to app_util_platform.o(i.app_util_critical_region_enter) for app_util_critical_region_enter
    nrf_drv_clock.o(i.nrf_drv_clock_lfclk_release) refers to nrf_drv_clock.o(i.lfclk_stop) for lfclk_stop
    nrf_drv_clock.o(i.nrf_drv_clock_lfclk_release) refers to app_util_platform.o(i.app_util_critical_region_exit) for app_util_critical_region_exit
    nrf_drv_clock.o(i.nrf_drv_clock_lfclk_release) refers to nrf_drv_clock.o(.bss) for .bss
    nrf_drv_clock.o(i.nrf_drv_clock_lfclk_request) refers to app_util_platform.o(i.app_util_critical_region_enter) for app_util_critical_region_enter
    nrf_drv_clock.o(i.nrf_drv_clock_lfclk_request) refers to app_util_platform.o(i.app_util_critical_region_exit) for app_util_critical_region_exit
    nrf_drv_clock.o(i.nrf_drv_clock_lfclk_request) refers to nrf_drv_clock.o(i.item_enqueue) for item_enqueue
    nrf_drv_clock.o(i.nrf_drv_clock_lfclk_request) refers to nrf_drv_clock.o(i.lfclk_start) for lfclk_start
    nrf_drv_clock.o(i.nrf_drv_clock_lfclk_request) refers to nrf_drv_clock.o(.bss) for .bss
    nrf_drv_clock.o(i.nrf_drv_clock_on_sd_disable) refers to nrf_drv_common.o(i.nrf_drv_common_irq_enable) for nrf_drv_common_irq_enable
    nrf_drv_clock.o(i.nrf_drv_clock_on_sd_disable) refers to nrf_drv_clock.o(i.nrf_drv_clock_lfclk_release) for nrf_drv_clock_lfclk_release
    nrf_drv_clock.o(i.nrf_drv_clock_on_sd_enable) refers to app_util_platform.o(i.app_util_critical_region_enter) for app_util_critical_region_enter
    nrf_drv_clock.o(i.nrf_drv_clock_on_sd_enable) refers to nrf_drv_clock.o(i.nrf_drv_clock_init) for nrf_drv_clock_init
    nrf_drv_clock.o(i.nrf_drv_clock_on_sd_enable) refers to app_util_platform.o(i.app_util_critical_region_exit) for app_util_critical_region_exit
    nrf_drv_clock.o(i.nrf_drv_clock_on_sd_enable) refers to nrf_drv_clock.o(.bss) for .bss
    nrf_drv_clock.o(i.nrf_drv_clock_on_soc_event) refers to nrf_drv_clock.o(i.clock_clk_started_notify) for clock_clk_started_notify
    nrf_drv_clock.o(i.nrf_drv_clock_uninit) refers to nrf_drv_common.o(i.nrf_drv_common_clock_irq_disable) for nrf_drv_common_clock_irq_disable
    nrf_drv_clock.o(i.nrf_drv_clock_uninit) refers to nrf_drv_clock.o(i.lfclk_stop) for lfclk_stop
    nrf_drv_clock.o(i.nrf_drv_clock_uninit) refers to nrf_drv_clock.o(i.hfclk_stop) for hfclk_stop
    nrf_drv_clock.o(i.nrf_drv_clock_uninit) refers to nrf_drv_clock.o(.bss) for .bss
    nrf_drv_gpiote.o(i.GPIOTE_IRQHandler) refers to nrf_drv_gpiote.o(i.nrf_gpiote_event_is_set) for nrf_gpiote_event_is_set
    nrf_drv_gpiote.o(i.GPIOTE_IRQHandler) refers to nrf_drv_gpiote.o(i.nrf_gpiote_event_clear) for nrf_gpiote_event_clear
    nrf_drv_gpiote.o(i.GPIOTE_IRQHandler) refers to nrf_drv_gpiote.o(i.nrf_gpio_ports_read) for nrf_gpio_ports_read
    nrf_drv_gpiote.o(i.GPIOTE_IRQHandler) refers to nrf_drv_gpiote.o(i.nrf_bitmask_bit_is_set) for nrf_bitmask_bit_is_set
    nrf_drv_gpiote.o(i.GPIOTE_IRQHandler) refers to nrf_drv_gpiote.o(i.channel_port_get) for channel_port_get
    nrf_drv_gpiote.o(i.GPIOTE_IRQHandler) refers to nrf_drv_gpiote.o(i.nrf_gpio_cfg_sense_set) for nrf_gpio_cfg_sense_set
    nrf_drv_gpiote.o(i.GPIOTE_IRQHandler) refers to nrf_drv_gpiote.o(.bss) for .bss
    nrf_drv_gpiote.o(i.channel_free) refers to nrf_drv_gpiote.o(.bss) for .bss
    nrf_drv_gpiote.o(i.channel_port_alloc) refers to nrf_drv_gpiote.o(.bss) for .bss
    nrf_drv_gpiote.o(i.channel_port_get) refers to nrf_drv_gpiote.o(.bss) for .bss
    nrf_drv_gpiote.o(i.nrf_drv_gpiote_clr_task_addr_get) refers to nrf_drv_gpiote.o(i.channel_port_get) for channel_port_get
    nrf_drv_gpiote.o(i.nrf_drv_gpiote_clr_task_trigger) refers to nrf_drv_gpiote.o(i.channel_port_get) for channel_port_get
    nrf_drv_gpiote.o(i.nrf_drv_gpiote_in_event_addr_get) refers to nrf_drv_gpiote.o(i.pin_in_use_by_te) for pin_in_use_by_te
    nrf_drv_gpiote.o(i.nrf_drv_gpiote_in_event_addr_get) refers to nrf_drv_gpiote.o(i.channel_port_get) for channel_port_get
    nrf_drv_gpiote.o(i.nrf_drv_gpiote_in_event_disable) refers to nrf_drv_gpiote.o(i.pin_in_use_by_port) for pin_in_use_by_port
    nrf_drv_gpiote.o(i.nrf_drv_gpiote_in_event_disable) refers to nrf_drv_gpiote.o(i.nrf_gpio_cfg_sense_set) for nrf_gpio_cfg_sense_set
    nrf_drv_gpiote.o(i.nrf_drv_gpiote_in_event_disable) refers to nrf_drv_gpiote.o(i.pin_in_use_by_te) for pin_in_use_by_te
    nrf_drv_gpiote.o(i.nrf_drv_gpiote_in_event_disable) refers to nrf_drv_gpiote.o(i.channel_port_get) for channel_port_get
    nrf_drv_gpiote.o(i.nrf_drv_gpiote_in_event_enable) refers to nrf_drv_gpiote.o(i.pin_in_use_by_port) for pin_in_use_by_port
    nrf_drv_gpiote.o(i.nrf_drv_gpiote_in_event_enable) refers to nrf_drv_gpiote.o(i.channel_port_get) for channel_port_get
    nrf_drv_gpiote.o(i.nrf_drv_gpiote_in_event_enable) refers to nrf_drv_gpiote.o(i.nrf_gpio_cfg_sense_set) for nrf_gpio_cfg_sense_set
    nrf_drv_gpiote.o(i.nrf_drv_gpiote_in_event_enable) refers to nrf_drv_gpiote.o(i.pin_in_use_by_te) for pin_in_use_by_te
    nrf_drv_gpiote.o(i.nrf_drv_gpiote_in_event_enable) refers to nrf_drv_gpiote.o(i.nrf_gpiote_event_clear) for nrf_gpiote_event_clear
    nrf_drv_gpiote.o(i.nrf_drv_gpiote_in_event_enable) refers to nrf_drv_gpiote.o(.bss) for .bss
    nrf_drv_gpiote.o(i.nrf_drv_gpiote_in_init) refers to nrf_drv_gpiote.o(i.channel_port_alloc) for channel_port_alloc
    nrf_drv_gpiote.o(i.nrf_drv_gpiote_in_init) refers to nrf_drv_gpiote.o(i.nrf_gpio_cfg) for nrf_gpio_cfg
    nrf_drv_gpiote.o(i.nrf_drv_gpiote_in_init) refers to nrf_drv_gpiote.o(.bss) for .bss
    nrf_drv_gpiote.o(i.nrf_drv_gpiote_in_uninit) refers to nrf_drv_gpiote.o(i.nrf_drv_gpiote_in_event_disable) for nrf_drv_gpiote_in_event_disable
    nrf_drv_gpiote.o(i.nrf_drv_gpiote_in_uninit) refers to nrf_drv_gpiote.o(i.pin_in_use_by_te) for pin_in_use_by_te
    nrf_drv_gpiote.o(i.nrf_drv_gpiote_in_uninit) refers to nrf_drv_gpiote.o(i.channel_port_get) for channel_port_get
    nrf_drv_gpiote.o(i.nrf_drv_gpiote_in_uninit) refers to nrf_drv_gpiote.o(i.nrf_gpio_cfg_default) for nrf_gpio_cfg_default
    nrf_drv_gpiote.o(i.nrf_drv_gpiote_in_uninit) refers to nrf_drv_gpiote.o(i.channel_free) for channel_free
    nrf_drv_gpiote.o(i.nrf_drv_gpiote_in_uninit) refers to nrf_drv_gpiote.o(.bss) for .bss
    nrf_drv_gpiote.o(i.nrf_drv_gpiote_init) refers to nrf_drv_gpiote.o(i.channel_free) for channel_free
    nrf_drv_gpiote.o(i.nrf_drv_gpiote_init) refers to nrf_drv_common.o(i.nrf_drv_common_irq_enable) for nrf_drv_common_irq_enable
    nrf_drv_gpiote.o(i.nrf_drv_gpiote_init) refers to nrf_drv_gpiote.o(i.nrf_gpiote_event_clear) for nrf_gpiote_event_clear
    nrf_drv_gpiote.o(i.nrf_drv_gpiote_init) refers to nrf_drv_gpiote.o(.bss) for .bss
    nrf_drv_gpiote.o(i.nrf_drv_gpiote_is_init) refers to nrf_drv_gpiote.o(.bss) for .bss
    nrf_drv_gpiote.o(i.nrf_drv_gpiote_out_init) refers to nrf_drv_gpiote.o(i.channel_port_alloc) for channel_port_alloc
    nrf_drv_gpiote.o(i.nrf_drv_gpiote_out_init) refers to nrf_drv_gpiote.o(i.nrf_gpio_cfg) for nrf_gpio_cfg
    nrf_drv_gpiote.o(i.nrf_drv_gpiote_out_init) refers to nrf_drv_gpiote.o(.bss) for .bss
    nrf_drv_gpiote.o(i.nrf_drv_gpiote_out_task_addr_get) refers to nrf_drv_gpiote.o(i.channel_port_get) for channel_port_get
    nrf_drv_gpiote.o(i.nrf_drv_gpiote_out_task_disable) refers to nrf_drv_gpiote.o(.bss) for .bss
    nrf_drv_gpiote.o(i.nrf_drv_gpiote_out_task_enable) refers to nrf_drv_gpiote.o(.bss) for .bss
    nrf_drv_gpiote.o(i.nrf_drv_gpiote_out_task_force) refers to nrf_drv_gpiote.o(.bss) for .bss
    nrf_drv_gpiote.o(i.nrf_drv_gpiote_out_task_trigger) refers to nrf_drv_gpiote.o(i.channel_port_get) for channel_port_get
    nrf_drv_gpiote.o(i.nrf_drv_gpiote_out_uninit) refers to nrf_drv_gpiote.o(i.pin_in_use_by_te) for pin_in_use_by_te
    nrf_drv_gpiote.o(i.nrf_drv_gpiote_out_uninit) refers to nrf_drv_gpiote.o(i.channel_port_get) for channel_port_get
    nrf_drv_gpiote.o(i.nrf_drv_gpiote_out_uninit) refers to nrf_drv_gpiote.o(i.channel_free) for channel_free
    nrf_drv_gpiote.o(i.nrf_drv_gpiote_out_uninit) refers to nrf_drv_gpiote.o(i.nrf_gpio_cfg_default) for nrf_gpio_cfg_default
    nrf_drv_gpiote.o(i.nrf_drv_gpiote_out_uninit) refers to nrf_drv_gpiote.o(.bss) for .bss
    nrf_drv_gpiote.o(i.nrf_drv_gpiote_set_task_addr_get) refers to nrf_drv_gpiote.o(i.channel_port_get) for channel_port_get
    nrf_drv_gpiote.o(i.nrf_drv_gpiote_set_task_trigger) refers to nrf_drv_gpiote.o(i.channel_port_get) for channel_port_get
    nrf_drv_gpiote.o(i.nrf_drv_gpiote_uninit) refers to nrf_drv_gpiote.o(i.nrf_drv_gpiote_out_uninit) for nrf_drv_gpiote_out_uninit
    nrf_drv_gpiote.o(i.nrf_drv_gpiote_uninit) refers to nrf_drv_gpiote.o(i.nrf_drv_gpiote_in_uninit) for nrf_drv_gpiote_in_uninit
    nrf_drv_gpiote.o(i.nrf_drv_gpiote_uninit) refers to nrf_drv_gpiote.o(.bss) for .bss
    nrf_drv_gpiote.o(i.nrf_gpio_cfg_default) refers to nrf_drv_gpiote.o(i.nrf_gpio_cfg) for nrf_gpio_cfg
    nrf_drv_gpiote.o(i.nrf_gpio_ports_read) refers to nrf_drv_gpiote.o(.constdata) for .constdata
    nrf_drv_gpiote.o(i.pin_in_use_by_port) refers to nrf_drv_gpiote.o(.bss) for .bss
    nrf_drv_gpiote.o(i.pin_in_use_by_te) refers to nrf_drv_gpiote.o(.bss) for .bss
    nrf_drv_twi.o(i.SPIM0_SPIS0_TWIM0_TWIS0_SPI0_TWI0_IRQHandler) refers to nrf_drv_twi.o(i.irq_handler_twim) for irq_handler_twim
    nrf_drv_twi.o(i.SPIM0_SPIS0_TWIM0_TWIS0_SPI0_TWI0_IRQHandler) refers to nrf_drv_twi.o(.bss) for .bss
    nrf_drv_twi.o(i.irq_handler_twim) refers to nrf_drv_twi.o(i.nrf_twim_event_check) for nrf_twim_event_check
    nrf_drv_twi.o(i.irq_handler_twim) refers to nrf_drv_twi.o(i.nrf_twim_event_clear) for nrf_twim_event_clear
    nrf_drv_twi.o(i.irq_handler_twim) refers to nrf_drv_twi.o(i.twim_list_enable_handle) for twim_list_enable_handle
    nrf_drv_twi.o(i.nrf_delay_us) refers to system_nrf52.o(.data) for SystemCoreClock
    nrf_drv_twi.o(i.nrf_drv_twi_disable) refers to nrf_drv_twi.o(.bss) for .bss
    nrf_drv_twi.o(i.nrf_drv_twi_enable) refers to nrf_drv_twi.o(.bss) for .bss
    nrf_drv_twi.o(i.nrf_drv_twi_init) refers to nrf_drv_twi.o(i.twi_clear_bus) for twi_clear_bus
    nrf_drv_twi.o(i.nrf_drv_twi_init) refers to nrf_drv_common.o(i.nrf_drv_common_irq_enable) for nrf_drv_common_irq_enable
    nrf_drv_twi.o(i.nrf_drv_twi_init) refers to nrf_drv_twi.o(.bss) for .bss
    nrf_drv_twi.o(i.nrf_drv_twi_is_busy) refers to nrf_drv_twi.o(.bss) for .bss
    nrf_drv_twi.o(i.nrf_drv_twi_rx) refers to nrf_drv_twi.o(i.nrf_drv_twi_xfer) for nrf_drv_twi_xfer
    nrf_drv_twi.o(i.nrf_drv_twi_rx) refers to nrf_drv_twi.o(.constdata) for .constdata
    nrf_drv_twi.o(i.nrf_drv_twi_tx) refers to nrf_drv_twi.o(i.nrf_drv_twi_xfer) for nrf_drv_twi_xfer
    nrf_drv_twi.o(i.nrf_drv_twi_uninit) refers to nrf_drv_twi.o(i.nrf_drv_twi_disable) for nrf_drv_twi_disable
    nrf_drv_twi.o(i.nrf_drv_twi_uninit) refers to nrf_drv_twi.o(.bss) for .bss
    nrf_drv_twi.o(i.nrf_drv_twi_xfer) refers to nrf_drv_twi.o(i.twim_xfer) for twim_xfer
    nrf_drv_twi.o(i.nrf_drv_twi_xfer) refers to nrf_drv_twi.o(.bss) for .bss
    nrf_drv_twi.o(i.twi_clear_bus) refers to nrf_drv_twi.o(i.nrf_gpio_pin_set) for nrf_gpio_pin_set
    nrf_drv_twi.o(i.twi_clear_bus) refers to nrf_drv_twi.o(i.nrf_delay_us) for nrf_delay_us
    nrf_drv_twi.o(i.twim_xfer) refers to nrf_drv_twi.o(i.nrf_drv_is_in_RAM) for nrf_drv_is_in_RAM
    nrf_drv_twi.o(i.twim_xfer) refers to nrf_drv_twi.o(i.nrf_twim_event_clear) for nrf_twim_event_clear
    nrf_drv_twi.o(i.twim_xfer) refers to nrf_drv_twi.o(i.twim_list_enable_handle) for twim_list_enable_handle
    nrf_drv_twi.o(i.twim_xfer) refers to nrf_drv_twi.o(i.nrf_twim_event_check) for nrf_twim_event_check
    nrf_drv_twi.o(i.twim_xfer) refers to nrf_drv_twi.o(i.twi_process_error) for twi_process_error
    app_button.o(i.app_button_disable) refers to nrf_drv_gpiote.o(i.nrf_drv_gpiote_in_event_disable) for nrf_drv_gpiote_in_event_disable
    app_button.o(i.app_button_disable) refers to app_timer.o(i.app_timer_stop) for app_timer_stop
    app_button.o(i.app_button_disable) refers to app_button.o(.data) for .data
    app_button.o(i.app_button_disable) refers to app_button.o(.constdata) for .constdata
    app_button.o(i.app_button_enable) refers to nrf_drv_gpiote.o(i.nrf_drv_gpiote_in_event_enable) for nrf_drv_gpiote_in_event_enable
    app_button.o(i.app_button_enable) refers to app_button.o(.data) for .data
    app_button.o(i.app_button_init) refers to nrf_drv_gpiote.o(i.nrf_drv_gpiote_is_init) for nrf_drv_gpiote_is_init
    app_button.o(i.app_button_init) refers to nrf_drv_gpiote.o(i.nrf_drv_gpiote_init) for nrf_drv_gpiote_init
    app_button.o(i.app_button_init) refers to nrf_drv_gpiote.o(i.nrf_drv_gpiote_in_init) for nrf_drv_gpiote_in_init
    app_button.o(i.app_button_init) refers to app_timer.o(i.app_timer_create) for app_timer_create
    app_button.o(i.app_button_init) refers to app_button.o(.data) for .data
    app_button.o(i.app_button_init) refers to app_button.o(.constdata) for .constdata
    app_button.o(i.app_button_init) refers to app_button.o(i.gpiote_event_handler) for gpiote_event_handler
    app_button.o(i.app_button_init) refers to app_button.o(i.detection_delay_timeout_handler) for detection_delay_timeout_handler
    app_button.o(i.app_button_is_pushed) refers to nrf_drv_gpiote.o(i.nrf_drv_gpiote_in_is_set) for nrf_drv_gpiote_in_is_set
    app_button.o(i.app_button_is_pushed) refers to app_button.o(.data) for .data
    app_button.o(i.detection_delay_timeout_handler) refers to nrf_drv_gpiote.o(i.nrf_drv_gpiote_in_is_set) for nrf_drv_gpiote_in_is_set
    app_button.o(i.detection_delay_timeout_handler) refers to app_button.o(.data) for .data
    app_button.o(i.gpiote_event_handler) refers to app_timer.o(i.app_timer_stop) for app_timer_stop
    app_button.o(i.gpiote_event_handler) refers to nrf_drv_gpiote.o(i.nrf_drv_gpiote_in_is_set) for nrf_drv_gpiote_in_is_set
    app_button.o(i.gpiote_event_handler) refers to app_timer.o(i.app_timer_start) for app_timer_start
    app_button.o(i.gpiote_event_handler) refers to app_button.o(.constdata) for .constdata
    app_button.o(i.gpiote_event_handler) refers to app_button.o(.data) for .data
    app_button.o(.constdata) refers to app_button.o(.bss) for m_detection_delay_timer_id_data
    app_error.o(i.app_error_handler) refers to app_error_weak.o(i.app_error_fault_handler) for app_error_fault_handler
    app_error.o(i.app_error_handler_bare) refers to app_error_weak.o(i.app_error_fault_handler) for app_error_fault_handler
    app_error.o(i.app_error_save_and_stop) refers to app_error.o(.bss) for .bss
    app_error_weak.o(i.app_error_fault_handler) refers to nrf_log_frontend.o(i.nrf_log_frontend_std_0) for nrf_log_frontend_std_0
    app_scheduler.o(i.app_sched_event_put) refers to app_util_platform.o(i.app_util_critical_region_enter) for app_util_critical_region_enter
    app_scheduler.o(i.app_sched_event_put) refers to app_scheduler.o(i.next_index) for next_index
    app_scheduler.o(i.app_sched_event_put) refers to app_util_platform.o(i.app_util_critical_region_exit) for app_util_critical_region_exit
    app_scheduler.o(i.app_sched_event_put) refers to memcpya.o(.text) for __aeabi_memcpy
    app_scheduler.o(i.app_sched_event_put) refers to app_scheduler.o(.data) for .data
    app_scheduler.o(i.app_sched_execute) refers to app_scheduler.o(i.next_index) for next_index
    app_scheduler.o(i.app_sched_execute) refers to app_scheduler.o(.data) for .data
    app_scheduler.o(i.app_sched_init) refers to app_scheduler.o(.data) for .data
    app_scheduler.o(i.app_sched_queue_space_get) refers to app_scheduler.o(.data) for .data
    app_scheduler.o(i.next_index) refers to app_scheduler.o(.data) for .data
    app_timer.o(i.RTC1_IRQHandler) refers to app_timer.o(i.timer_timeouts_check) for timer_timeouts_check
    app_timer.o(i.SWI0_EGU0_IRQHandler) refers to app_timer.o(i.timer_list_handler) for timer_list_handler
    app_timer.o(i.app_timer_create) refers to app_timer.o(.bss) for .bss
    app_timer.o(i.app_timer_init) refers to app_timer.o(i.rtc1_stop) for rtc1_stop
    app_timer.o(i.app_timer_init) refers to app_timer.o(i.__NVIC_ClearPendingIRQ) for __NVIC_ClearPendingIRQ
    app_timer.o(i.app_timer_init) refers to app_timer.o(i.__NVIC_SetPriority) for __NVIC_SetPriority
    app_timer.o(i.app_timer_init) refers to app_timer.o(i.__NVIC_EnableIRQ) for __NVIC_EnableIRQ
    app_timer.o(i.app_timer_init) refers to app_timer.o(i.rtc1_init) for rtc1_init
    app_timer.o(i.app_timer_init) refers to app_timer.o(.bss) for .bss
    app_timer.o(i.app_timer_init) refers to app_timer.o(.data) for .data
    app_timer.o(i.app_timer_start) refers to app_timer.o(i.timer_start_op_schedule) for timer_start_op_schedule
    app_timer.o(i.app_timer_start) refers to app_timer.o(.bss) for .bss
    app_timer.o(i.app_timer_stop) refers to app_timer.o(i.timer_stop_op_schedule) for timer_stop_op_schedule
    app_timer.o(i.app_timer_stop) refers to app_timer.o(.bss) for .bss
    app_timer.o(i.app_timer_stop_all) refers to app_timer.o(i.timer_stop_op_schedule) for timer_stop_op_schedule
    app_timer.o(i.app_timer_stop_all) refers to app_timer.o(.bss) for .bss
    app_timer.o(i.compare_reg_update) refers to app_timer.o(i.rtc1_start) for rtc1_start
    app_timer.o(i.compare_reg_update) refers to app_timer.o(i.nrf_delay_us) for nrf_delay_us
    app_timer.o(i.compare_reg_update) refers to app_timer.o(i.timer_timeouts_check_sched) for timer_timeouts_check_sched
    app_timer.o(i.compare_reg_update) refers to app_timer.o(i.rtc1_stop) for rtc1_stop
    app_timer.o(i.compare_reg_update) refers to app_timer.o(.data) for .data
    app_timer.o(i.elapsed_ticks_acquire) refers to app_timer.o(.data) for .data
    app_timer.o(i.expired_timers_handler) refers to app_timer.o(.data) for .data
    app_timer.o(i.list_insertions_handler) refers to app_timer.o(i.timer_list_remove) for timer_list_remove
    app_timer.o(i.list_insertions_handler) refers to app_timer.o(i.timer_list_insert) for timer_list_insert
    app_timer.o(i.list_insertions_handler) refers to app_timer.o(.data) for .data
    app_timer.o(i.list_insertions_handler) refers to app_timer.o(.bss) for .bss
    app_timer.o(i.nrf_delay_us) refers to system_nrf52.o(.data) for SystemCoreClock
    app_timer.o(i.rtc1_init) refers to app_timer.o(i.__NVIC_SetPriority) for __NVIC_SetPriority
    app_timer.o(i.rtc1_start) refers to app_timer.o(i.__NVIC_ClearPendingIRQ) for __NVIC_ClearPendingIRQ
    app_timer.o(i.rtc1_start) refers to app_timer.o(i.__NVIC_EnableIRQ) for __NVIC_EnableIRQ
    app_timer.o(i.rtc1_start) refers to app_timer.o(i.nrf_delay_us) for nrf_delay_us
    app_timer.o(i.rtc1_start) refers to app_timer.o(.data) for .data
    app_timer.o(i.rtc1_stop) refers to app_timer.o(i.nrf_delay_us) for nrf_delay_us
    app_timer.o(i.rtc1_stop) refers to app_timer.o(.data) for .data
    app_timer.o(i.timer_list_handler) refers to app_timer.o(i.elapsed_ticks_acquire) for elapsed_ticks_acquire
    app_timer.o(i.timer_list_handler) refers to app_timer.o(i.expired_timers_handler) for expired_timers_handler
    app_timer.o(i.timer_list_handler) refers to app_timer.o(i.list_insertions_handler) for list_insertions_handler
    app_timer.o(i.timer_list_handler) refers to app_timer.o(i.compare_reg_update) for compare_reg_update
    app_timer.o(i.timer_list_handler) refers to app_timer.o(.data) for .data
    app_timer.o(i.timer_list_handler_sched) refers to app_timer.o(i.__NVIC_SetPendingIRQ) for __NVIC_SetPendingIRQ
    app_timer.o(i.timer_list_insert) refers to app_timer.o(.data) for .data
    app_timer.o(i.timer_list_remove) refers to app_timer.o(i.nrf_delay_us) for nrf_delay_us
    app_timer.o(i.timer_list_remove) refers to app_timer.o(.data) for .data
    app_timer.o(i.timer_start_op_schedule) refers to app_util_platform.o(i.app_util_critical_region_enter) for app_util_critical_region_enter
    app_timer.o(i.timer_start_op_schedule) refers to app_timer.o(i.user_op_alloc) for user_op_alloc
    app_timer.o(i.timer_start_op_schedule) refers to app_timer.o(i.user_op_enque) for user_op_enque
    app_timer.o(i.timer_start_op_schedule) refers to app_util_platform.o(i.app_util_critical_region_exit) for app_util_critical_region_exit
    app_timer.o(i.timer_start_op_schedule) refers to app_timer.o(i.timer_list_handler_sched) for timer_list_handler_sched
    app_timer.o(i.timer_stop_op_schedule) refers to app_util_platform.o(i.app_util_critical_region_enter) for app_util_critical_region_enter
    app_timer.o(i.timer_stop_op_schedule) refers to app_timer.o(i.user_op_alloc) for user_op_alloc
    app_timer.o(i.timer_stop_op_schedule) refers to app_timer.o(i.user_op_enque) for user_op_enque
    app_timer.o(i.timer_stop_op_schedule) refers to app_util_platform.o(i.app_util_critical_region_exit) for app_util_critical_region_exit
    app_timer.o(i.timer_stop_op_schedule) refers to app_timer.o(i.timer_list_handler_sched) for timer_list_handler_sched
    app_timer.o(i.timer_timeouts_check) refers to app_timer.o(i.timeout_handler_exec) for timeout_handler_exec
    app_timer.o(i.timer_timeouts_check) refers to app_timer.o(i.timer_list_handler_sched) for timer_list_handler_sched
    app_timer.o(i.timer_timeouts_check) refers to app_timer.o(.data) for .data
    app_timer.o(i.timer_timeouts_check_sched) refers to app_timer.o(i.__NVIC_SetPendingIRQ) for __NVIC_SetPendingIRQ
    app_timer.o(i.user_op_alloc) refers to app_timer.o(.bss) for .bss
    app_timer.o(i.user_op_enque) refers to app_timer.o(.bss) for .bss
    app_util_platform.o(i.app_util_critical_region_enter) refers to app_util_platform.o(.bss) for .bss
    app_util_platform.o(i.app_util_critical_region_exit) refers to app_util_platform.o(.bss) for .bss
    app_util_platform.o(i.app_util_disable_irq) refers to app_util_platform.o(.data) for .data
    app_util_platform.o(i.app_util_enable_irq) refers to app_util_platform.o(.data) for .data
    nrf_assert.o(i.assert_nrf_callback) refers to app_error_weak.o(i.app_error_fault_handler) for app_error_fault_handler
    nrf_strerror.o(i.nrf_strerror_find) refers to nrf_strerror.o(.constdata) for .constdata
    nrf_strerror.o(i.nrf_strerror_get) refers to nrf_strerror.o(i.nrf_strerror_find) for nrf_strerror_find
    nrf_strerror.o(i.nrf_strerror_get) refers to nrf_strerror.o(.constdata) for .constdata
    nrf_strerror.o(.constdata) refers to nrf_strerror.o(.conststring) for .conststring
    app_twi.o(i.app_twi_init) refers to nrf_drv_twi.o(i.nrf_drv_twi_init) for nrf_drv_twi_init
    app_twi.o(i.app_twi_init) refers to nrf_drv_twi.o(i.nrf_drv_twi_enable) for nrf_drv_twi_enable
    app_twi.o(i.app_twi_init) refers to app_twi.o(i.twi_event_handler) for twi_event_handler
    app_twi.o(i.app_twi_perform) refers to app_util_platform.o(i.app_util_critical_region_enter) for app_util_critical_region_enter
    app_twi.o(i.app_twi_perform) refers to app_util_platform.o(i.app_util_critical_region_exit) for app_util_critical_region_exit
    app_twi.o(i.app_twi_perform) refers to memcpya.o(.text) for __aeabi_memcpy4
    app_twi.o(i.app_twi_perform) refers to app_twi.o(i.app_twi_schedule) for app_twi_schedule
    app_twi.o(i.app_twi_perform) refers to app_twi.o(.constdata) for .constdata
    app_twi.o(i.app_twi_schedule) refers to nrf_queue.o(i.nrf_queue_push) for nrf_queue_push
    app_twi.o(i.app_twi_schedule) refers to app_twi.o(i.start_pending_transaction) for start_pending_transaction
    app_twi.o(i.app_twi_uninit) refers to nrf_drv_twi.o(i.nrf_drv_twi_uninit) for nrf_drv_twi_uninit
    app_twi.o(i.start_pending_transaction) refers to app_util_platform.o(i.app_util_critical_region_enter) for app_util_critical_region_enter
    app_twi.o(i.start_pending_transaction) refers to nrf_queue.o(i.nrf_queue_generic_pop) for nrf_queue_generic_pop
    app_twi.o(i.start_pending_transaction) refers to app_util_platform.o(i.app_util_critical_region_exit) for app_util_critical_region_exit
    app_twi.o(i.start_pending_transaction) refers to memcmp.o(.text) for memcmp
    app_twi.o(i.start_pending_transaction) refers to nrf_drv_twi.o(i.nrf_drv_twi_uninit) for nrf_drv_twi_uninit
    app_twi.o(i.start_pending_transaction) refers to nrf_drv_twi.o(i.nrf_drv_twi_init) for nrf_drv_twi_init
    app_twi.o(i.start_pending_transaction) refers to nrf_drv_twi.o(i.nrf_drv_twi_enable) for nrf_drv_twi_enable
    app_twi.o(i.start_pending_transaction) refers to app_twi.o(i.start_transfer) for start_transfer
    app_twi.o(i.start_pending_transaction) refers to app_twi.o(i.transaction_end_signal) for transaction_end_signal
    app_twi.o(i.start_pending_transaction) refers to app_twi.o(i.twi_event_handler) for twi_event_handler
    app_twi.o(i.start_transfer) refers to nrf_drv_twi.o(i.nrf_drv_twi_xfer) for nrf_drv_twi_xfer
    app_twi.o(i.twi_event_handler) refers to app_twi.o(i.transaction_end_signal) for transaction_end_signal
    app_twi.o(i.twi_event_handler) refers to app_twi.o(i.start_pending_transaction) for start_pending_transaction
    app_twi.o(i.twi_event_handler) refers to app_twi.o(i.start_transfer) for start_transfer
    app_twi.o(.constdata) refers to app_twi.o(i.internal_transaction_cb) for internal_transaction_cb
    nrf_queue.o(i.nrf_queue_available_get) refers to nrf_queue.o(i.nrf_queue_utilization_get) for nrf_queue_utilization_get
    nrf_queue.o(i.nrf_queue_generic_pop) refers to app_util_platform.o(i.app_util_critical_region_enter) for app_util_critical_region_enter
    nrf_queue.o(i.nrf_queue_generic_pop) refers to nrf_queue.o(i.nrf_queue_is_empty) for nrf_queue_is_empty
    nrf_queue.o(i.nrf_queue_generic_pop) refers to app_util_platform.o(i.app_util_critical_region_exit) for app_util_critical_region_exit
    nrf_queue.o(i.nrf_queue_generic_pop) refers to nrf_queue.o(i.nrf_queue_next_idx) for nrf_queue_next_idx
    nrf_queue.o(i.nrf_queue_generic_pop) refers to memcpya.o(.text) for __aeabi_memcpy
    nrf_queue.o(i.nrf_queue_in) refers to app_util_platform.o(i.app_util_critical_region_enter) for app_util_critical_region_enter
    nrf_queue.o(i.nrf_queue_in) refers to nrf_queue.o(i.nrf_queue_available_get) for nrf_queue_available_get
    nrf_queue.o(i.nrf_queue_in) refers to nrf_queue.o(i.queue_write) for queue_write
    nrf_queue.o(i.nrf_queue_in) refers to app_util_platform.o(i.app_util_critical_region_exit) for app_util_critical_region_exit
    nrf_queue.o(i.nrf_queue_is_full) refers to nrf_queue.o(i.nrf_queue_next_idx) for nrf_queue_next_idx
    nrf_queue.o(i.nrf_queue_out) refers to app_util_platform.o(i.app_util_critical_region_enter) for app_util_critical_region_enter
    nrf_queue.o(i.nrf_queue_out) refers to nrf_queue.o(i.queue_utilization_get) for queue_utilization_get
    nrf_queue.o(i.nrf_queue_out) refers to nrf_queue.o(i.queue_read) for queue_read
    nrf_queue.o(i.nrf_queue_out) refers to app_util_platform.o(i.app_util_critical_region_exit) for app_util_critical_region_exit
    nrf_queue.o(i.nrf_queue_push) refers to app_util_platform.o(i.app_util_critical_region_enter) for app_util_critical_region_enter
    nrf_queue.o(i.nrf_queue_push) refers to nrf_queue.o(i.nrf_queue_is_full) for nrf_queue_is_full
    nrf_queue.o(i.nrf_queue_push) refers to app_util_platform.o(i.app_util_critical_region_exit) for app_util_critical_region_exit
    nrf_queue.o(i.nrf_queue_push) refers to nrf_queue.o(i.nrf_queue_next_idx) for nrf_queue_next_idx
    nrf_queue.o(i.nrf_queue_push) refers to memcpya.o(.text) for __aeabi_memcpy
    nrf_queue.o(i.nrf_queue_push) refers to nrf_queue.o(i.queue_utilization_get) for queue_utilization_get
    nrf_queue.o(i.nrf_queue_read) refers to app_util_platform.o(i.app_util_critical_region_enter) for app_util_critical_region_enter
    nrf_queue.o(i.nrf_queue_read) refers to nrf_queue.o(i.queue_utilization_get) for queue_utilization_get
    nrf_queue.o(i.nrf_queue_read) refers to nrf_queue.o(i.queue_read) for queue_read
    nrf_queue.o(i.nrf_queue_read) refers to app_util_platform.o(i.app_util_critical_region_exit) for app_util_critical_region_exit
    nrf_queue.o(i.nrf_queue_reset) refers to app_util_platform.o(i.app_util_critical_region_enter) for app_util_critical_region_enter
    nrf_queue.o(i.nrf_queue_reset) refers to app_util_platform.o(i.app_util_critical_region_exit) for app_util_critical_region_exit
    nrf_queue.o(i.nrf_queue_utilization_get) refers to app_util_platform.o(i.app_util_critical_region_enter) for app_util_critical_region_enter
    nrf_queue.o(i.nrf_queue_utilization_get) refers to nrf_queue.o(i.queue_utilization_get) for queue_utilization_get
    nrf_queue.o(i.nrf_queue_utilization_get) refers to app_util_platform.o(i.app_util_critical_region_exit) for app_util_critical_region_exit
    nrf_queue.o(i.nrf_queue_write) refers to app_util_platform.o(i.app_util_critical_region_enter) for app_util_critical_region_enter
    nrf_queue.o(i.nrf_queue_write) refers to nrf_queue.o(i.nrf_queue_available_get) for nrf_queue_available_get
    nrf_queue.o(i.nrf_queue_write) refers to app_util_platform.o(i.app_util_critical_region_exit) for app_util_critical_region_exit
    nrf_queue.o(i.nrf_queue_write) refers to nrf_queue.o(i.queue_write) for queue_write
    nrf_queue.o(i.queue_read) refers to memcpya.o(.text) for __aeabi_memcpy
    nrf_queue.o(i.queue_write) refers to nrf_queue.o(i.nrf_queue_available_get) for nrf_queue_available_get
    nrf_queue.o(i.queue_write) refers to memcpya.o(.text) for __aeabi_memcpy
    nrf_queue.o(i.queue_write) refers to nrf_queue.o(i.nrf_queue_next_idx) for nrf_queue_next_idx
    nrf_queue.o(i.queue_write) refers to nrf_queue.o(i.queue_utilization_get) for queue_utilization_get
    nrf_log_backend_serial.o(i.nrf_log_backend_getchar) refers to nrf_log_backend_serial.o(i.serial_get_byte) for serial_get_byte
    nrf_log_backend_serial.o(i.nrf_log_backend_hexdump_handler_get) refers to nrf_log_backend_serial.o(i.nrf_log_backend_serial_hexdump_handler) for nrf_log_backend_serial_hexdump_handler
    nrf_log_backend_serial.o(i.nrf_log_backend_init) refers to segger_rtt.o(i.SEGGER_RTT_Init) for SEGGER_RTT_Init
    nrf_log_backend_serial.o(i.nrf_log_backend_init) refers to nrf_log_backend_serial.o(.data) for .data
    nrf_log_backend_serial.o(i.nrf_log_backend_serial_hexdump_handler) refers to nrf_log_backend_serial.o(i.serial_is_busy) for serial_is_busy
    nrf_log_backend_serial.o(i.nrf_log_backend_serial_hexdump_handler) refers to nrf_log_backend_serial.o(i.timestamp_process) for timestamp_process
    nrf_log_backend_serial.o(i.nrf_log_backend_serial_hexdump_handler) refers to strlen.o(.text) for strlen
    nrf_log_backend_serial.o(i.nrf_log_backend_serial_hexdump_handler) refers to memcpya.o(.text) for __aeabi_memcpy
    nrf_log_backend_serial.o(i.nrf_log_backend_serial_hexdump_handler) refers to nrf_log_backend_serial.o(i.byte2hex) for byte2hex
    nrf_log_backend_serial.o(i.nrf_log_backend_serial_hexdump_handler) refers to ctype_o.o(.text) for __rt_ctype_table
    nrf_log_backend_serial.o(i.nrf_log_backend_serial_hexdump_handler) refers to nrf_log_backend_serial.o(i.serial_tx) for serial_tx
    nrf_log_backend_serial.o(i.nrf_log_backend_serial_std_handler) refers to nrf_log_backend_serial.o(i.serial_is_busy) for serial_is_busy
    nrf_log_backend_serial.o(i.nrf_log_backend_serial_std_handler) refers to nrf_log_backend_serial.o(i.timestamp_process) for timestamp_process
    nrf_log_backend_serial.o(i.nrf_log_backend_serial_std_handler) refers to strlen.o(.text) for strlen
    nrf_log_backend_serial.o(i.nrf_log_backend_serial_std_handler) refers to memcpya.o(.text) for __aeabi_memcpy
    nrf_log_backend_serial.o(i.nrf_log_backend_serial_std_handler) refers to printf8.o(i.__0snprintf$8) for __2snprintf
    nrf_log_backend_serial.o(i.nrf_log_backend_serial_std_handler) refers to nrf_log_backend_serial.o(i.buf_len_update) for buf_len_update
    nrf_log_backend_serial.o(i.nrf_log_backend_serial_std_handler) refers to nrf_log_backend_serial.o(i.serial_tx) for serial_tx
    nrf_log_backend_serial.o(i.nrf_log_backend_std_handler_get) refers to nrf_log_backend_serial.o(i.nrf_log_backend_serial_std_handler) for nrf_log_backend_serial_std_handler
    nrf_log_backend_serial.o(i.serial_get_byte) refers to segger_rtt.o(i.SEGGER_RTT_WaitKey) for SEGGER_RTT_WaitKey
    nrf_log_backend_serial.o(i.serial_tx) refers to segger_rtt.o(i.SEGGER_RTT_WriteNoLock) for SEGGER_RTT_WriteNoLock
    nrf_log_backend_serial.o(i.timestamp_process) refers to printf8.o(i.__0snprintf$8) for __2snprintf
    nrf_log_backend_serial.o(i.timestamp_process) refers to nrf_log_backend_serial.o(i.buf_len_update) for buf_len_update
    nrf_log_frontend.o(i.buffer_is_empty) refers to nrf_log_frontend.o(.bss) for .bss
    nrf_log_frontend.o(i.nrf_log_blocking_backend_set) refers to nrf_log_backend_serial.o(i.nrf_log_backend_init) for nrf_log_backend_init
    nrf_log_frontend.o(i.nrf_log_direct_feed) refers to nrf_log_frontend.o(.bss) for .bss
    nrf_log_frontend.o(i.nrf_log_frontend_dequeue) refers to nrf_log_frontend.o(i.buffer_is_empty) for buffer_is_empty
    nrf_log_frontend.o(i.nrf_log_frontend_dequeue) refers to nrf_log_frontend.o(.bss) for .bss
    nrf_log_frontend.o(i.nrf_log_frontend_hexdump) refers to nrf_log_frontend.o(.bss) for .bss
    nrf_log_frontend.o(i.nrf_log_frontend_init) refers to nrf_log_frontend.o(i.nrf_log_handlers_set) for nrf_log_handlers_set
    nrf_log_frontend.o(i.nrf_log_frontend_std_0) refers to nrf_log_frontend.o(i.nrf_log_direct_feed) for nrf_log_direct_feed
    nrf_log_frontend.o(i.nrf_log_frontend_std_1) refers to nrf_log_frontend.o(i.nrf_log_direct_feed) for nrf_log_direct_feed
    nrf_log_frontend.o(i.nrf_log_frontend_std_2) refers to nrf_log_frontend.o(i.nrf_log_direct_feed) for nrf_log_direct_feed
    nrf_log_frontend.o(i.nrf_log_frontend_std_3) refers to nrf_log_frontend.o(i.nrf_log_direct_feed) for nrf_log_direct_feed
    nrf_log_frontend.o(i.nrf_log_frontend_std_4) refers to nrf_log_frontend.o(i.nrf_log_direct_feed) for nrf_log_direct_feed
    nrf_log_frontend.o(i.nrf_log_frontend_std_5) refers to nrf_log_frontend.o(i.nrf_log_direct_feed) for nrf_log_direct_feed
    nrf_log_frontend.o(i.nrf_log_frontend_std_6) refers to nrf_log_frontend.o(i.nrf_log_direct_feed) for nrf_log_direct_feed
    nrf_log_frontend.o(i.nrf_log_getchar) refers to nrf_log_backend_serial.o(i.nrf_log_backend_getchar) for nrf_log_backend_getchar
    nrf_log_frontend.o(i.nrf_log_handlers_set) refers to nrf_log_frontend.o(.bss) for .bss
    nrf_log_frontend.o(i.nrf_log_init) refers to nrf_log_backend_serial.o(i.nrf_log_backend_init) for nrf_log_backend_init
    nrf_log_frontend.o(i.nrf_log_init) refers to nrf_log_backend_serial.o(i.nrf_log_backend_hexdump_handler_get) for nrf_log_backend_hexdump_handler_get
    nrf_log_frontend.o(i.nrf_log_init) refers to nrf_log_backend_serial.o(i.nrf_log_backend_std_handler_get) for nrf_log_backend_std_handler_get
    nrf_log_frontend.o(i.nrf_log_init) refers to nrf_log_frontend.o(i.nrf_log_frontend_init) for nrf_log_frontend_init
    segger_rtt.o(i.SEGGER_RTT_ConfigDownBuffer) refers to segger_rtt.o(i._DoInit) for _DoInit
    segger_rtt.o(i.SEGGER_RTT_ConfigDownBuffer) refers to app_util_platform.o(i.app_util_critical_region_enter) for app_util_critical_region_enter
    segger_rtt.o(i.SEGGER_RTT_ConfigDownBuffer) refers to app_util_platform.o(i.app_util_critical_region_exit) for app_util_critical_region_exit
    segger_rtt.o(i.SEGGER_RTT_ConfigDownBuffer) refers to segger_rtt.o(.bss) for .bss
    segger_rtt.o(i.SEGGER_RTT_ConfigUpBuffer) refers to segger_rtt.o(i._DoInit) for _DoInit
    segger_rtt.o(i.SEGGER_RTT_ConfigUpBuffer) refers to app_util_platform.o(i.app_util_critical_region_enter) for app_util_critical_region_enter
    segger_rtt.o(i.SEGGER_RTT_ConfigUpBuffer) refers to app_util_platform.o(i.app_util_critical_region_exit) for app_util_critical_region_exit
    segger_rtt.o(i.SEGGER_RTT_ConfigUpBuffer) refers to segger_rtt.o(.bss) for .bss
    segger_rtt.o(i.SEGGER_RTT_GetKey) refers to segger_rtt.o(i.SEGGER_RTT_Read) for SEGGER_RTT_Read
    segger_rtt.o(i.SEGGER_RTT_HasData) refers to segger_rtt.o(.bss) for .bss
    segger_rtt.o(i.SEGGER_RTT_HasKey) refers to segger_rtt.o(i._DoInit) for _DoInit
    segger_rtt.o(i.SEGGER_RTT_HasKey) refers to segger_rtt.o(.bss) for .bss
    segger_rtt.o(i.SEGGER_RTT_Init) refers to segger_rtt.o(i._DoInit) for _DoInit
    segger_rtt.o(i.SEGGER_RTT_Init) refers to segger_rtt.o(.bss) for .bss
    segger_rtt.o(i.SEGGER_RTT_Read) refers to app_util_platform.o(i.app_util_critical_region_enter) for app_util_critical_region_enter
    segger_rtt.o(i.SEGGER_RTT_Read) refers to segger_rtt.o(i.SEGGER_RTT_ReadNoLock) for SEGGER_RTT_ReadNoLock
    segger_rtt.o(i.SEGGER_RTT_Read) refers to app_util_platform.o(i.app_util_critical_region_exit) for app_util_critical_region_exit
    segger_rtt.o(i.SEGGER_RTT_ReadNoLock) refers to segger_rtt.o(i._DoInit) for _DoInit
    segger_rtt.o(i.SEGGER_RTT_ReadNoLock) refers to memcpya.o(.text) for __aeabi_memcpy
    segger_rtt.o(i.SEGGER_RTT_ReadNoLock) refers to segger_rtt.o(.bss) for .bss
    segger_rtt.o(i.SEGGER_RTT_SetNameDownBuffer) refers to segger_rtt.o(i._DoInit) for _DoInit
    segger_rtt.o(i.SEGGER_RTT_SetNameDownBuffer) refers to app_util_platform.o(i.app_util_critical_region_enter) for app_util_critical_region_enter
    segger_rtt.o(i.SEGGER_RTT_SetNameDownBuffer) refers to app_util_platform.o(i.app_util_critical_region_exit) for app_util_critical_region_exit
    segger_rtt.o(i.SEGGER_RTT_SetNameDownBuffer) refers to segger_rtt.o(.bss) for .bss
    segger_rtt.o(i.SEGGER_RTT_SetNameUpBuffer) refers to segger_rtt.o(i._DoInit) for _DoInit
    segger_rtt.o(i.SEGGER_RTT_SetNameUpBuffer) refers to app_util_platform.o(i.app_util_critical_region_enter) for app_util_critical_region_enter
    segger_rtt.o(i.SEGGER_RTT_SetNameUpBuffer) refers to app_util_platform.o(i.app_util_critical_region_exit) for app_util_critical_region_exit
    segger_rtt.o(i.SEGGER_RTT_SetNameUpBuffer) refers to segger_rtt.o(.bss) for .bss
    segger_rtt.o(i.SEGGER_RTT_SetTerminal) refers to segger_rtt.o(i._DoInit) for _DoInit
    segger_rtt.o(i.SEGGER_RTT_SetTerminal) refers to app_util_platform.o(i.app_util_critical_region_enter) for app_util_critical_region_enter
    segger_rtt.o(i.SEGGER_RTT_SetTerminal) refers to segger_rtt.o(i._GetAvailWriteSpace) for _GetAvailWriteSpace
    segger_rtt.o(i.SEGGER_RTT_SetTerminal) refers to segger_rtt.o(i._WriteNoCheck) for _WriteNoCheck
    segger_rtt.o(i.SEGGER_RTT_SetTerminal) refers to segger_rtt.o(i._WriteBlocking) for _WriteBlocking
    segger_rtt.o(i.SEGGER_RTT_SetTerminal) refers to app_util_platform.o(i.app_util_critical_region_exit) for app_util_critical_region_exit
    segger_rtt.o(i.SEGGER_RTT_SetTerminal) refers to segger_rtt.o(.bss) for .bss
    segger_rtt.o(i.SEGGER_RTT_SetTerminal) refers to segger_rtt.o(.data) for .data
    segger_rtt.o(i.SEGGER_RTT_TerminalOut) refers to segger_rtt.o(i._DoInit) for _DoInit
    segger_rtt.o(i.SEGGER_RTT_TerminalOut) refers to strlen.o(.text) for strlen
    segger_rtt.o(i.SEGGER_RTT_TerminalOut) refers to app_util_platform.o(i.app_util_critical_region_enter) for app_util_critical_region_enter
    segger_rtt.o(i.SEGGER_RTT_TerminalOut) refers to segger_rtt.o(i._GetAvailWriteSpace) for _GetAvailWriteSpace
    segger_rtt.o(i.SEGGER_RTT_TerminalOut) refers to app_util_platform.o(i.app_util_critical_region_exit) for app_util_critical_region_exit
    segger_rtt.o(i.SEGGER_RTT_TerminalOut) refers to segger_rtt.o(i._PostTerminalSwitch) for _PostTerminalSwitch
    segger_rtt.o(i.SEGGER_RTT_TerminalOut) refers to segger_rtt.o(i._WriteBlocking) for _WriteBlocking
    segger_rtt.o(i.SEGGER_RTT_TerminalOut) refers to segger_rtt.o(.bss) for .bss
    segger_rtt.o(i.SEGGER_RTT_TerminalOut) refers to segger_rtt.o(.data) for .data
    segger_rtt.o(i.SEGGER_RTT_WaitKey) refers to segger_rtt.o(i.SEGGER_RTT_GetKey) for SEGGER_RTT_GetKey
    segger_rtt.o(i.SEGGER_RTT_Write) refers to segger_rtt.o(i._DoInit) for _DoInit
    segger_rtt.o(i.SEGGER_RTT_Write) refers to app_util_platform.o(i.app_util_critical_region_enter) for app_util_critical_region_enter
    segger_rtt.o(i.SEGGER_RTT_Write) refers to segger_rtt.o(i.SEGGER_RTT_WriteNoLock) for SEGGER_RTT_WriteNoLock
    segger_rtt.o(i.SEGGER_RTT_Write) refers to app_util_platform.o(i.app_util_critical_region_exit) for app_util_critical_region_exit
    segger_rtt.o(i.SEGGER_RTT_Write) refers to segger_rtt.o(.bss) for .bss
    segger_rtt.o(i.SEGGER_RTT_WriteNoLock) refers to segger_rtt.o(i._GetAvailWriteSpace) for _GetAvailWriteSpace
    segger_rtt.o(i.SEGGER_RTT_WriteNoLock) refers to segger_rtt.o(i._WriteNoCheck) for _WriteNoCheck
    segger_rtt.o(i.SEGGER_RTT_WriteNoLock) refers to segger_rtt.o(i._WriteBlocking) for _WriteBlocking
    segger_rtt.o(i.SEGGER_RTT_WriteNoLock) refers to segger_rtt.o(.bss) for .bss
    segger_rtt.o(i.SEGGER_RTT_WriteSkipNoLock) refers to memcpya.o(.text) for __aeabi_memcpy
    segger_rtt.o(i.SEGGER_RTT_WriteSkipNoLock) refers to segger_rtt.o(.bss) for .bss
    segger_rtt.o(i.SEGGER_RTT_WriteString) refers to strlen.o(.text) for strlen
    segger_rtt.o(i.SEGGER_RTT_WriteString) refers to segger_rtt.o(i.SEGGER_RTT_Write) for SEGGER_RTT_Write
    segger_rtt.o(i._DoInit) refers to strcpy.o(.text) for strcpy
    segger_rtt.o(i._DoInit) refers to segger_rtt.o(.bss) for .bss
    segger_rtt.o(i._PostTerminalSwitch) refers to segger_rtt.o(i._WriteBlocking) for _WriteBlocking
    segger_rtt.o(i._PostTerminalSwitch) refers to segger_rtt.o(.data) for .data
    segger_rtt.o(i._WriteBlocking) refers to memcpya.o(.text) for __aeabi_memcpy
    segger_rtt.o(i._WriteNoCheck) refers to memcpya.o(.text) for __aeabi_memcpy
    softdevice_handler.o(i.SWI2_EGU2_IRQHandler) refers to app_error.o(i.app_error_handler_bare) for app_error_handler_bare
    softdevice_handler.o(i.SWI2_EGU2_IRQHandler) refers to softdevice_handler.o(i.intern_softdevice_events_execute) for intern_softdevice_events_execute
    softdevice_handler.o(i.SWI2_EGU2_IRQHandler) refers to softdevice_handler.o(.data) for .data
    softdevice_handler.o(i.intern_softdevice_events_execute) refers to app_error.o(i.app_error_handler_bare) for app_error_handler_bare
    softdevice_handler.o(i.intern_softdevice_events_execute) refers to nrf_drv_clock.o(i.nrf_drv_clock_on_soc_event) for nrf_drv_clock_on_soc_event
    softdevice_handler.o(i.intern_softdevice_events_execute) refers to softdevice_handler.o(.data) for .data
    softdevice_handler.o(i.sd_nvic_EnableIRQ) refers to softdevice_handler.o(i.__sd_nvic_app_accessible_irq) for __sd_nvic_app_accessible_irq
    softdevice_handler.o(i.sd_nvic_EnableIRQ) refers to softdevice_handler.o(i.__NVIC_EnableIRQ) for __NVIC_EnableIRQ
    softdevice_handler.o(i.sd_nvic_EnableIRQ) refers to app_util_platform.o(.bss) for nrf_nvic_state
    softdevice_handler.o(i.softdevice_ble_evt_handler_set) refers to softdevice_handler.o(.data) for .data
    softdevice_handler.o(i.softdevice_enable) refers to nrf_log_frontend.o(i.nrf_log_frontend_std_1) for nrf_log_frontend_std_1
    softdevice_handler.o(i.softdevice_fault_handler) refers to app_error_weak.o(i.app_error_fault_handler) for app_error_fault_handler
    softdevice_handler.o(i.softdevice_handler_init) refers to softdevice_handler.o(i.__NVIC_DisableIRQ) for __NVIC_DisableIRQ
    softdevice_handler.o(i.softdevice_handler_init) refers to softdevice_handler.o(i.__NVIC_EnableIRQ) for __NVIC_EnableIRQ
    softdevice_handler.o(i.softdevice_handler_init) refers to nrf_drv_clock.o(i.nrf_drv_clock_on_sd_enable) for nrf_drv_clock_on_sd_enable
    softdevice_handler.o(i.softdevice_handler_init) refers to softdevice_handler.o(i.sd_nvic_EnableIRQ) for sd_nvic_EnableIRQ
    softdevice_handler.o(i.softdevice_handler_init) refers to softdevice_handler.o(.data) for .data
    softdevice_handler.o(i.softdevice_handler_init) refers to softdevice_handler.o(i.softdevice_fault_handler) for softdevice_fault_handler
    softdevice_handler.o(i.softdevice_handler_is_enabled) refers to softdevice_handler.o(.data) for .data
    softdevice_handler.o(i.softdevice_handler_is_suspended) refers to softdevice_handler.o(.data) for .data
    softdevice_handler.o(i.softdevice_handler_resume) refers to softdevice_handler.o(i.__sd_nvic_app_accessible_irq) for __sd_nvic_app_accessible_irq
    softdevice_handler.o(i.softdevice_handler_resume) refers to app_error.o(i.app_error_handler_bare) for app_error_handler_bare
    softdevice_handler.o(i.softdevice_handler_resume) refers to softdevice_handler.o(i.sd_nvic_EnableIRQ) for sd_nvic_EnableIRQ
    softdevice_handler.o(i.softdevice_handler_resume) refers to softdevice_handler.o(.data) for .data
    softdevice_handler.o(i.softdevice_handler_sd_disable) refers to nrf_drv_clock.o(i.nrf_drv_clock_on_sd_disable) for nrf_drv_clock_on_sd_disable
    softdevice_handler.o(i.softdevice_handler_sd_disable) refers to softdevice_handler.o(.data) for .data
    softdevice_handler.o(i.softdevice_handler_suspend) refers to softdevice_handler.o(i.__sd_nvic_app_accessible_irq) for __sd_nvic_app_accessible_irq
    softdevice_handler.o(i.softdevice_handler_suspend) refers to softdevice_handler.o(i.__NVIC_DisableIRQ) for __NVIC_DisableIRQ
    softdevice_handler.o(i.softdevice_handler_suspend) refers to app_error.o(i.app_error_handler_bare) for app_error_handler_bare
    softdevice_handler.o(i.softdevice_handler_suspend) refers to app_util_platform.o(.bss) for nrf_nvic_state
    softdevice_handler.o(i.softdevice_handler_suspend) refers to softdevice_handler.o(.data) for .data
    softdevice_handler.o(i.softdevice_sys_evt_handler_set) refers to softdevice_handler.o(.data) for .data
    arm_startup_nrf52.o(RESET) refers to arm_startup_nrf52.o(STACK) for __initial_sp
    arm_startup_nrf52.o(RESET) refers to arm_startup_nrf52.o(.text) for Reset_Handler
    arm_startup_nrf52.o(RESET) refers to nrf_drv_clock.o(i.POWER_CLOCK_IRQHandler) for POWER_CLOCK_IRQHandler
    arm_startup_nrf52.o(RESET) refers to nrf_drv_twi.o(i.SPIM0_SPIS0_TWIM0_TWIS0_SPI0_TWI0_IRQHandler) for SPIM0_SPIS0_TWIM0_TWIS0_SPI0_TWI0_IRQHandler
    arm_startup_nrf52.o(RESET) refers to nrf_drv_gpiote.o(i.GPIOTE_IRQHandler) for GPIOTE_IRQHandler
    arm_startup_nrf52.o(RESET) refers to app_timer.o(i.RTC1_IRQHandler) for RTC1_IRQHandler
    arm_startup_nrf52.o(RESET) refers to app_timer.o(i.SWI0_EGU0_IRQHandler) for SWI0_EGU0_IRQHandler
    arm_startup_nrf52.o(RESET) refers to softdevice_handler.o(i.SWI2_EGU2_IRQHandler) for SWI2_EGU2_IRQHandler
    arm_startup_nrf52.o(.text) refers to system_nrf52.o(i.SystemInit) for SystemInit
    arm_startup_nrf52.o(.text) refers to entry.o(.ARM.Collect$$$$00000000) for __main
    system_nrf52.o(i.SystemCoreClockUpdate) refers to system_nrf52.o(.data) for .data
    system_nrf52.o(i.SystemInit) refers to system_nrf52.o(i.errata_12) for errata_12
    system_nrf52.o(i.SystemInit) refers to system_nrf52.o(i.errata_16) for errata_16
    system_nrf52.o(i.SystemInit) refers to system_nrf52.o(i.errata_31) for errata_31
    system_nrf52.o(i.SystemInit) refers to system_nrf52.o(i.errata_32) for errata_32
    system_nrf52.o(i.SystemInit) refers to system_nrf52.o(i.errata_36) for errata_36
    system_nrf52.o(i.SystemInit) refers to system_nrf52.o(i.errata_37) for errata_37
    system_nrf52.o(i.SystemInit) refers to system_nrf52.o(i.errata_57) for errata_57
    system_nrf52.o(i.SystemInit) refers to system_nrf52.o(i.errata_66) for errata_66
    system_nrf52.o(i.SystemInit) refers to system_nrf52.o(i.errata_108) for errata_108
    system_nrf52.o(i.SystemInit) refers to system_nrf52.o(i.errata_136) for errata_136
    system_nrf52.o(i.SystemInit) refers to system_nrf52.o(i.errata_182) for errata_182
    system_nrf52.o(i.SystemInit) refers to system_nrf52.o(i.SystemCoreClockUpdate) for SystemCoreClockUpdate
    entry.o(.ARM.Collect$$$$00000000) refers (Special) to entry10a.o(.ARM.Collect$$$$0000000D) for __rt_final_cpp
    entry.o(.ARM.Collect$$$$00000000) refers (Special) to entry11a.o(.ARM.Collect$$$$0000000F) for __rt_final_exit
    entry.o(.ARM.Collect$$$$00000000) refers (Special) to entry7b.o(.ARM.Collect$$$$00000008) for _main_clock
    entry.o(.ARM.Collect$$$$00000000) refers (Special) to entry8b.o(.ARM.Collect$$$$0000000A) for _main_cpp_init
    entry.o(.ARM.Collect$$$$00000000) refers (Special) to entry9a.o(.ARM.Collect$$$$0000000B) for _main_init
    entry.o(.ARM.Collect$$$$00000000) refers (Special) to entry5.o(.ARM.Collect$$$$00000004) for _main_scatterload
    entry.o(.ARM.Collect$$$$00000000) refers (Special) to entry2.o(.ARM.Collect$$$$00000001) for _main_stk
    ctype_o.o(.text) refers to ctype_o.o(.constdata) for .constdata
    ctype_o.o(.constdata) refers to ctype_o.o(.constdata) for __ctype_table
    isalnum_o.o(.text) refers to ctype_o.o(.text) for __rt_ctype_table
    isalpha_o.o(.text) refers to ctype_o.o(.text) for __rt_ctype_table
    isblank_o.o(.text) refers to ctype_o.o(.constdata) for __ctype_table
    iscntrl_o.o(.text) refers to ctype_o.o(.text) for __rt_ctype_table
    isdigit_o.o(.text) refers to ctype_o.o(.text) for __rt_ctype_table
    isgraph_o.o(.text) refers to ctype_o.o(.text) for __rt_ctype_table
    islower_o.o(.text) refers to ctype_o.o(.text) for __rt_ctype_table
    isprint_o.o(.text) refers to ctype_o.o(.text) for __rt_ctype_table
    ispunct_o.o(.text) refers to ctype_o.o(.text) for __rt_ctype_table
    isspace_o.o(.text) refers to ctype_o.o(.text) for __rt_ctype_table
    isupper_o.o(.text) refers to ctype_o.o(.text) for __rt_ctype_table
    isxdigit_o.o(.text) refers to ctype_o.o(.text) for __rt_ctype_table
    printfb.o(i.__0fprintf$bare) refers to printfb.o(i._printf_core) for _printf_core
    printfb.o(i.__0fprintf$bare) refers to fputc.o(i.fputc) for fputc
    printfb.o(i.__0printf$bare) refers to printfb.o(i._printf_core) for _printf_core
    printfb.o(i.__0printf$bare) refers to fputc.o(i.fputc) for fputc
    printfb.o(i.__0printf$bare) refers to stdout.o(.data) for __stdout
    printfb.o(i.__0snprintf$bare) refers to printfb.o(i._printf_core) for _printf_core
    printfb.o(i.__0snprintf$bare) refers to printfb.o(i._snputc) for _snputc
    printfb.o(i.__0sprintf$bare) refers to printfb.o(i._printf_core) for _printf_core
    printfb.o(i.__0sprintf$bare) refers to printfb.o(i._sputc) for _sputc
    printfb.o(i.__0vfprintf$bare) refers to printfb.o(i._printf_core) for _printf_core
    printfb.o(i.__0vfprintf$bare) refers to fputc.o(i.fputc) for fputc
    printfb.o(i.__0vprintf$bare) refers to printfb.o(i._printf_core) for _printf_core
    printfb.o(i.__0vprintf$bare) refers to fputc.o(i.fputc) for fputc
    printfb.o(i.__0vprintf$bare) refers to stdout.o(.data) for __stdout
    printfb.o(i.__0vsnprintf$bare) refers to printfb.o(i._printf_core) for _printf_core
    printfb.o(i.__0vsnprintf$bare) refers to printfb.o(i._snputc) for _snputc
    printfb.o(i.__0vsprintf$bare) refers to printfb.o(i._printf_core) for _printf_core
    printfb.o(i.__0vsprintf$bare) refers to printfb.o(i._sputc) for _sputc
    printf0.o(i.__0fprintf$0) refers to printf0.o(i._printf_core) for _printf_core
    printf0.o(i.__0fprintf$0) refers to fputc.o(i.fputc) for fputc
    printf0.o(i.__0printf$0) refers to printf0.o(i._printf_core) for _printf_core
    printf0.o(i.__0printf$0) refers to fputc.o(i.fputc) for fputc
    printf0.o(i.__0printf$0) refers to stdout.o(.data) for __stdout
    printf0.o(i.__0snprintf$0) refers to printf0.o(i._printf_core) for _printf_core
    printf0.o(i.__0snprintf$0) refers to printf0.o(i._snputc) for _snputc
    printf0.o(i.__0sprintf$0) refers to printf0.o(i._printf_core) for _printf_core
    printf0.o(i.__0sprintf$0) refers to printf0.o(i._sputc) for _sputc
    printf0.o(i.__0vfprintf$0) refers to printf0.o(i._printf_core) for _printf_core
    printf0.o(i.__0vfprintf$0) refers to fputc.o(i.fputc) for fputc
    printf0.o(i.__0vprintf$0) refers to printf0.o(i._printf_core) for _printf_core
    printf0.o(i.__0vprintf$0) refers to fputc.o(i.fputc) for fputc
    printf0.o(i.__0vprintf$0) refers to stdout.o(.data) for __stdout
    printf0.o(i.__0vsnprintf$0) refers to printf0.o(i._printf_core) for _printf_core
    printf0.o(i.__0vsnprintf$0) refers to printf0.o(i._snputc) for _snputc
    printf0.o(i.__0vsprintf$0) refers to printf0.o(i._printf_core) for _printf_core
    printf0.o(i.__0vsprintf$0) refers to printf0.o(i._sputc) for _sputc
    printf1.o(i.__0fprintf$1) refers to printf1.o(i._printf_core) for _printf_core
    printf1.o(i.__0fprintf$1) refers to fputc.o(i.fputc) for fputc
    printf1.o(i.__0printf$1) refers to printf1.o(i._printf_core) for _printf_core
    printf1.o(i.__0printf$1) refers to fputc.o(i.fputc) for fputc
    printf1.o(i.__0printf$1) refers to stdout.o(.data) for __stdout
    printf1.o(i.__0snprintf$1) refers to printf1.o(i._printf_core) for _printf_core
    printf1.o(i.__0snprintf$1) refers to printf1.o(i._snputc) for _snputc
    printf1.o(i.__0sprintf$1) refers to printf1.o(i._printf_core) for _printf_core
    printf1.o(i.__0sprintf$1) refers to printf1.o(i._sputc) for _sputc
    printf1.o(i.__0vfprintf$1) refers to printf1.o(i._printf_core) for _printf_core
    printf1.o(i.__0vfprintf$1) refers to fputc.o(i.fputc) for fputc
    printf1.o(i.__0vprintf$1) refers to printf1.o(i._printf_core) for _printf_core
    printf1.o(i.__0vprintf$1) refers to fputc.o(i.fputc) for fputc
    printf1.o(i.__0vprintf$1) refers to stdout.o(.data) for __stdout
    printf1.o(i.__0vsnprintf$1) refers to printf1.o(i._printf_core) for _printf_core
    printf1.o(i.__0vsnprintf$1) refers to printf1.o(i._snputc) for _snputc
    printf1.o(i.__0vsprintf$1) refers to printf1.o(i._printf_core) for _printf_core
    printf1.o(i.__0vsprintf$1) refers to printf1.o(i._sputc) for _sputc
    printf1.o(i._printf_core) refers to uidiv.o(.text) for __aeabi_uidivmod
    printf2.o(i.__0fprintf$2) refers to printf2.o(i._printf_core) for _printf_core
    printf2.o(i.__0fprintf$2) refers to fputc.o(i.fputc) for fputc
    printf2.o(i.__0printf$2) refers to printf2.o(i._printf_core) for _printf_core
    printf2.o(i.__0printf$2) refers to fputc.o(i.fputc) for fputc
    printf2.o(i.__0printf$2) refers to stdout.o(.data) for __stdout
    printf2.o(i.__0snprintf$2) refers to printf2.o(i._printf_core) for _printf_core
    printf2.o(i.__0snprintf$2) refers to printf2.o(i._snputc) for _snputc
    printf2.o(i.__0sprintf$2) refers to printf2.o(i._printf_core) for _printf_core
    printf2.o(i.__0sprintf$2) refers to printf2.o(i._sputc) for _sputc
    printf2.o(i.__0vfprintf$2) refers to printf2.o(i._printf_core) for _printf_core
    printf2.o(i.__0vfprintf$2) refers to fputc.o(i.fputc) for fputc
    printf2.o(i.__0vprintf$2) refers to printf2.o(i._printf_core) for _printf_core
    printf2.o(i.__0vprintf$2) refers to fputc.o(i.fputc) for fputc
    printf2.o(i.__0vprintf$2) refers to stdout.o(.data) for __stdout
    printf2.o(i.__0vsnprintf$2) refers to printf2.o(i._printf_core) for _printf_core
    printf2.o(i.__0vsnprintf$2) refers to printf2.o(i._snputc) for _snputc
    printf2.o(i.__0vsprintf$2) refers to printf2.o(i._printf_core) for _printf_core
    printf2.o(i.__0vsprintf$2) refers to printf2.o(i._sputc) for _sputc
    printf3.o(i.__0fprintf$3) refers to printf3.o(i._printf_core) for _printf_core
    printf3.o(i.__0fprintf$3) refers to fputc.o(i.fputc) for fputc
    printf3.o(i.__0printf$3) refers to printf3.o(i._printf_core) for _printf_core
    printf3.o(i.__0printf$3) refers to fputc.o(i.fputc) for fputc
    printf3.o(i.__0printf$3) refers to stdout.o(.data) for __stdout
    printf3.o(i.__0snprintf$3) refers to printf3.o(i._printf_core) for _printf_core
    printf3.o(i.__0snprintf$3) refers to printf3.o(i._snputc) for _snputc
    printf3.o(i.__0sprintf$3) refers to printf3.o(i._printf_core) for _printf_core
    printf3.o(i.__0sprintf$3) refers to printf3.o(i._sputc) for _sputc
    printf3.o(i.__0vfprintf$3) refers to printf3.o(i._printf_core) for _printf_core
    printf3.o(i.__0vfprintf$3) refers to fputc.o(i.fputc) for fputc
    printf3.o(i.__0vprintf$3) refers to printf3.o(i._printf_core) for _printf_core
    printf3.o(i.__0vprintf$3) refers to fputc.o(i.fputc) for fputc
    printf3.o(i.__0vprintf$3) refers to stdout.o(.data) for __stdout
    printf3.o(i.__0vsnprintf$3) refers to printf3.o(i._printf_core) for _printf_core
    printf3.o(i.__0vsnprintf$3) refers to printf3.o(i._snputc) for _snputc
    printf3.o(i.__0vsprintf$3) refers to printf3.o(i._printf_core) for _printf_core
    printf3.o(i.__0vsprintf$3) refers to printf3.o(i._sputc) for _sputc
    printf3.o(i._printf_core) refers to uidiv.o(.text) for __aeabi_uidivmod
    printf4.o(i.__0fprintf$4) refers to printf4.o(i._printf_core) for _printf_core
    printf4.o(i.__0fprintf$4) refers to fputc.o(i.fputc) for fputc
    printf4.o(i.__0printf$4) refers to printf4.o(i._printf_core) for _printf_core
    printf4.o(i.__0printf$4) refers to fputc.o(i.fputc) for fputc
    printf4.o(i.__0printf$4) refers to stdout.o(.data) for __stdout
    printf4.o(i.__0snprintf$4) refers to printf4.o(i._printf_core) for _printf_core
    printf4.o(i.__0snprintf$4) refers to printf4.o(i._snputc) for _snputc
    printf4.o(i.__0sprintf$4) refers to printf4.o(i._printf_core) for _printf_core
    printf4.o(i.__0sprintf$4) refers to printf4.o(i._sputc) for _sputc
    printf4.o(i.__0vfprintf$4) refers to printf4.o(i._printf_core) for _printf_core
    printf4.o(i.__0vfprintf$4) refers to fputc.o(i.fputc) for fputc
    printf4.o(i.__0vprintf$4) refers to printf4.o(i._printf_core) for _printf_core
    printf4.o(i.__0vprintf$4) refers to fputc.o(i.fputc) for fputc
    printf4.o(i.__0vprintf$4) refers to stdout.o(.data) for __stdout
    printf4.o(i.__0vsnprintf$4) refers to printf4.o(i._printf_core) for _printf_core
    printf4.o(i.__0vsnprintf$4) refers to printf4.o(i._snputc) for _snputc
    printf4.o(i.__0vsprintf$4) refers to printf4.o(i._printf_core) for _printf_core
    printf4.o(i.__0vsprintf$4) refers to printf4.o(i._sputc) for _sputc
    printf4.o(i._printf_core) refers to uldiv.o(.text) for __aeabi_uldivmod
    printf5.o(i.__0fprintf$5) refers to printf5.o(i._printf_core) for _printf_core
    printf5.o(i.__0fprintf$5) refers to fputc.o(i.fputc) for fputc
    printf5.o(i.__0printf$5) refers to printf5.o(i._printf_core) for _printf_core
    printf5.o(i.__0printf$5) refers to fputc.o(i.fputc) for fputc
    printf5.o(i.__0printf$5) refers to stdout.o(.data) for __stdout
    printf5.o(i.__0snprintf$5) refers to printf5.o(i._printf_core) for _printf_core
    printf5.o(i.__0snprintf$5) refers to printf5.o(i._snputc) for _snputc
    printf5.o(i.__0sprintf$5) refers to printf5.o(i._printf_core) for _printf_core
    printf5.o(i.__0sprintf$5) refers to printf5.o(i._sputc) for _sputc
    printf5.o(i.__0vfprintf$5) refers to printf5.o(i._printf_core) for _printf_core
    printf5.o(i.__0vfprintf$5) refers to fputc.o(i.fputc) for fputc
    printf5.o(i.__0vprintf$5) refers to printf5.o(i._printf_core) for _printf_core
    printf5.o(i.__0vprintf$5) refers to fputc.o(i.fputc) for fputc
    printf5.o(i.__0vprintf$5) refers to stdout.o(.data) for __stdout
    printf5.o(i.__0vsnprintf$5) refers to printf5.o(i._printf_core) for _printf_core
    printf5.o(i.__0vsnprintf$5) refers to printf5.o(i._snputc) for _snputc
    printf5.o(i.__0vsprintf$5) refers to printf5.o(i._printf_core) for _printf_core
    printf5.o(i.__0vsprintf$5) refers to printf5.o(i._sputc) for _sputc
    printf5.o(i._printf_core) refers to uldiv.o(.text) for __aeabi_uldivmod
    printf6.o(i.__0fprintf$6) refers to printf6.o(i._printf_core) for _printf_core
    printf6.o(i.__0fprintf$6) refers to fputc.o(i.fputc) for fputc
    printf6.o(i.__0printf$6) refers to printf6.o(i._printf_core) for _printf_core
    printf6.o(i.__0printf$6) refers to fputc.o(i.fputc) for fputc
    printf6.o(i.__0printf$6) refers to stdout.o(.data) for __stdout
    printf6.o(i.__0snprintf$6) refers to printf6.o(i._printf_core) for _printf_core
    printf6.o(i.__0snprintf$6) refers to printf6.o(i._snputc) for _snputc
    printf6.o(i.__0sprintf$6) refers to printf6.o(i._printf_core) for _printf_core
    printf6.o(i.__0sprintf$6) refers to printf6.o(i._sputc) for _sputc
    printf6.o(i.__0vfprintf$6) refers to printf6.o(i._printf_core) for _printf_core
    printf6.o(i.__0vfprintf$6) refers to fputc.o(i.fputc) for fputc
    printf6.o(i.__0vprintf$6) refers to printf6.o(i._printf_core) for _printf_core
    printf6.o(i.__0vprintf$6) refers to fputc.o(i.fputc) for fputc
    printf6.o(i.__0vprintf$6) refers to stdout.o(.data) for __stdout
    printf6.o(i.__0vsnprintf$6) refers to printf6.o(i._printf_core) for _printf_core
    printf6.o(i.__0vsnprintf$6) refers to printf6.o(i._snputc) for _snputc
    printf6.o(i.__0vsprintf$6) refers to printf6.o(i._printf_core) for _printf_core
    printf6.o(i.__0vsprintf$6) refers to printf6.o(i._sputc) for _sputc
    printf6.o(i._printf_core) refers to printf6.o(i._printf_pre_padding) for _printf_pre_padding
    printf6.o(i._printf_core) refers to uidiv.o(.text) for __aeabi_uidivmod
    printf6.o(i._printf_core) refers to printf6.o(i._printf_post_padding) for _printf_post_padding
    printf7.o(i.__0fprintf$7) refers to printf7.o(i._printf_core) for _printf_core
    printf7.o(i.__0fprintf$7) refers to fputc.o(i.fputc) for fputc
    printf7.o(i.__0printf$7) refers to printf7.o(i._printf_core) for _printf_core
    printf7.o(i.__0printf$7) refers to fputc.o(i.fputc) for fputc
    printf7.o(i.__0printf$7) refers to stdout.o(.data) for __stdout
    printf7.o(i.__0snprintf$7) refers to printf7.o(i._printf_core) for _printf_core
    printf7.o(i.__0snprintf$7) refers to printf7.o(i._snputc) for _snputc
    printf7.o(i.__0sprintf$7) refers to printf7.o(i._printf_core) for _printf_core
    printf7.o(i.__0sprintf$7) refers to printf7.o(i._sputc) for _sputc
    printf7.o(i.__0vfprintf$7) refers to printf7.o(i._printf_core) for _printf_core
    printf7.o(i.__0vfprintf$7) refers to fputc.o(i.fputc) for fputc
    printf7.o(i.__0vprintf$7) refers to printf7.o(i._printf_core) for _printf_core
    printf7.o(i.__0vprintf$7) refers to fputc.o(i.fputc) for fputc
    printf7.o(i.__0vprintf$7) refers to stdout.o(.data) for __stdout
    printf7.o(i.__0vsnprintf$7) refers to printf7.o(i._printf_core) for _printf_core
    printf7.o(i.__0vsnprintf$7) refers to printf7.o(i._snputc) for _snputc
    printf7.o(i.__0vsprintf$7) refers to printf7.o(i._printf_core) for _printf_core
    printf7.o(i.__0vsprintf$7) refers to printf7.o(i._sputc) for _sputc
    printf7.o(i._printf_core) refers to printf7.o(i._printf_pre_padding) for _printf_pre_padding
    printf7.o(i._printf_core) refers to uldiv.o(.text) for __aeabi_uldivmod
    printf7.o(i._printf_core) refers to printf7.o(i._printf_post_padding) for _printf_post_padding
    printf8.o(i.__0fprintf$8) refers to printf8.o(i._printf_core) for _printf_core
    printf8.o(i.__0fprintf$8) refers to fputc.o(i.fputc) for fputc
    printf8.o(i.__0printf$8) refers to printf8.o(i._printf_core) for _printf_core
    printf8.o(i.__0printf$8) refers to fputc.o(i.fputc) for fputc
    printf8.o(i.__0printf$8) refers to stdout.o(.data) for __stdout
    printf8.o(i.__0snprintf$8) refers to printf8.o(i._printf_core) for _printf_core
    printf8.o(i.__0snprintf$8) refers to printf8.o(i._snputc) for _snputc
    printf8.o(i.__0sprintf$8) refers to printf8.o(i._printf_core) for _printf_core
    printf8.o(i.__0sprintf$8) refers to printf8.o(i._sputc) for _sputc
    printf8.o(i.__0vfprintf$8) refers to printf8.o(i._printf_core) for _printf_core
    printf8.o(i.__0vfprintf$8) refers to fputc.o(i.fputc) for fputc
    printf8.o(i.__0vprintf$8) refers to printf8.o(i._printf_core) for _printf_core
    printf8.o(i.__0vprintf$8) refers to fputc.o(i.fputc) for fputc
    printf8.o(i.__0vprintf$8) refers to stdout.o(.data) for __stdout
    printf8.o(i.__0vsnprintf$8) refers to printf8.o(i._printf_core) for _printf_core
    printf8.o(i.__0vsnprintf$8) refers to printf8.o(i._snputc) for _snputc
    printf8.o(i.__0vsprintf$8) refers to printf8.o(i._printf_core) for _printf_core
    printf8.o(i.__0vsprintf$8) refers to printf8.o(i._sputc) for _sputc
    printf8.o(i._printf_core) refers to printf8.o(i._printf_pre_padding) for _printf_pre_padding
    printf8.o(i._printf_core) refers to uldiv.o(.text) for __aeabi_uldivmod
    printf8.o(i._printf_core) refers to printf8.o(i._printf_post_padding) for _printf_post_padding
    printfa.o(i.__0fprintf) refers (Special) to iusefp.o(.text) for __I$use$fp
    printfa.o(i.__0fprintf) refers to printfa.o(i._printf_core) for _printf_core
    printfa.o(i.__0fprintf) refers to fputc.o(i.fputc) for fputc
    printfa.o(i.__0printf) refers (Special) to iusefp.o(.text) for __I$use$fp
    printfa.o(i.__0printf) refers to printfa.o(i._printf_core) for _printf_core
    printfa.o(i.__0printf) refers to fputc.o(i.fputc) for fputc
    printfa.o(i.__0printf) refers to stdout.o(.data) for __stdout
    printfa.o(i.__0snprintf) refers (Special) to iusefp.o(.text) for __I$use$fp
    printfa.o(i.__0snprintf) refers to printfa.o(i._printf_core) for _printf_core
    printfa.o(i.__0snprintf) refers to printfa.o(i._snputc) for _snputc
    printfa.o(i.__0sprintf) refers (Special) to iusefp.o(.text) for __I$use$fp
    printfa.o(i.__0sprintf) refers to printfa.o(i._printf_core) for _printf_core
    printfa.o(i.__0sprintf) refers to printfa.o(i._sputc) for _sputc
    printfa.o(i.__0vfprintf) refers (Special) to iusefp.o(.text) for __I$use$fp
    printfa.o(i.__0vfprintf) refers to printfa.o(i._printf_core) for _printf_core
    printfa.o(i.__0vfprintf) refers to fputc.o(i.fputc) for fputc
    printfa.o(i.__0vprintf) refers (Special) to iusefp.o(.text) for __I$use$fp
    printfa.o(i.__0vprintf) refers to printfa.o(i._printf_core) for _printf_core
    printfa.o(i.__0vprintf) refers to fputc.o(i.fputc) for fputc
    printfa.o(i.__0vprintf) refers to stdout.o(.data) for __stdout
    printfa.o(i.__0vsnprintf) refers (Special) to iusefp.o(.text) for __I$use$fp
    printfa.o(i.__0vsnprintf) refers to printfa.o(i._printf_core) for _printf_core
    printfa.o(i.__0vsnprintf) refers to printfa.o(i._snputc) for _snputc
    printfa.o(i.__0vsprintf) refers (Special) to iusefp.o(.text) for __I$use$fp
    printfa.o(i.__0vsprintf) refers to printfa.o(i._printf_core) for _printf_core
    printfa.o(i.__0vsprintf) refers to printfa.o(i._sputc) for _sputc
    printfa.o(i._fp_digits) refers (Special) to iusefp.o(.text) for __I$use$fp
    printfa.o(i._fp_digits) refers to dmul.o(.text) for __aeabi_dmul
    printfa.o(i._fp_digits) refers to ddiv.o(.text) for __aeabi_ddiv
    printfa.o(i._fp_digits) refers to cdrcmple.o(.text) for __aeabi_cdrcmple
    printfa.o(i._fp_digits) refers to dadd.o(.text) for __aeabi_dadd
    printfa.o(i._fp_digits) refers to dfixul.o(.text) for __aeabi_d2ulz
    printfa.o(i._fp_digits) refers to uldiv.o(.text) for __aeabi_uldivmod
    printfa.o(i._printf_core) refers (Special) to iusefp.o(.text) for __I$use$fp
    printfa.o(i._printf_core) refers to printfa.o(i._printf_pre_padding) for _printf_pre_padding
    printfa.o(i._printf_core) refers to uldiv.o(.text) for __aeabi_uldivmod
    printfa.o(i._printf_core) refers to printfa.o(i._printf_post_padding) for _printf_post_padding
    printfa.o(i._printf_core) refers to printfa.o(i._fp_digits) for _fp_digits
    printfa.o(i._printf_core) refers to uidiv.o(.text) for __aeabi_uidivmod
    printfa.o(i._printf_post_padding) refers (Special) to iusefp.o(.text) for __I$use$fp
    printfa.o(i._printf_pre_padding) refers (Special) to iusefp.o(.text) for __I$use$fp
    printfa.o(i._snputc) refers (Special) to iusefp.o(.text) for __I$use$fp
    printfa.o(i._sputc) refers (Special) to iusefp.o(.text) for __I$use$fp
    entry2.o(.ARM.Collect$$$$00000001) refers to entry2.o(.ARM.Collect$$$$00002712) for __lit__00000000
    entry2.o(.ARM.Collect$$$$00002712) refers to arm_startup_nrf52.o(STACK) for __initial_sp
    entry2.o(__vectab_stack_and_reset_area) refers to arm_startup_nrf52.o(STACK) for __initial_sp
    entry2.o(__vectab_stack_and_reset_area) refers to entry.o(.ARM.Collect$$$$00000000) for __main
    entry5.o(.ARM.Collect$$$$00000004) refers to init.o(.text) for __scatterload
    entry9a.o(.ARM.Collect$$$$0000000B) refers to main.o(i.main) for main
    entry9b.o(.ARM.Collect$$$$0000000C) refers to main.o(i.main) for main
    fputc.o(i.fputc) refers (Special) to iusesemip.o(.text) for __I$use$semihosting$fputc
    fputc.o(i.fputc) refers (Special) to semi.o(.text) for __semihosting_library_function
    uldiv.o(.text) refers to llushr.o(.text) for __aeabi_llsr
    uldiv.o(.text) refers to llshl.o(.text) for __aeabi_llsl
    dadd.o(.text) refers to llshl.o(.text) for __aeabi_llsl
    dadd.o(.text) refers to llsshr.o(.text) for __aeabi_lasr
    dadd.o(.text) refers to depilogue.o(.text) for _double_epilogue
    dmul.o(.text) refers to depilogue.o(.text) for _double_epilogue
    ddiv.o(.text) refers to depilogue.o(.text) for _double_round
    dfixul.o(.text) refers to llushr.o(.text) for __aeabi_llsr
    dfixul.o(.text) refers to llshl.o(.text) for __aeabi_llsl
    init.o(.text) refers to entry5.o(.ARM.Collect$$$$00000004) for __main_after_scatterload
    depilogue.o(.text) refers to llshl.o(.text) for __aeabi_llsl
    depilogue.o(.text) refers to llushr.o(.text) for __aeabi_llsr


==============================================================================

Removing Unused input sections from the image.

    Removing main.o(.rev16_text), (4 bytes).
    Removing main.o(.revsh_text), (4 bytes).
    Removing main.o(.rrx_text), (6 bytes).
    Removing main.o(i.assert_nrf_callback), (16 bytes).
    Removing twi_slave_tiny_unwrap.o(.rev16_text), (4 bytes).
    Removing twi_slave_tiny_unwrap.o(.revsh_text), (4 bytes).
    Removing twi_slave_tiny_unwrap.o(.rrx_text), (6 bytes).
    Removing boards.o(.rev16_text), (4 bytes).
    Removing boards.o(.revsh_text), (4 bytes).
    Removing boards.o(.rrx_text), (6 bytes).
    Removing boards.o(i.bsp_board_button_idx_to_pin), (12 bytes).
    Removing boards.o(i.bsp_board_button_state_get), (36 bytes).
    Removing boards.o(i.bsp_board_buttons_init), (36 bytes).
    Removing boards.o(i.bsp_board_led_idx_to_pin), (12 bytes).
    Removing boards.o(i.bsp_board_led_invert), (36 bytes).
    Removing boards.o(i.bsp_board_led_off), (16 bytes).
    Removing boards.o(i.bsp_board_led_on), (16 bytes).
    Removing boards.o(i.bsp_board_led_state_get), (36 bytes).
    Removing boards.o(i.bsp_board_leds_init), (44 bytes).
    Removing boards.o(i.bsp_board_leds_off), (18 bytes).
    Removing boards.o(i.bsp_board_leds_on), (18 bytes).
    Removing boards.o(i.bsp_board_pin_to_button_idx), (36 bytes).
    Removing boards.o(i.bsp_board_pin_to_led_idx), (36 bytes).
    Removing boards.o(i.nrf_gpio_cfg), (36 bytes).
    Removing boards.o(i.nrf_gpio_pin_write), (24 bytes).
    Removing boards.o(.constdata), (8 bytes).
    Removing bsp.o(.rev16_text), (4 bytes).
    Removing bsp.o(.revsh_text), (4 bytes).
    Removing bsp.o(.rrx_text), (6 bytes).
    Removing bsp.o(i.bsp_button_is_pressed), (4 bytes).
    Removing bsp.o(i.bsp_buttons_disable), (4 bytes).
    Removing bsp.o(i.bsp_buttons_enable), (4 bytes).
    Removing bsp.o(i.bsp_init), (16 bytes).
    Removing bsp.o(i.bsp_wakeup_button_disable), (4 bytes).
    Removing bsp.o(i.bsp_wakeup_button_enable), (4 bytes).
    Removing bsp_nfc.o(.rev16_text), (4 bytes).
    Removing bsp_nfc.o(.revsh_text), (4 bytes).
    Removing bsp_nfc.o(.rrx_text), (6 bytes).
    Removing ble_advdata.o(.rev16_text), (4 bytes).
    Removing ble_advdata.o(.revsh_text), (4 bytes).
    Removing ble_advdata.o(.rrx_text), (6 bytes).
    Removing ble_conn_params.o(.rev16_text), (4 bytes).
    Removing ble_conn_params.o(.revsh_text), (4 bytes).
    Removing ble_conn_params.o(.rrx_text), (6 bytes).
    Removing ble_conn_params.o(i.ble_conn_params_change_conn_params), (76 bytes).
    Removing ble_conn_params.o(i.ble_conn_params_init), (92 bytes).
    Removing ble_conn_params.o(i.ble_conn_params_on_ble_evt), (36 bytes).
    Removing ble_conn_params.o(i.ble_conn_params_stop), (12 bytes).
    Removing ble_conn_params.o(i.conn_params_negotiation), (100 bytes).
    Removing ble_conn_params.o(i.is_conn_params_ok), (28 bytes).
    Removing ble_conn_params.o(i.on_conn_params_update), (20 bytes).
    Removing ble_conn_params.o(i.on_connect), (40 bytes).
    Removing ble_conn_params.o(i.on_disconnect), (56 bytes).
    Removing ble_conn_params.o(i.on_write), (72 bytes).
    Removing ble_conn_params.o(i.update_timeout_handler), (96 bytes).
    Removing ble_conn_params.o(.bss), (32 bytes).
    Removing ble_conn_params.o(.bss), (28 bytes).
    Removing ble_conn_params.o(.constdata), (4 bytes).
    Removing ble_conn_params.o(.data), (20 bytes).
    Removing ble_srv_common.o(.rev16_text), (4 bytes).
    Removing ble_srv_common.o(.revsh_text), (4 bytes).
    Removing ble_srv_common.o(.rrx_text), (6 bytes).
    Removing ble_srv_common.o(i.ble_srv_ascii_to_utf8), (18 bytes).
    Removing ble_srv_common.o(i.ble_srv_is_indication_enabled), (14 bytes).
    Removing ble_srv_common.o(i.ble_srv_is_notification_enabled), (14 bytes).
    Removing ble_srv_common.o(i.ble_srv_report_ref_encode), (14 bytes).
    Removing ble_srv_common.o(i.characteristic_add), (424 bytes).
    Removing ble_srv_common.o(i.descriptor_add), (178 bytes).
    Removing ble_srv_common.o(i.set_security_req), (118 bytes).
    Removing nrf_drv_clock.o(.rev16_text), (4 bytes).
    Removing nrf_drv_clock.o(.revsh_text), (4 bytes).
    Removing nrf_drv_clock.o(.rrx_text), (6 bytes).
    Removing nrf_drv_clock.o(i.hfclk_start), (32 bytes).
    Removing nrf_drv_clock.o(i.hfclk_stop), (44 bytes).
    Removing nrf_drv_clock.o(i.item_enqueue), (26 bytes).
    Removing nrf_drv_clock.o(i.lfclk_start), (32 bytes).
    Removing nrf_drv_clock.o(i.lfclk_stop), (40 bytes).
    Removing nrf_drv_clock.o(i.nrf_clock_hf_is_running), (28 bytes).
    Removing nrf_drv_clock.o(i.nrf_drv_clock_calibration_abort), (4 bytes).
    Removing nrf_drv_clock.o(i.nrf_drv_clock_calibration_start), (4 bytes).
    Removing nrf_drv_clock.o(i.nrf_drv_clock_hfclk_is_running), (32 bytes).
    Removing nrf_drv_clock.o(i.nrf_drv_clock_hfclk_release), (44 bytes).
    Removing nrf_drv_clock.o(i.nrf_drv_clock_hfclk_request), (96 bytes).
    Removing nrf_drv_clock.o(i.nrf_drv_clock_init_check), (12 bytes).
    Removing nrf_drv_clock.o(i.nrf_drv_clock_is_calibrating), (4 bytes).
    Removing nrf_drv_clock.o(i.nrf_drv_clock_lfclk_is_running), (28 bytes).
    Removing nrf_drv_clock.o(i.nrf_drv_clock_lfclk_release), (44 bytes).
    Removing nrf_drv_clock.o(i.nrf_drv_clock_lfclk_request), (96 bytes).
    Removing nrf_drv_clock.o(i.nrf_drv_clock_on_sd_disable), (18 bytes).
    Removing nrf_drv_clock.o(i.nrf_drv_clock_uninit), (40 bytes).
    Removing nrf_drv_clock.o(.constdata), (19 bytes).
    Removing nrf_drv_clock.o(.constdata), (32 bytes).
    Removing nrf_drv_clock.o(.constdata), (32 bytes).
    Removing nrf_drv_clock.o(.constdata), (29 bytes).
    Removing nrf_drv_common.o(.rev16_text), (4 bytes).
    Removing nrf_drv_common.o(.revsh_text), (4 bytes).
    Removing nrf_drv_common.o(.rrx_text), (6 bytes).
    Removing nrf_drv_common.o(i.nrf_drv_common_clock_irq_disable), (20 bytes).
    Removing nrf_drv_gpiote.o(.rev16_text), (4 bytes).
    Removing nrf_drv_gpiote.o(.revsh_text), (4 bytes).
    Removing nrf_drv_gpiote.o(.rrx_text), (6 bytes).
    Removing nrf_drv_gpiote.o(i.channel_free), (28 bytes).
    Removing nrf_drv_gpiote.o(i.channel_port_alloc), (84 bytes).
    Removing nrf_drv_gpiote.o(i.nrf_drv_gpiote_clr_task_addr_get), (24 bytes).
    Removing nrf_drv_gpiote.o(i.nrf_drv_gpiote_clr_task_trigger), (28 bytes).
    Removing nrf_drv_gpiote.o(i.nrf_drv_gpiote_in_event_addr_get), (44 bytes).
    Removing nrf_drv_gpiote.o(i.nrf_drv_gpiote_in_event_disable), (72 bytes).
    Removing nrf_drv_gpiote.o(i.nrf_drv_gpiote_in_event_enable), (176 bytes).
    Removing nrf_drv_gpiote.o(i.nrf_drv_gpiote_in_init), (180 bytes).
    Removing nrf_drv_gpiote.o(i.nrf_drv_gpiote_in_is_set), (24 bytes).
    Removing nrf_drv_gpiote.o(i.nrf_drv_gpiote_in_uninit), (76 bytes).
    Removing nrf_drv_gpiote.o(i.nrf_drv_gpiote_init), (92 bytes).
    Removing nrf_drv_gpiote.o(i.nrf_drv_gpiote_is_init), (20 bytes).
    Removing nrf_drv_gpiote.o(i.nrf_drv_gpiote_out_clear), (16 bytes).
    Removing nrf_drv_gpiote.o(i.nrf_drv_gpiote_out_init), (180 bytes).
    Removing nrf_drv_gpiote.o(i.nrf_drv_gpiote_out_set), (16 bytes).
    Removing nrf_drv_gpiote.o(i.nrf_drv_gpiote_out_task_addr_get), (20 bytes).
    Removing nrf_drv_gpiote.o(i.nrf_drv_gpiote_out_task_disable), (36 bytes).
    Removing nrf_drv_gpiote.o(i.nrf_drv_gpiote_out_task_enable), (36 bytes).
    Removing nrf_drv_gpiote.o(i.nrf_drv_gpiote_out_task_force), (48 bytes).
    Removing nrf_drv_gpiote.o(i.nrf_drv_gpiote_out_task_trigger), (24 bytes).
    Removing nrf_drv_gpiote.o(i.nrf_drv_gpiote_out_toggle), (26 bytes).
    Removing nrf_drv_gpiote.o(i.nrf_drv_gpiote_out_uninit), (72 bytes).
    Removing nrf_drv_gpiote.o(i.nrf_drv_gpiote_set_task_addr_get), (24 bytes).
    Removing nrf_drv_gpiote.o(i.nrf_drv_gpiote_set_task_trigger), (28 bytes).
    Removing nrf_drv_gpiote.o(i.nrf_drv_gpiote_uninit), (64 bytes).
    Removing nrf_drv_gpiote.o(i.nrf_gpio_cfg), (36 bytes).
    Removing nrf_drv_gpiote.o(i.nrf_gpio_cfg_default), (18 bytes).
    Removing nrf_drv_gpiote.o(i.pin_in_use_by_port), (24 bytes).
    Removing nrf_drv_gpiote.o(i.pin_in_use_by_te), (24 bytes).
    Removing nrf_drv_gpiote.o(.constdata), (20 bytes).
    Removing nrf_drv_gpiote.o(.constdata), (24 bytes).
    Removing nrf_drv_gpiote.o(.constdata), (23 bytes).
    Removing nrf_drv_uart.o(.rev16_text), (4 bytes).
    Removing nrf_drv_uart.o(.revsh_text), (4 bytes).
    Removing nrf_drv_uart.o(.rrx_text), (6 bytes).
    Removing nrf_drv_twi.o(.rev16_text), (4 bytes).
    Removing nrf_drv_twi.o(.revsh_text), (4 bytes).
    Removing nrf_drv_twi.o(.rrx_text), (6 bytes).
    Removing nrf_drv_twi.o(i.nrf_drv_twi_data_count_get), (4 bytes).
    Removing nrf_drv_twi.o(i.nrf_drv_twi_is_busy), (28 bytes).
    Removing nrf_drv_twi.o(i.nrf_drv_twi_rx), (36 bytes).
    Removing nrf_drv_twi.o(i.nrf_drv_twi_start_task_get), (16 bytes).
    Removing nrf_drv_twi.o(i.nrf_drv_twi_stopped_event_get), (8 bytes).
    Removing nrf_drv_twi.o(i.nrf_drv_twi_tx), (38 bytes).
    Removing nrf_drv_twi.o(.constdata), (17 bytes).
    Removing nrf_drv_twi.o(.constdata), (10 bytes).
    Removing nrf_drv_twi.o(.constdata), (17 bytes).
    Removing nrf_drv_twi.o(.constdata), (12 bytes).
    Removing app_button.o(.rev16_text), (4 bytes).
    Removing app_button.o(.revsh_text), (4 bytes).
    Removing app_button.o(.rrx_text), (6 bytes).
    Removing app_button.o(i.app_button_disable), (48 bytes).
    Removing app_button.o(i.app_button_enable), (36 bytes).
    Removing app_button.o(i.app_button_init), (112 bytes).
    Removing app_button.o(i.app_button_is_pushed), (40 bytes).
    Removing app_button.o(i.detection_delay_timeout_handler), (112 bytes).
    Removing app_button.o(i.gpiote_event_handler), (88 bytes).
    Removing app_button.o(.bss), (32 bytes).
    Removing app_button.o(.constdata), (8 bytes).
    Removing app_button.o(.data), (20 bytes).
    Removing app_error.o(.rev16_text), (4 bytes).
    Removing app_error.o(.revsh_text), (4 bytes).
    Removing app_error.o(.rrx_text), (6 bytes).
    Removing app_error.o(i.app_error_handler), (24 bytes).
    Removing app_error.o(i.app_error_save_and_stop), (100 bytes).
    Removing app_error.o(.bss), (32 bytes).
    Removing app_error_weak.o(.rev16_text), (4 bytes).
    Removing app_error_weak.o(.revsh_text), (4 bytes).
    Removing app_error_weak.o(.rrx_text), (6 bytes).
    Removing app_scheduler.o(.rev16_text), (4 bytes).
    Removing app_scheduler.o(.revsh_text), (4 bytes).
    Removing app_scheduler.o(.rrx_text), (6 bytes).
    Removing app_scheduler.o(i.app_sched_event_put), (144 bytes).
    Removing app_scheduler.o(i.app_sched_execute), (64 bytes).
    Removing app_scheduler.o(i.app_sched_init), (56 bytes).
    Removing app_scheduler.o(i.app_sched_queue_space_get), (36 bytes).
    Removing app_scheduler.o(i.next_index), (24 bytes).
    Removing app_scheduler.o(.data), (16 bytes).
    Removing app_timer.o(.rev16_text), (4 bytes).
    Removing app_timer.o(.revsh_text), (4 bytes).
    Removing app_timer.o(.rrx_text), (6 bytes).
    Removing app_timer.o(i.app_timer_cnt_diff_compute), (8 bytes).
    Removing app_timer.o(i.app_timer_cnt_get), (12 bytes).
    Removing app_timer.o(i.app_timer_create), (52 bytes).
    Removing app_timer.o(i.app_timer_pause), (12 bytes).
    Removing app_timer.o(i.app_timer_resume), (12 bytes).
    Removing app_timer.o(i.app_timer_start), (60 bytes).
    Removing app_timer.o(i.app_timer_stop), (40 bytes).
    Removing app_timer.o(i.app_timer_stop_all), (24 bytes).
    Removing app_timer.o(i.timer_start_op_schedule), (92 bytes).
    Removing app_timer.o(i.timer_stop_op_schedule), (62 bytes).
    Removing app_timer.o(i.user_op_alloc), (48 bytes).
    Removing app_timer.o(i.user_op_enque), (12 bytes).
    Removing app_util_platform.o(.rev16_text), (4 bytes).
    Removing app_util_platform.o(.revsh_text), (4 bytes).
    Removing app_util_platform.o(.rrx_text), (6 bytes).
    Removing app_util_platform.o(i.app_util_disable_irq), (16 bytes).
    Removing app_util_platform.o(i.app_util_enable_irq), (20 bytes).
    Removing app_util_platform.o(i.current_int_priority_get), (54 bytes).
    Removing app_util_platform.o(i.privilege_level_get), (28 bytes).
    Removing app_util_platform.o(.data), (4 bytes).
    Removing hardfault_implementation.o(.rev16_text), (4 bytes).
    Removing hardfault_implementation.o(.revsh_text), (4 bytes).
    Removing hardfault_implementation.o(.rrx_text), (6 bytes).
    Removing nrf_assert.o(.rev16_text), (4 bytes).
    Removing nrf_assert.o(.revsh_text), (4 bytes).
    Removing nrf_assert.o(.rrx_text), (6 bytes).
    Removing nrf_assert.o(i.assert_nrf_callback), (22 bytes).
    Removing nrf_strerror.o(.rev16_text), (4 bytes).
    Removing nrf_strerror.o(.revsh_text), (4 bytes).
    Removing nrf_strerror.o(.rrx_text), (6 bytes).
    Removing nrf_strerror.o(i.nrf_strerror_find), (56 bytes).
    Removing nrf_strerror.o(i.nrf_strerror_get), (20 bytes).
    Removing nrf_strerror.o(.constdata), (260 bytes).
    Removing nrf_strerror.o(.conststring), (776 bytes).
    Removing app_twi.o(.rev16_text), (4 bytes).
    Removing app_twi.o(.revsh_text), (4 bytes).
    Removing app_twi.o(.rrx_text), (6 bytes).
    Removing app_twi.o(i.app_twi_uninit), (20 bytes).
    Removing nrf_queue.o(.rev16_text), (4 bytes).
    Removing nrf_queue.o(.revsh_text), (4 bytes).
    Removing nrf_queue.o(.rrx_text), (6 bytes).
    Removing nrf_queue.o(i.nrf_queue_available_get), (16 bytes).
    Removing nrf_queue.o(i.nrf_queue_in), (74 bytes).
    Removing nrf_queue.o(i.nrf_queue_max_utilization_get), (6 bytes).
    Removing nrf_queue.o(i.nrf_queue_out), (60 bytes).
    Removing nrf_queue.o(i.nrf_queue_read), (64 bytes).
    Removing nrf_queue.o(i.nrf_queue_reset), (32 bytes).
    Removing nrf_queue.o(i.nrf_queue_utilization_get), (34 bytes).
    Removing nrf_queue.o(i.nrf_queue_write), (68 bytes).
    Removing nrf_queue.o(i.queue_read), (104 bytes).
    Removing nrf_queue.o(i.queue_write), (146 bytes).
    Removing nrf_log_backend_serial.o(.rev16_text), (4 bytes).
    Removing nrf_log_backend_serial.o(.revsh_text), (4 bytes).
    Removing nrf_log_backend_serial.o(.rrx_text), (6 bytes).
    Removing nrf_log_backend_serial.o(i.nrf_log_backend_getchar), (4 bytes).
    Removing nrf_log_backend_serial.o(i.serial_get_byte), (10 bytes).
    Removing nrf_log_backend_serial.o(.constdata), (5 bytes).
    Removing nrf_log_frontend.o(.rev16_text), (4 bytes).
    Removing nrf_log_frontend.o(.revsh_text), (4 bytes).
    Removing nrf_log_frontend.o(.rrx_text), (6 bytes).
    Removing nrf_log_frontend.o(i.buffer_is_empty), (20 bytes).
    Removing nrf_log_frontend.o(i.nrf_log_blocking_backend_set), (6 bytes).
    Removing nrf_log_frontend.o(i.nrf_log_frontend_dequeue), (360 bytes).
    Removing nrf_log_frontend.o(i.nrf_log_frontend_std_2), (16 bytes).
    Removing nrf_log_frontend.o(i.nrf_log_frontend_std_3), (20 bytes).
    Removing nrf_log_frontend.o(i.nrf_log_frontend_std_4), (24 bytes).
    Removing nrf_log_frontend.o(i.nrf_log_frontend_std_5), (30 bytes).
    Removing nrf_log_frontend.o(i.nrf_log_frontend_std_6), (36 bytes).
    Removing nrf_log_frontend.o(i.nrf_log_getchar), (4 bytes).
    Removing nrf_log_frontend.o(i.nrf_log_push), (2 bytes).
    Removing segger_rtt.o(.rev16_text), (4 bytes).
    Removing segger_rtt.o(.revsh_text), (4 bytes).
    Removing segger_rtt.o(.rrx_text), (6 bytes).
    Removing segger_rtt.o(i.SEGGER_RTT_ConfigDownBuffer), (100 bytes).
    Removing segger_rtt.o(i.SEGGER_RTT_ConfigUpBuffer), (100 bytes).
    Removing segger_rtt.o(i.SEGGER_RTT_GetKey), (28 bytes).
    Removing segger_rtt.o(i.SEGGER_RTT_HasData), (24 bytes).
    Removing segger_rtt.o(i.SEGGER_RTT_HasKey), (36 bytes).
    Removing segger_rtt.o(i.SEGGER_RTT_Read), (44 bytes).
    Removing segger_rtt.o(i.SEGGER_RTT_ReadNoLock), (124 bytes).
    Removing segger_rtt.o(i.SEGGER_RTT_SetNameDownBuffer), (68 bytes).
    Removing segger_rtt.o(i.SEGGER_RTT_SetNameUpBuffer), (68 bytes).
    Removing segger_rtt.o(i.SEGGER_RTT_SetTerminal), (144 bytes).
    Removing segger_rtt.o(i.SEGGER_RTT_TerminalOut), (232 bytes).
    Removing segger_rtt.o(i.SEGGER_RTT_WaitKey), (12 bytes).
    Removing segger_rtt.o(i.SEGGER_RTT_Write), (60 bytes).
    Removing segger_rtt.o(i.SEGGER_RTT_WriteSkipNoLock), (160 bytes).
    Removing segger_rtt.o(i.SEGGER_RTT_WriteString), (26 bytes).
    Removing segger_rtt.o(i._PostTerminalSwitch), (32 bytes).
    Removing segger_rtt.o(.data), (17 bytes).
    Removing softdevice_handler.o(.rev16_text), (4 bytes).
    Removing softdevice_handler.o(.revsh_text), (4 bytes).
    Removing softdevice_handler.o(.rrx_text), (6 bytes).
    Removing softdevice_handler.o(i.softdevice_ble_evt_handler_set), (20 bytes).
    Removing softdevice_handler.o(i.softdevice_handler_is_suspended), (12 bytes).
    Removing softdevice_handler.o(i.softdevice_handler_resume), (72 bytes).
    Removing softdevice_handler.o(i.softdevice_handler_sd_disable), (28 bytes).
    Removing softdevice_handler.o(i.softdevice_handler_suspend), (64 bytes).
    Removing softdevice_handler.o(i.softdevice_sys_evt_handler_set), (20 bytes).
    Removing arm_startup_nrf52.o(HEAP), (8192 bytes).
    Removing system_nrf52.o(.rev16_text), (4 bytes).
    Removing system_nrf52.o(.revsh_text), (4 bytes).
    Removing system_nrf52.o(.rrx_text), (6 bytes).
    Removing dadd.o(.text), (334 bytes).
    Removing dmul.o(.text), (228 bytes).
    Removing ddiv.o(.text), (222 bytes).
    Removing dfixul.o(.text), (48 bytes).
    Removing cdrcmple.o(.text), (48 bytes).
    Removing depilogue.o(.text), (186 bytes).

291 unused section(s) (total 19511 bytes) removed from the image.

==============================================================================

Image Symbol Table

    Local Symbols

    Symbol Name                              Value     Ov Type        Size  Object(Section)

    ../clib/microlib/ctype/ctype.c           0x00000000   Number         0  isdigit_o.o ABSOLUTE
    ../clib/microlib/ctype/ctype.c           0x00000000   Number         0  isalpha_o.o ABSOLUTE
    ../clib/microlib/ctype/ctype.c           0x00000000   Number         0  isalnum_o.o ABSOLUTE
    ../clib/microlib/ctype/ctype.c           0x00000000   Number         0  ctype_o.o ABSOLUTE
    ../clib/microlib/ctype/ctype.c           0x00000000   Number         0  iscntrl_o.o ABSOLUTE
    ../clib/microlib/ctype/ctype.c           0x00000000   Number         0  isblank_o.o ABSOLUTE
    ../clib/microlib/ctype/ctype.c           0x00000000   Number         0  isgraph_o.o ABSOLUTE
    ../clib/microlib/ctype/ctype.c           0x00000000   Number         0  islower_o.o ABSOLUTE
    ../clib/microlib/ctype/ctype.c           0x00000000   Number         0  isprint_o.o ABSOLUTE
    ../clib/microlib/ctype/ctype.c           0x00000000   Number         0  ispunct_o.o ABSOLUTE
    ../clib/microlib/ctype/ctype.c           0x00000000   Number         0  isspace_o.o ABSOLUTE
    ../clib/microlib/ctype/ctype.c           0x00000000   Number         0  isupper_o.o ABSOLUTE
    ../clib/microlib/ctype/ctype.c           0x00000000   Number         0  isxdigit_o.o ABSOLUTE
    ../clib/microlib/division.c              0x00000000   Number         0  uldiv.o ABSOLUTE
    ../clib/microlib/division.c              0x00000000   Number         0  uidiv.o ABSOLUTE
    ../clib/microlib/init/entry.s            0x00000000   Number         0  entry8b.o ABSOLUTE
    ../clib/microlib/init/entry.s            0x00000000   Number         0  entry7b.o ABSOLUTE
    ../clib/microlib/init/entry.s            0x00000000   Number         0  entry7a.o ABSOLUTE
    ../clib/microlib/init/entry.s            0x00000000   Number         0  entry.o ABSOLUTE
    ../clib/microlib/init/entry.s            0x00000000   Number         0  entry8a.o ABSOLUTE
    ../clib/microlib/init/entry.s            0x00000000   Number         0  entry5.o ABSOLUTE
    ../clib/microlib/init/entry.s            0x00000000   Number         0  entry9b.o ABSOLUTE
    ../clib/microlib/init/entry.s            0x00000000   Number         0  entry11b.o ABSOLUTE
    ../clib/microlib/init/entry.s            0x00000000   Number         0  entry11a.o ABSOLUTE
    ../clib/microlib/init/entry.s            0x00000000   Number         0  entry10b.o ABSOLUTE
    ../clib/microlib/init/entry.s            0x00000000   Number         0  entry10a.o ABSOLUTE
    ../clib/microlib/init/entry.s            0x00000000   Number         0  entry2.o ABSOLUTE
    ../clib/microlib/init/entry.s            0x00000000   Number         0  entry9a.o ABSOLUTE
    ../clib/microlib/longlong.c              0x00000000   Number         0  llshl.o ABSOLUTE
    ../clib/microlib/longlong.c              0x00000000   Number         0  llushr.o ABSOLUTE
    ../clib/microlib/longlong.c              0x00000000   Number         0  llsshr.o ABSOLUTE
    ../clib/microlib/printf/printf.c         0x00000000   Number         0  printf4.o ABSOLUTE
    ../clib/microlib/printf/printf.c         0x00000000   Number         0  printf6.o ABSOLUTE
    ../clib/microlib/printf/printf.c         0x00000000   Number         0  printf7.o ABSOLUTE
    ../clib/microlib/printf/printf.c         0x00000000   Number         0  printfa.o ABSOLUTE
    ../clib/microlib/printf/printf.c         0x00000000   Number         0  printf8.o ABSOLUTE
    ../clib/microlib/printf/printf.c         0x00000000   Number         0  printf5.o ABSOLUTE
    ../clib/microlib/printf/printf.c         0x00000000   Number         0  printf1.o ABSOLUTE
    ../clib/microlib/printf/printf.c         0x00000000   Number         0  printfb.o ABSOLUTE
    ../clib/microlib/printf/printf.c         0x00000000   Number         0  printf0.o ABSOLUTE
    ../clib/microlib/printf/printf.c         0x00000000   Number         0  printf2.o ABSOLUTE
    ../clib/microlib/printf/printf.c         0x00000000   Number         0  printf3.o ABSOLUTE
    ../clib/microlib/printf/stubs.s          0x00000000   Number         0  stubs.o ABSOLUTE
    ../clib/microlib/stdio/fputc.c           0x00000000   Number         0  fputc.o ABSOLUTE
    ../clib/microlib/stdio/semi.s            0x00000000   Number         0  semi.o ABSOLUTE
    ../clib/microlib/stdio/streams.c         0x00000000   Number         0  stdout.o ABSOLUTE
    ../clib/microlib/string/memcmp.c         0x00000000   Number         0  memcmp.o ABSOLUTE
    ../clib/microlib/string/memcpy.c         0x00000000   Number         0  memcpyb.o ABSOLUTE
    ../clib/microlib/string/memcpy.c         0x00000000   Number         0  memcpya.o ABSOLUTE
    ../clib/microlib/string/memset.c         0x00000000   Number         0  memseta.o ABSOLUTE
    ../clib/microlib/string/strcpy.c         0x00000000   Number         0  strcpy.o ABSOLUTE
    ../clib/microlib/string/strlen.c         0x00000000   Number         0  strlen.o ABSOLUTE
    ../clib/microlib/stubs.s                 0x00000000   Number         0  iusefp.o ABSOLUTE
    ../clib/microlib/stubs.s                 0x00000000   Number         0  iusesemip.o ABSOLUTE
    ../fplib/microlib/fpadd.c                0x00000000   Number         0  dadd.o ABSOLUTE
    ../fplib/microlib/fpdiv.c                0x00000000   Number         0  ddiv.o ABSOLUTE
    ../fplib/microlib/fpepilogue.c           0x00000000   Number         0  depilogue.o ABSOLUTE
    ../fplib/microlib/fpfix.c                0x00000000   Number         0  dfixul.o ABSOLUTE
    ../fplib/microlib/fpmul.c                0x00000000   Number         0  dmul.o ABSOLUTE
    ..\..\..\..\..\..\components\ble\common\ble_advdata.c 0x00000000   Number         0  ble_advdata.o ABSOLUTE
    ..\..\..\..\..\..\components\ble\common\ble_conn_params.c 0x00000000   Number         0  ble_conn_params.o ABSOLUTE
    ..\..\..\..\..\..\components\ble\common\ble_srv_common.c 0x00000000   Number         0  ble_srv_common.o ABSOLUTE
    ..\..\..\..\..\..\components\boards\boards.c 0x00000000   Number         0  boards.o ABSOLUTE
    ..\..\..\..\..\..\components\drivers_nrf\clock\nrf_drv_clock.c 0x00000000   Number         0  nrf_drv_clock.o ABSOLUTE
    ..\..\..\..\..\..\components\drivers_nrf\common\nrf_drv_common.c 0x00000000   Number         0  nrf_drv_common.o ABSOLUTE
    ..\..\..\..\..\..\components\drivers_nrf\gpiote\nrf_drv_gpiote.c 0x00000000   Number         0  nrf_drv_gpiote.o ABSOLUTE
    ..\..\..\..\..\..\components\drivers_nrf\twi_master\nrf_drv_twi.c 0x00000000   Number         0  nrf_drv_twi.o ABSOLUTE
    ..\..\..\..\..\..\components\drivers_nrf\uart\nrf_drv_uart.c 0x00000000   Number         0  nrf_drv_uart.o ABSOLUTE
    ..\..\..\..\..\..\components\libraries\bsp\bsp.c 0x00000000   Number         0  bsp.o ABSOLUTE
    ..\..\..\..\..\..\components\libraries\bsp\bsp_nfc.c 0x00000000   Number         0  bsp_nfc.o ABSOLUTE
    ..\..\..\..\..\..\components\libraries\button\app_button.c 0x00000000   Number         0  app_button.o ABSOLUTE
    ..\..\..\..\..\..\components\libraries\hardfault\hardfault_implementation.c 0x00000000   Number         0  hardfault_implementation.o ABSOLUTE
    ..\..\..\..\..\..\components\libraries\log\src\nrf_log_backend_serial.c 0x00000000   Number         0  nrf_log_backend_serial.o ABSOLUTE
    ..\..\..\..\..\..\components\libraries\log\src\nrf_log_frontend.c 0x00000000   Number         0  nrf_log_frontend.o ABSOLUTE
    ..\..\..\..\..\..\components\libraries\queue\nrf_queue.c 0x00000000   Number         0  nrf_queue.o ABSOLUTE
    ..\..\..\..\..\..\components\libraries\scheduler\app_scheduler.c 0x00000000   Number         0  app_scheduler.o ABSOLUTE
    ..\..\..\..\..\..\components\libraries\strerror\nrf_strerror.c 0x00000000   Number         0  nrf_strerror.o ABSOLUTE
    ..\..\..\..\..\..\components\libraries\timer\app_timer.c 0x00000000   Number         0  app_timer.o ABSOLUTE
    ..\..\..\..\..\..\components\libraries\twi\app_twi.c 0x00000000   Number         0  app_twi.o ABSOLUTE
    ..\..\..\..\..\..\components\libraries\util\app_error.c 0x00000000   Number         0  app_error.o ABSOLUTE
    ..\..\..\..\..\..\components\libraries\util\app_error_weak.c 0x00000000   Number         0  app_error_weak.o ABSOLUTE
    ..\..\..\..\..\..\components\libraries\util\app_util_platform.c 0x00000000   Number         0  app_util_platform.o ABSOLUTE
    ..\..\..\..\..\..\components\libraries\util\nrf_assert.c 0x00000000   Number         0  nrf_assert.o ABSOLUTE
    ..\..\..\..\..\..\components\softdevice\common\softdevice_handler\softdevice_handler.c 0x00000000   Number         0  softdevice_handler.o ABSOLUTE
    ..\..\..\..\..\..\external\segger_rtt\RTT_Syscalls_KEIL.c 0x00000000   Number         0  rtt_syscalls_keil.o ABSOLUTE
    ..\..\..\..\..\..\external\segger_rtt\SEGGER_RTT.c 0x00000000   Number         0  segger_rtt.o ABSOLUTE
    ..\..\..\..\..\..\external\segger_rtt\SEGGER_RTT_printf.c 0x00000000   Number         0  segger_rtt_printf.o ABSOLUTE
    ..\..\..\main.c                          0x00000000   Number         0  main.o ABSOLUTE
    ..\..\..\twi_slave_tiny_unwrap.c         0x00000000   Number         0  twi_slave_tiny_unwrap.o ABSOLUTE
    ..\\..\\..\\..\\..\\..\\components\\ble\\common\\ble_advdata.c 0x00000000   Number         0  ble_advdata.o ABSOLUTE
    ..\\..\\..\\..\\..\\..\\components\\ble\\common\\ble_conn_params.c 0x00000000   Number         0  ble_conn_params.o ABSOLUTE
    ..\\..\\..\\..\\..\\..\\components\\ble\\common\\ble_srv_common.c 0x00000000   Number         0  ble_srv_common.o ABSOLUTE
    ..\\..\\..\\..\\..\\..\\components\\boards\\boards.c 0x00000000   Number         0  boards.o ABSOLUTE
    ..\\..\\..\\..\\..\\..\\components\\drivers_nrf\\clock\\nrf_drv_clock.c 0x00000000   Number         0  nrf_drv_clock.o ABSOLUTE
    ..\\..\\..\\..\\..\\..\\components\\drivers_nrf\\common\\nrf_drv_common.c 0x00000000   Number         0  nrf_drv_common.o ABSOLUTE
    ..\\..\\..\\..\\..\\..\\components\\drivers_nrf\\gpiote\\nrf_drv_gpiote.c 0x00000000   Number         0  nrf_drv_gpiote.o ABSOLUTE
    ..\\..\\..\\..\\..\\..\\components\\drivers_nrf\\twi_master\\nrf_drv_twi.c 0x00000000   Number         0  nrf_drv_twi.o ABSOLUTE
    ..\\..\\..\\..\\..\\..\\components\\drivers_nrf\\uart\\nrf_drv_uart.c 0x00000000   Number         0  nrf_drv_uart.o ABSOLUTE
    ..\\..\\..\\..\\..\\..\\components\\libraries\\bsp\\bsp.c 0x00000000   Number         0  bsp.o ABSOLUTE
    ..\\..\\..\\..\\..\\..\\components\\libraries\\bsp\\bsp_nfc.c 0x00000000   Number         0  bsp_nfc.o ABSOLUTE
    ..\\..\\..\\..\\..\\..\\components\\libraries\\button\\app_button.c 0x00000000   Number         0  app_button.o ABSOLUTE
    ..\\..\\..\\..\\..\\..\\components\\libraries\\hardfault\\hardfault_implementation.c 0x00000000   Number         0  hardfault_implementation.o ABSOLUTE
    ..\\..\\..\\..\\..\\..\\components\\libraries\\log\\src\\nrf_log_backend_serial.c 0x00000000   Number         0  nrf_log_backend_serial.o ABSOLUTE
    ..\\..\\..\\..\\..\\..\\components\\libraries\\log\\src\\nrf_log_frontend.c 0x00000000   Number         0  nrf_log_frontend.o ABSOLUTE
    ..\\..\\..\\..\\..\\..\\components\\libraries\\queue\\nrf_queue.c 0x00000000   Number         0  nrf_queue.o ABSOLUTE
    ..\\..\\..\\..\\..\\..\\components\\libraries\\scheduler\\app_scheduler.c 0x00000000   Number         0  app_scheduler.o ABSOLUTE
    ..\\..\\..\\..\\..\\..\\components\\libraries\\strerror\\nrf_strerror.c 0x00000000   Number         0  nrf_strerror.o ABSOLUTE
    ..\\..\\..\\..\\..\\..\\components\\libraries\\timer\\app_timer.c 0x00000000   Number         0  app_timer.o ABSOLUTE
    ..\\..\\..\\..\\..\\..\\components\\libraries\\twi\\app_twi.c 0x00000000   Number         0  app_twi.o ABSOLUTE
    ..\\..\\..\\..\\..\\..\\components\\libraries\\util\\app_error.c 0x00000000   Number         0  app_error.o ABSOLUTE
    ..\\..\\..\\..\\..\\..\\components\\libraries\\util\\app_error_weak.c 0x00000000   Number         0  app_error_weak.o ABSOLUTE
    ..\\..\\..\\..\\..\\..\\components\\libraries\\util\\app_util_platform.c 0x00000000   Number         0  app_util_platform.o ABSOLUTE
    ..\\..\\..\\..\\..\\..\\components\\libraries\\util\\nrf_assert.c 0x00000000   Number         0  nrf_assert.o ABSOLUTE
    ..\\..\\..\\..\\..\\..\\components\\softdevice\\common\\softdevice_handler\\softdevice_handler.c 0x00000000   Number         0  softdevice_handler.o ABSOLUTE
    ..\\..\\..\\..\\..\\..\\external\\segger_rtt\\SEGGER_RTT.c 0x00000000   Number         0  segger_rtt.o ABSOLUTE
    ..\\..\\..\\main.c                       0x00000000   Number         0  main.o ABSOLUTE
    ..\\..\\..\\twi_slave_tiny_unwrap.c      0x00000000   Number         0  twi_slave_tiny_unwrap.o ABSOLUTE
    RTE\Device\nRF52832_xxAA\arm_startup_nrf52.s 0x00000000   Number         0  arm_startup_nrf52.o ABSOLUTE
    RTE\Device\nRF52832_xxAA\system_nrf52.c  0x00000000   Number         0  system_nrf52.o ABSOLUTE
    RTE\\Device\\nRF52832_xxAA\\system_nrf52.c 0x00000000   Number         0  system_nrf52.o ABSOLUTE
    cdrcmple.s                               0x00000000   Number         0  cdrcmple.o ABSOLUTE
    dc.s                                     0x00000000   Number         0  dc.o ABSOLUTE
    handlers.s                               0x00000000   Number         0  handlers.o ABSOLUTE
    init.s                                   0x00000000   Number         0  init.o ABSOLUTE
    RESET                                    0x0001f000   Section      512  arm_startup_nrf52.o(RESET)
    .ARM.Collect$$$$00000000                 0x0001f200   Section        0  entry.o(.ARM.Collect$$$$00000000)
    .ARM.Collect$$$$00000001                 0x0001f200   Section        4  entry2.o(.ARM.Collect$$$$00000001)
    .ARM.Collect$$$$00000004                 0x0001f204   Section        4  entry5.o(.ARM.Collect$$$$00000004)
    .ARM.Collect$$$$00000008                 0x0001f208   Section        0  entry7b.o(.ARM.Collect$$$$00000008)
    .ARM.Collect$$$$0000000A                 0x0001f208   Section        0  entry8b.o(.ARM.Collect$$$$0000000A)
    .ARM.Collect$$$$0000000B                 0x0001f208   Section        8  entry9a.o(.ARM.Collect$$$$0000000B)
    .ARM.Collect$$$$0000000D                 0x0001f210   Section        0  entry10a.o(.ARM.Collect$$$$0000000D)
    .ARM.Collect$$$$0000000F                 0x0001f210   Section        0  entry11a.o(.ARM.Collect$$$$0000000F)
    .ARM.Collect$$$$00002712                 0x0001f210   Section        4  entry2.o(.ARM.Collect$$$$00002712)
    __lit__00000000                          0x0001f210   Data           4  entry2.o(.ARM.Collect$$$$00002712)
    .text                                    0x0001f214   Section       36  arm_startup_nrf52.o(.text)
    $v0                                      0x0001f214   Number         0  arm_startup_nrf52.o(.text)
    .text                                    0x0001f238   Section        0  ctype_o.o(.text)
    .text                                    0x0001f240   Section        0  memcpya.o(.text)
    .text                                    0x0001f264   Section        0  memseta.o(.text)
    .text                                    0x0001f288   Section        0  strlen.o(.text)
    .text                                    0x0001f296   Section        0  memcmp.o(.text)
    .text                                    0x0001f2b0   Section        0  strcpy.o(.text)
    .text                                    0x0001f2c2   Section        0  uldiv.o(.text)
    .text                                    0x0001f324   Section       36  init.o(.text)
    .text                                    0x0001f348   Section        0  llshl.o(.text)
    .text                                    0x0001f366   Section        0  llushr.o(.text)
    i.GPIOTE_IRQHandler                      0x0001f388   Section        0  nrf_drv_gpiote.o(i.GPIOTE_IRQHandler)
    i.POWER_CLOCK_IRQHandler                 0x0001f534   Section        0  nrf_drv_clock.o(i.POWER_CLOCK_IRQHandler)
    i.RTC1_IRQHandler                        0x0001f58c   Section        0  app_timer.o(i.RTC1_IRQHandler)
    i.SEGGER_RTT_Init                        0x0001f5a4   Section        0  segger_rtt.o(i.SEGGER_RTT_Init)
    i.SEGGER_RTT_WriteNoLock                 0x0001f5b8   Section        0  segger_rtt.o(i.SEGGER_RTT_WriteNoLock)
    i.SPIM0_SPIS0_TWIM0_TWIS0_SPI0_TWI0_IRQHandler 0x0001f624   Section        0  nrf_drv_twi.o(i.SPIM0_SPIS0_TWIM0_TWIS0_SPI0_TWI0_IRQHandler)
    i.SWI0_EGU0_IRQHandler                   0x0001f634   Section        0  app_timer.o(i.SWI0_EGU0_IRQHandler)
    i.SWI2_EGU2_IRQHandler                   0x0001f638   Section        0  softdevice_handler.o(i.SWI2_EGU2_IRQHandler)
    i.SystemCoreClockUpdate                  0x0001f660   Section        0  system_nrf52.o(i.SystemCoreClockUpdate)
    i.SystemInit                             0x0001f670   Section        0  system_nrf52.o(i.SystemInit)
    i._DoInit                                0x0001f834   Section        0  segger_rtt.o(i._DoInit)
    _DoInit                                  0x0001f835   Thumb Code    76  segger_rtt.o(i._DoInit)
    i._GetAvailWriteSpace                    0x0001f89c   Section        0  segger_rtt.o(i._GetAvailWriteSpace)
    _GetAvailWriteSpace                      0x0001f89d   Thumb Code    24  segger_rtt.o(i._GetAvailWriteSpace)
    i._WriteBlocking                         0x0001f8b4   Section        0  segger_rtt.o(i._WriteBlocking)
    _WriteBlocking                           0x0001f8b5   Thumb Code    92  segger_rtt.o(i._WriteBlocking)
    i._WriteNoCheck                          0x0001f910   Section        0  segger_rtt.o(i._WriteNoCheck)
    _WriteNoCheck                            0x0001f911   Thumb Code    68  segger_rtt.o(i._WriteNoCheck)
    i.__0snprintf$8                          0x0001f954   Section        0  printf8.o(i.__0snprintf$8)
    i.__NVIC_ClearPendingIRQ                 0x0001f984   Section        0  app_timer.o(i.__NVIC_ClearPendingIRQ)
    __NVIC_ClearPendingIRQ                   0x0001f985   Thumb Code    26  app_timer.o(i.__NVIC_ClearPendingIRQ)
    i.__NVIC_DisableIRQ                      0x0001f99e   Section        0  softdevice_handler.o(i.__NVIC_DisableIRQ)
    __NVIC_DisableIRQ                        0x0001f99f   Thumb Code    34  softdevice_handler.o(i.__NVIC_DisableIRQ)
    i.__NVIC_EnableIRQ                       0x0001f9c0   Section        0  app_timer.o(i.__NVIC_EnableIRQ)
    __NVIC_EnableIRQ                         0x0001f9c1   Thumb Code    26  app_timer.o(i.__NVIC_EnableIRQ)
    i.__NVIC_EnableIRQ                       0x0001f9da   Section        0  softdevice_handler.o(i.__NVIC_EnableIRQ)
    __NVIC_EnableIRQ                         0x0001f9db   Thumb Code    26  softdevice_handler.o(i.__NVIC_EnableIRQ)
    i.__NVIC_SetPendingIRQ                   0x0001f9f4   Section        0  app_timer.o(i.__NVIC_SetPendingIRQ)
    __NVIC_SetPendingIRQ                     0x0001f9f5   Thumb Code    26  app_timer.o(i.__NVIC_SetPendingIRQ)
    i.__NVIC_SetPriority                     0x0001fa0e   Section        0  app_timer.o(i.__NVIC_SetPriority)
    __NVIC_SetPriority                       0x0001fa0f   Thumb Code    32  app_timer.o(i.__NVIC_SetPriority)
    i.__scatterload_copy                     0x0001fa2e   Section       14  handlers.o(i.__scatterload_copy)
    i.__scatterload_null                     0x0001fa3c   Section        2  handlers.o(i.__scatterload_null)
    i.__scatterload_zeroinit                 0x0001fa3e   Section       14  handlers.o(i.__scatterload_zeroinit)
    i.__sd_nvic_app_accessible_irq           0x0001fa4c   Section        0  softdevice_handler.o(i.__sd_nvic_app_accessible_irq)
    __sd_nvic_app_accessible_irq             0x0001fa4d   Thumb Code    44  softdevice_handler.o(i.__sd_nvic_app_accessible_irq)
    i._printf_core                           0x0001fa7c   Section        0  printf8.o(i._printf_core)
    _printf_core                             0x0001fa7d   Thumb Code   996  printf8.o(i._printf_core)
    i._printf_post_padding                   0x0001fe8c   Section        0  printf8.o(i._printf_post_padding)
    _printf_post_padding                     0x0001fe8d   Thumb Code    36  printf8.o(i._printf_post_padding)
    i._printf_pre_padding                    0x0001feb0   Section        0  printf8.o(i._printf_pre_padding)
    _printf_pre_padding                      0x0001feb1   Thumb Code    46  printf8.o(i._printf_pre_padding)
    i._snputc                                0x0001fede   Section        0  printf8.o(i._snputc)
    _snputc                                  0x0001fedf   Thumb Code    22  printf8.o(i._snputc)
    i.adv_data_encode                        0x0001fef4   Section        0  ble_advdata.o(i.adv_data_encode)
    i.advdata_check                          0x00020002   Section        0  ble_advdata.o(i.advdata_check)
    advdata_check                            0x00020003   Thumb Code    14  ble_advdata.o(i.advdata_check)
    i.advertising_init                       0x00020010   Section        0  main.o(i.advertising_init)
    advertising_init                         0x00020011   Thumb Code    86  main.o(i.advertising_init)
    i.advertising_start                      0x00020070   Section        0  main.o(i.advertising_start)
    advertising_start                        0x00020071   Thumb Code    36  main.o(i.advertising_start)
    i.app_error_fault_handler                0x00020098   Section        0  app_error_weak.o(i.app_error_fault_handler)
    i.app_error_handler_bare                 0x000200f8   Section        0  app_error.o(i.app_error_handler_bare)
    i.app_timer_init                         0x00020110   Section        0  app_timer.o(i.app_timer_init)
    i.app_twi_init                           0x0002015c   Section        0  app_twi.o(i.app_twi_init)
    i.app_twi_perform                        0x0002019c   Section        0  app_twi.o(i.app_twi_perform)
    i.app_twi_schedule                       0x0002020c   Section        0  app_twi.o(i.app_twi_schedule)
    i.app_util_critical_region_enter         0x00020228   Section        0  app_util_platform.o(i.app_util_critical_region_enter)
    i.app_util_critical_region_exit          0x0002026c   Section        0  app_util_platform.o(i.app_util_critical_region_exit)
    i.appearance_encode                      0x0002029c   Section        0  ble_advdata.o(i.appearance_encode)
    appearance_encode                        0x0002029d   Thumb Code    72  ble_advdata.o(i.appearance_encode)
    i.ble_advdata_set                        0x000202e4   Section        0  ble_advdata.o(i.ble_advdata_set)
    i.ble_device_addr_encode                 0x0002034e   Section        0  ble_advdata.o(i.ble_device_addr_encode)
    ble_device_addr_encode                   0x0002034f   Thumb Code   102  ble_advdata.o(i.ble_device_addr_encode)
    i.ble_stack_init                         0x000203b4   Section        0  main.o(i.ble_stack_init)
    ble_stack_init                           0x000203b5   Thumb Code   142  main.o(i.ble_stack_init)
    i.bsp_indication_set                     0x0002044c   Section        0  bsp.o(i.bsp_indication_set)
    i.buf_len_update                         0x00020450   Section        0  nrf_log_backend_serial.o(i.buf_len_update)
    buf_len_update                           0x00020451   Thumb Code    18  nrf_log_backend_serial.o(i.buf_len_update)
    i.byte2hex                               0x00020462   Section        0  nrf_log_backend_serial.o(i.byte2hex)
    byte2hex                                 0x00020463   Thumb Code    42  nrf_log_backend_serial.o(i.byte2hex)
    i.channel_port_get                       0x0002048c   Section        0  nrf_drv_gpiote.o(i.channel_port_get)
    channel_port_get                         0x0002048d   Thumb Code    10  nrf_drv_gpiote.o(i.channel_port_get)
    i.clock_clk_started_notify               0x0002049c   Section        0  nrf_drv_clock.o(i.clock_clk_started_notify)
    clock_clk_started_notify                 0x0002049d   Thumb Code    36  nrf_drv_clock.o(i.clock_clk_started_notify)
    i.compare_reg_update                     0x000204c4   Section        0  app_timer.o(i.compare_reg_update)
    compare_reg_update                       0x000204c5   Thumb Code   112  app_timer.o(i.compare_reg_update)
    i.conn_int_check                         0x0002053c   Section        0  ble_advdata.o(i.conn_int_check)
    conn_int_check                           0x0002053d   Thumb Code    64  ble_advdata.o(i.conn_int_check)
    i.conn_int_encode                        0x0002057c   Section        0  ble_advdata.o(i.conn_int_encode)
    conn_int_encode                          0x0002057d   Thumb Code    90  ble_advdata.o(i.conn_int_encode)
    i.elapsed_ticks_acquire                  0x000205d8   Section        0  app_timer.o(i.elapsed_ticks_acquire)
    elapsed_ticks_acquire                    0x000205d9   Thumb Code    58  app_timer.o(i.elapsed_ticks_acquire)
    i.errata_108                             0x00020618   Section        0  system_nrf52.o(i.errata_108)
    errata_108                               0x00020619   Thumb Code    56  system_nrf52.o(i.errata_108)
    i.errata_12                              0x00020654   Section        0  system_nrf52.o(i.errata_12)
    errata_12                                0x00020655   Thumb Code    56  system_nrf52.o(i.errata_12)
    i.errata_136                             0x00020690   Section        0  system_nrf52.o(i.errata_136)
    errata_136                               0x00020691   Thumb Code    56  system_nrf52.o(i.errata_136)
    i.errata_16                              0x000206cc   Section        0  system_nrf52.o(i.errata_16)
    errata_16                                0x000206cd   Thumb Code    40  system_nrf52.o(i.errata_16)
    i.errata_182                             0x000206f8   Section        0  system_nrf52.o(i.errata_182)
    errata_182                               0x000206f9   Thumb Code    28  system_nrf52.o(i.errata_182)
    i.errata_31                              0x00020714   Section        0  system_nrf52.o(i.errata_31)
    errata_31                                0x00020715   Thumb Code    56  system_nrf52.o(i.errata_31)
    i.errata_32                              0x00020750   Section        0  system_nrf52.o(i.errata_32)
    errata_32                                0x00020751   Thumb Code    40  system_nrf52.o(i.errata_32)
    i.errata_36                              0x0002077c   Section        0  system_nrf52.o(i.errata_36)
    errata_36                                0x0002077d   Thumb Code    56  system_nrf52.o(i.errata_36)
    i.errata_37                              0x000207b8   Section        0  system_nrf52.o(i.errata_37)
    errata_37                                0x000207b9   Thumb Code    40  system_nrf52.o(i.errata_37)
    i.errata_57                              0x000207e4   Section        0  system_nrf52.o(i.errata_57)
    errata_57                                0x000207e5   Thumb Code    40  system_nrf52.o(i.errata_57)
    i.errata_66                              0x00020810   Section        0  system_nrf52.o(i.errata_66)
    errata_66                                0x00020811   Thumb Code    40  system_nrf52.o(i.errata_66)
    i.expired_timers_handler                 0x0002083c   Section        0  app_timer.o(i.expired_timers_handler)
    expired_timers_handler                   0x0002083d   Thumb Code    68  app_timer.o(i.expired_timers_handler)
    i.flags_encode                           0x00020884   Section        0  ble_advdata.o(i.flags_encode)
    flags_encode                             0x00020885   Thumb Code    50  ble_advdata.o(i.flags_encode)
    i.intern_softdevice_events_execute       0x000208b8   Section        0  softdevice_handler.o(i.intern_softdevice_events_execute)
    i.internal_transaction_cb                0x00020930   Section        0  app_twi.o(i.internal_transaction_cb)
    internal_transaction_cb                  0x00020931   Thumb Code    12  app_twi.o(i.internal_transaction_cb)
    i.irq_handler_twim                       0x0002093c   Section        0  nrf_drv_twi.o(i.irq_handler_twim)
    irq_handler_twim                         0x0002093d   Thumb Code   406  nrf_drv_twi.o(i.irq_handler_twim)
    i.item_dequeue                           0x00020ad2   Section        0  nrf_drv_clock.o(i.item_dequeue)
    item_dequeue                             0x00020ad3   Thumb Code    14  nrf_drv_clock.o(i.item_dequeue)
    i.list_insertions_handler                0x00020ae0   Section        0  app_timer.o(i.list_insertions_handler)
    list_insertions_handler                  0x00020ae1   Thumb Code   236  app_timer.o(i.list_insertions_handler)
    i.log_init                               0x00020bd8   Section        0  main.o(i.log_init)
    log_init                                 0x00020bd9   Thumb Code    22  main.o(i.log_init)
    i.main                                   0x00020bf0   Section        0  main.o(i.main)
    i.manuf_specific_data_encode             0x00020c50   Section        0  ble_advdata.o(i.manuf_specific_data_encode)
    manuf_specific_data_encode               0x00020c51   Thumb Code   104  ble_advdata.o(i.manuf_specific_data_encode)
    i.name_encode                            0x00020cb8   Section        0  ble_advdata.o(i.name_encode)
    name_encode                              0x00020cb9   Thumb Code   154  ble_advdata.o(i.name_encode)
    i.nrf_bitmask_bit_is_set                 0x00020d52   Section        0  nrf_drv_gpiote.o(i.nrf_bitmask_bit_is_set)
    nrf_bitmask_bit_is_set                   0x00020d53   Thumb Code    16  nrf_drv_gpiote.o(i.nrf_bitmask_bit_is_set)
    i.nrf_clock_event_check                  0x00020d62   Section        0  nrf_drv_clock.o(i.nrf_clock_event_check)
    nrf_clock_event_check                    0x00020d63   Thumb Code    14  nrf_drv_clock.o(i.nrf_clock_event_check)
    i.nrf_clock_event_clear                  0x00020d70   Section        0  nrf_drv_clock.o(i.nrf_clock_event_clear)
    nrf_clock_event_clear                    0x00020d71   Thumb Code    16  nrf_drv_clock.o(i.nrf_clock_event_clear)
    i.nrf_delay_us                           0x00020d80   Section        0  nrf_drv_twi.o(i.nrf_delay_us)
    nrf_delay_us                             0x00020d81   Thumb Code   132  nrf_drv_twi.o(i.nrf_delay_us)
    i.nrf_delay_us                           0x00020e0c   Section        0  app_timer.o(i.nrf_delay_us)
    nrf_delay_us                             0x00020e0d   Thumb Code   132  app_timer.o(i.nrf_delay_us)
    i.nrf_drv_clock_init                     0x00020e98   Section        0  nrf_drv_clock.o(i.nrf_drv_clock_init)
    i.nrf_drv_clock_on_sd_enable             0x00020eec   Section        0  nrf_drv_clock.o(i.nrf_drv_clock_on_sd_enable)
    i.nrf_drv_clock_on_soc_event             0x00020f1c   Section        0  nrf_drv_clock.o(i.nrf_drv_clock_on_soc_event)
    i.nrf_drv_common_irq_enable              0x00020f26   Section        0  nrf_drv_common.o(i.nrf_drv_common_irq_enable)
    i.nrf_drv_is_in_RAM                      0x00020f62   Section        0  nrf_drv_twi.o(i.nrf_drv_is_in_RAM)
    nrf_drv_is_in_RAM                        0x00020f63   Thumb Code    16  nrf_drv_twi.o(i.nrf_drv_is_in_RAM)
    i.nrf_drv_twi_disable                    0x00020f74   Section        0  nrf_drv_twi.o(i.nrf_drv_twi_disable)
    i.nrf_drv_twi_enable                     0x00020fa8   Section        0  nrf_drv_twi.o(i.nrf_drv_twi_enable)
    i.nrf_drv_twi_init                       0x00020fcc   Section        0  nrf_drv_twi.o(i.nrf_drv_twi_init)
    i.nrf_drv_twi_uninit                     0x00021060   Section        0  nrf_drv_twi.o(i.nrf_drv_twi_uninit)
    i.nrf_drv_twi_xfer                       0x000210dc   Section        0  nrf_drv_twi.o(i.nrf_drv_twi_xfer)
    i.nrf_gpio_cfg_sense_set                 0x00021104   Section        0  nrf_drv_gpiote.o(i.nrf_gpio_cfg_sense_set)
    nrf_gpio_cfg_sense_set                   0x00021105   Thumb Code    30  nrf_drv_gpiote.o(i.nrf_gpio_cfg_sense_set)
    i.nrf_gpio_pin_set                       0x00021122   Section        0  nrf_drv_twi.o(i.nrf_gpio_pin_set)
    nrf_gpio_pin_set                         0x00021123   Thumb Code    16  nrf_drv_twi.o(i.nrf_gpio_pin_set)
    i.nrf_gpio_ports_read                    0x00021134   Section        0  nrf_drv_gpiote.o(i.nrf_gpio_ports_read)
    nrf_gpio_ports_read                      0x00021135   Thumb Code    32  nrf_drv_gpiote.o(i.nrf_gpio_ports_read)
    i.nrf_gpiote_event_clear                 0x00021158   Section        0  nrf_drv_gpiote.o(i.nrf_gpiote_event_clear)
    nrf_gpiote_event_clear                   0x00021159   Thumb Code    16  nrf_drv_gpiote.o(i.nrf_gpiote_event_clear)
    i.nrf_gpiote_event_is_set                0x0002116c   Section        0  nrf_drv_gpiote.o(i.nrf_gpiote_event_is_set)
    nrf_gpiote_event_is_set                  0x0002116d   Thumb Code    14  nrf_drv_gpiote.o(i.nrf_gpiote_event_is_set)
    i.nrf_log_backend_hexdump_handler_get    0x00021180   Section        0  nrf_log_backend_serial.o(i.nrf_log_backend_hexdump_handler_get)
    i.nrf_log_backend_init                   0x00021188   Section        0  nrf_log_backend_serial.o(i.nrf_log_backend_init)
    i.nrf_log_backend_serial_hexdump_handler 0x000211b0   Section        0  nrf_log_backend_serial.o(i.nrf_log_backend_serial_hexdump_handler)
    nrf_log_backend_serial_hexdump_handler   0x000211b1   Thumb Code   286  nrf_log_backend_serial.o(i.nrf_log_backend_serial_hexdump_handler)
    i.nrf_log_backend_serial_std_handler     0x000212ce   Section        0  nrf_log_backend_serial.o(i.nrf_log_backend_serial_std_handler)
    nrf_log_backend_serial_std_handler       0x000212cf   Thumb Code   310  nrf_log_backend_serial.o(i.nrf_log_backend_serial_std_handler)
    i.nrf_log_backend_std_handler_get        0x00021404   Section        0  nrf_log_backend_serial.o(i.nrf_log_backend_std_handler_get)
    i.nrf_log_direct_feed                    0x0002140c   Section        0  nrf_log_frontend.o(i.nrf_log_direct_feed)
    nrf_log_direct_feed                      0x0002140d   Thumb Code    22  nrf_log_frontend.o(i.nrf_log_direct_feed)
    i.nrf_log_frontend_hexdump               0x00021428   Section        0  nrf_log_frontend.o(i.nrf_log_frontend_hexdump)
    i.nrf_log_frontend_init                  0x00021460   Section        0  nrf_log_frontend.o(i.nrf_log_frontend_init)
    i.nrf_log_frontend_std_0                 0x00021464   Section        0  nrf_log_frontend.o(i.nrf_log_frontend_std_0)
    i.nrf_log_frontend_std_1                 0x0002146c   Section        0  nrf_log_frontend.o(i.nrf_log_frontend_std_1)
    i.nrf_log_handlers_set                   0x0002147c   Section        0  nrf_log_frontend.o(i.nrf_log_handlers_set)
    i.nrf_log_init                           0x00021488   Section        0  nrf_log_frontend.o(i.nrf_log_init)
    i.nrf_queue_generic_pop                  0x000214ac   Section        0  nrf_queue.o(i.nrf_queue_generic_pop)
    i.nrf_queue_is_empty                     0x00021538   Section        0  nrf_queue.o(i.nrf_queue_is_empty)
    i.nrf_queue_is_full                      0x0002154a   Section        0  nrf_queue.o(i.nrf_queue_is_full)
    i.nrf_queue_next_idx                     0x00021562   Section        0  nrf_queue.o(i.nrf_queue_next_idx)
    nrf_queue_next_idx                       0x00021563   Thumb Code    14  nrf_queue.o(i.nrf_queue_next_idx)
    i.nrf_queue_push                         0x00021570   Section        0  nrf_queue.o(i.nrf_queue_push)
    i.nrf_twim_event_check                   0x0002161e   Section        0  nrf_drv_twi.o(i.nrf_twim_event_check)
    nrf_twim_event_check                     0x0002161f   Thumb Code    10  nrf_drv_twi.o(i.nrf_twim_event_check)
    i.nrf_twim_event_clear                   0x00021628   Section        0  nrf_drv_twi.o(i.nrf_twim_event_clear)
    nrf_twim_event_clear                     0x00021629   Thumb Code    12  nrf_drv_twi.o(i.nrf_twim_event_clear)
    i.power_manage                           0x00021634   Section        0  main.o(i.power_manage)
    power_manage                             0x00021635   Thumb Code    12  main.o(i.power_manage)
    i.queue_utilization_get                  0x00021640   Section        0  nrf_queue.o(i.queue_utilization_get)
    queue_utilization_get                    0x00021641   Thumb Code    24  nrf_queue.o(i.queue_utilization_get)
    i.read_reg                               0x00021658   Section        0  twi_slave_tiny_unwrap.o(i.read_reg)
    read_reg                                 0x00021659   Thumb Code    50  twi_slave_tiny_unwrap.o(i.read_reg)
    i.rtc1_init                              0x00021694   Section        0  app_timer.o(i.rtc1_init)
    rtc1_init                                0x00021695   Thumb Code    12  app_timer.o(i.rtc1_init)
    i.rtc1_start                             0x000216a4   Section        0  app_timer.o(i.rtc1_start)
    rtc1_start                               0x000216a5   Thumb Code    44  app_timer.o(i.rtc1_start)
    i.rtc1_stop                              0x000216d8   Section        0  app_timer.o(i.rtc1_stop)
    rtc1_stop                                0x000216d9   Thumb Code    56  app_timer.o(i.rtc1_stop)
    i.sd_nvic_EnableIRQ                      0x0002171c   Section        0  softdevice_handler.o(i.sd_nvic_EnableIRQ)
    sd_nvic_EnableIRQ                        0x0002171d   Thumb Code   122  softdevice_handler.o(i.sd_nvic_EnableIRQ)
    i.serial_is_busy                         0x0002179c   Section        0  nrf_log_backend_serial.o(i.serial_is_busy)
    serial_is_busy                           0x0002179d   Thumb Code     4  nrf_log_backend_serial.o(i.serial_is_busy)
    i.serial_tx                              0x000217a0   Section        0  nrf_log_backend_serial.o(i.serial_tx)
    serial_tx                                0x000217a1   Thumb Code    46  nrf_log_backend_serial.o(i.serial_tx)
    i.service_data_encode                    0x000217ce   Section        0  ble_advdata.o(i.service_data_encode)
    service_data_encode                      0x000217cf   Thumb Code   140  ble_advdata.o(i.service_data_encode)
    i.softdevice_app_ram_start_get           0x0002185c   Section        0  softdevice_handler.o(i.softdevice_app_ram_start_get)
    i.softdevice_enable                      0x00021870   Section        0  softdevice_handler.o(i.softdevice_enable)
    i.softdevice_fault_handler               0x0002198c   Section        0  softdevice_handler.o(i.softdevice_fault_handler)
    i.softdevice_handler_init                0x00021990   Section        0  softdevice_handler.o(i.softdevice_handler_init)
    i.softdevice_handler_is_enabled          0x00021a04   Section        0  softdevice_handler.o(i.softdevice_handler_is_enabled)
    i.srdata_check                           0x00021a10   Section        0  ble_advdata.o(i.srdata_check)
    srdata_check                             0x00021a11   Thumb Code    14  ble_advdata.o(i.srdata_check)
    i.start_pending_transaction              0x00021a20   Section        0  app_twi.o(i.start_pending_transaction)
    start_pending_transaction                0x00021a21   Thumb Code   162  app_twi.o(i.start_pending_transaction)
    i.start_transfer                         0x00021ac8   Section        0  app_twi.o(i.start_transfer)
    start_transfer                           0x00021ac9   Thumb Code   172  app_twi.o(i.start_transfer)
    i.test_case                              0x00021b74   Section        0  twi_slave_tiny_unwrap.o(i.test_case)
    test_case                                0x00021b75   Thumb Code    46  twi_slave_tiny_unwrap.o(i.test_case)
    i.timeout_handler_exec                   0x00021bb0   Section        0  app_timer.o(i.timeout_handler_exec)
    timeout_handler_exec                     0x00021bb1   Thumb Code     8  app_timer.o(i.timeout_handler_exec)
    i.timer_list_handler                     0x00021bb8   Section        0  app_timer.o(i.timer_list_handler)
    timer_list_handler                       0x00021bb9   Thumb Code    62  app_timer.o(i.timer_list_handler)
    i.timer_list_handler_sched               0x00021bfc   Section        0  app_timer.o(i.timer_list_handler_sched)
    timer_list_handler_sched                 0x00021bfd   Thumb Code     6  app_timer.o(i.timer_list_handler_sched)
    i.timer_list_insert                      0x00021c04   Section        0  app_timer.o(i.timer_list_insert)
    timer_list_insert                        0x00021c05   Thumb Code    66  app_timer.o(i.timer_list_insert)
    i.timer_list_remove                      0x00021c4c   Section        0  app_timer.o(i.timer_list_remove)
    timer_list_remove                        0x00021c4d   Thumb Code    94  app_timer.o(i.timer_list_remove)
    i.timer_timeouts_check                   0x00021cb4   Section        0  app_timer.o(i.timer_timeouts_check)
    timer_timeouts_check                     0x00021cb5   Thumb Code   116  app_timer.o(i.timer_timeouts_check)
    i.timer_timeouts_check_sched             0x00021d30   Section        0  app_timer.o(i.timer_timeouts_check_sched)
    timer_timeouts_check_sched               0x00021d31   Thumb Code     6  app_timer.o(i.timer_timeouts_check_sched)
    i.timers_init                            0x00021d36   Section        0  main.o(i.timers_init)
    timers_init                              0x00021d37   Thumb Code    20  main.o(i.timers_init)
    i.timestamp_process                      0x00021d4c   Section        0  nrf_log_backend_serial.o(i.timestamp_process)
    timestamp_process                        0x00021d4d   Thumb Code    44  nrf_log_backend_serial.o(i.timestamp_process)
    i.transaction_end_signal                 0x00021d80   Section        0  app_twi.o(i.transaction_end_signal)
    transaction_end_signal                   0x00021d81   Thumb Code    26  app_twi.o(i.transaction_end_signal)
    i.twi_clear_bus                          0x00021d9a   Section        0  nrf_drv_twi.o(i.twi_clear_bus)
    twi_clear_bus                            0x00021d9b   Thumb Code   174  nrf_drv_twi.o(i.twi_clear_bus)
    i.twi_event_handler                      0x00021e48   Section        0  app_twi.o(i.twi_event_handler)
    twi_event_handler                        0x00021e49   Thumb Code    64  app_twi.o(i.twi_event_handler)
    i.twi_init                               0x00021e88   Section        0  twi_slave_tiny_unwrap.o(i.twi_init)
    twi_init                                 0x00021e89   Thumb Code    46  twi_slave_tiny_unwrap.o(i.twi_init)
    i.twi_process_error                      0x00021ebc   Section        0  nrf_drv_twi.o(i.twi_process_error)
    twi_process_error                        0x00021ebd   Thumb Code    30  nrf_drv_twi.o(i.twi_process_error)
    i.twi_slave_tiny_main_unwrap             0x00021eda   Section        0  twi_slave_tiny_unwrap.o(i.twi_slave_tiny_main_unwrap)
    i.twim_list_enable_handle                0x00021ef6   Section        0  nrf_drv_twi.o(i.twim_list_enable_handle)
    twim_list_enable_handle                  0x00021ef7   Thumb Code    40  nrf_drv_twi.o(i.twim_list_enable_handle)
    i.twim_xfer                              0x00021f20   Section        0  nrf_drv_twi.o(i.twim_xfer)
    twim_xfer                                0x00021f21   Thumb Code   590  nrf_drv_twi.o(i.twim_xfer)
    i.tx_power_level_encode                  0x00022174   Section        0  ble_advdata.o(i.tx_power_level_encode)
    tx_power_level_encode                    0x00022175   Thumb Code    50  ble_advdata.o(i.tx_power_level_encode)
    i.uint16_encode                          0x000221a6   Section        0  ble_advdata.o(i.uint16_encode)
    uint16_encode                            0x000221a7   Thumb Code    10  ble_advdata.o(i.uint16_encode)
    i.uuid_list_encode                       0x000221b0   Section        0  ble_advdata.o(i.uuid_list_encode)
    uuid_list_encode                         0x000221b1   Thumb Code    56  ble_advdata.o(i.uuid_list_encode)
    i.uuid_list_sized_encode                 0x000221e8   Section        0  ble_advdata.o(i.uuid_list_sized_encode)
    uuid_list_sized_encode                   0x000221e9   Thumb Code   164  ble_advdata.o(i.uuid_list_sized_encode)
    i.write_reg                              0x0002228c   Section        0  twi_slave_tiny_unwrap.o(i.write_reg)
    write_reg                                0x0002228d   Thumb Code    78  twi_slave_tiny_unwrap.o(i.write_reg)
    .constdata                               0x000222e0   Section        4  main.o(.constdata)
    .constdata                               0x000222e4   Section       20  twi_slave_tiny_unwrap.o(.constdata)
    m_app_twi_queue                          0x000222e4   Data          20  twi_slave_tiny_unwrap.o(.constdata)
    .constdata                               0x000222f8   Section       56  twi_slave_tiny_unwrap.o(.constdata)
    m_app_twi                                0x00022300   Data          16  twi_slave_tiny_unwrap.o(.constdata)
    .constdata                               0x00022330   Section        4  nrf_drv_gpiote.o(.constdata)
    .constdata                               0x00022334   Section       20  app_twi.o(.constdata)
    .constdata                               0x00022348   Section      129  ctype_o.o(.constdata)
    .constdata                               0x000223cc   Section        4  ctype_o.o(.constdata)
    table                                    0x000223cc   Data           4  ctype_o.o(.constdata)
    .data                                    0x20001b38   Section       23  main.o(.data)
    m_beacon_info                            0x20001b38   Data          23  main.o(.data)
    .data                                    0x20001b4f   Section        1  twi_slave_tiny_unwrap.o(.data)
    tx_buff                                  0x20001b4f   Data           1  twi_slave_tiny_unwrap.o(.data)
    .data                                    0x20001b50   Section       20  app_timer.o(.data)
    m_ticks_elapsed_q_read_ind               0x20001b50   Data           1  app_timer.o(.data)
    m_ticks_elapsed_q_write_ind              0x20001b51   Data           1  app_timer.o(.data)
    m_rtc1_running                           0x20001b52   Data           1  app_timer.o(.data)
    m_rtc1_reset                             0x20001b53   Data           1  app_timer.o(.data)
    mp_timer_id_head                         0x20001b54   Data           4  app_timer.o(.data)
    m_ticks_latest                           0x20001b58   Data           4  app_timer.o(.data)
    m_ticks_elapsed                          0x20001b5c   Data           8  app_timer.o(.data)
    .data                                    0x20001b64   Section        2  nrf_log_backend_serial.o(.data)
    m_initialized                            0x20001b64   Data           1  nrf_log_backend_serial.o(.data)
    m_blocking_mode                          0x20001b65   Data           1  nrf_log_backend_serial.o(.data)
    .data                                    0x20001b68   Section       20  softdevice_handler.o(.data)
    m_softdevice_enabled                     0x20001b68   Data           1  softdevice_handler.o(.data)
    m_suspended                              0x20001b69   Data           1  softdevice_handler.o(.data)
    m_ble_evt_buffer_size                    0x20001b6a   Data           2  softdevice_handler.o(.data)
    m_evt_schedule_func                      0x20001b6c   Data           4  softdevice_handler.o(.data)
    m_sys_evt_handler                        0x20001b70   Data           4  softdevice_handler.o(.data)
    mp_ble_evt_buffer                        0x20001b74   Data           4  softdevice_handler.o(.data)
    m_ble_evt_handler                        0x20001b78   Data           4  softdevice_handler.o(.data)
    .data                                    0x20001b7c   Section        4  system_nrf52.o(.data)
    __tagsym$$used                           0x20001b7c   Number         0  system_nrf52.o(.data)
    .bss                                     0x20001b80   Section       96  main.o(.bss)
    BLE_EVT_BUFFER                           0x20001b80   Data          80  main.o(.bss)
    m_adv_params                             0x20001bd0   Data          16  main.o(.bss)
    .bss                                     0x20001be0   Section       28  twi_slave_tiny_unwrap.o(.bss)
    m_app_twi_queue_nrf_queue_buffer         0x20001be0   Data          28  twi_slave_tiny_unwrap.o(.bss)
    .bss                                     0x20001bfc   Section       12  twi_slave_tiny_unwrap.o(.bss)
    m_app_twi_queue_nrf_queue_cb             0x20001bfc   Data          12  twi_slave_tiny_unwrap.o(.bss)
    .bss                                     0x20001c08   Section       28  twi_slave_tiny_unwrap.o(.bss)
    m_app_twi_cb                             0x20001c08   Data          28  twi_slave_tiny_unwrap.o(.bss)
    .bss                                     0x20001c24   Section       20  nrf_drv_clock.o(.bss)
    m_clock_cb                               0x20001c24   Data          20  nrf_drv_clock.o(.bss)
    .bss                                     0x20001c38   Section       88  nrf_drv_gpiote.o(.bss)
    m_cb                                     0x20001c38   Data          88  nrf_drv_gpiote.o(.bss)
    .bss                                     0x20001c90   Section       44  nrf_drv_twi.o(.bss)
    m_cb                                     0x20001c90   Data          44  nrf_drv_twi.o(.bss)
    .bss                                     0x20001cbc   Section      268  app_timer.o(.bss)
    m_op_queue                               0x20001cbc   Data         268  app_timer.o(.bss)
    .bss                                     0x20001dc8   Section       12  app_util_platform.o(.bss)
    .bss                                     0x20001dd4   Section       28  nrf_log_frontend.o(.bss)
    m_log_data                               0x20001dd4   Data          28  nrf_log_frontend.o(.bss)
    .bss                                     0x20001df0   Section     1160  segger_rtt.o(.bss)
    _acUpBuffer                              0x20001df0   Data        1024  segger_rtt.o(.bss)
    _acDownBuffer                            0x200021f0   Data          16  segger_rtt.o(.bss)
    STACK                                    0x20002278   Section     8192  arm_startup_nrf52.o(STACK)

    Global Symbols

    Symbol Name                              Value     Ov Type        Size  Object(Section)

    BuildAttributes$$THM_ISAv4$E$P$D$K$B$S$7EM$VFPi3$EXTD16$VFPS$VFMA$PE$A:L22UL41UL21$X:L11$S22US41US21$IEEE1$IW$USESV6$~STKCKD$USESV7$~SHL$OSPACE$ROPI$EBA8$MICROLIB$REQ8$PRES8$EABIv2 0x00000000   Number         0  anon$$obj.o ABSOLUTE
    __ARM_use_no_argv                        0x00000000   Number         0  main.o ABSOLUTE
    _printf_a                                0x00000000   Number         0  stubs.o ABSOLUTE
    _printf_c                                0x00000000   Number         0  stubs.o ABSOLUTE
    _printf_charcount                        0x00000000   Number         0  stubs.o ABSOLUTE
    _printf_d                                0x00000000   Number         0  stubs.o ABSOLUTE
    _printf_e                                0x00000000   Number         0  stubs.o ABSOLUTE
    _printf_f                                0x00000000   Number         0  stubs.o ABSOLUTE
    _printf_flags                            0x00000000   Number         0  stubs.o ABSOLUTE
    _printf_fp_dec                           0x00000000   Number         0  stubs.o ABSOLUTE
    _printf_fp_hex                           0x00000000   Number         0  stubs.o ABSOLUTE
    _printf_g                                0x00000000   Number         0  stubs.o ABSOLUTE
    _printf_i                                0x00000000   Number         0  stubs.o ABSOLUTE
    _printf_int_dec                          0x00000000   Number         0  stubs.o ABSOLUTE
    _printf_l                                0x00000000   Number         0  stubs.o ABSOLUTE
    _printf_lc                               0x00000000   Number         0  stubs.o ABSOLUTE
    _printf_ll                               0x00000000   Number         0  stubs.o ABSOLUTE
    _printf_lld                              0x00000000   Number         0  stubs.o ABSOLUTE
    _printf_lli                              0x00000000   Number         0  stubs.o ABSOLUTE
    _printf_llo                              0x00000000   Number         0  stubs.o ABSOLUTE
    _printf_llu                              0x00000000   Number         0  stubs.o ABSOLUTE
    _printf_llx                              0x00000000   Number         0  stubs.o ABSOLUTE
    _printf_longlong_dec                     0x00000000   Number         0  stubs.o ABSOLUTE
    _printf_longlong_hex                     0x00000000   Number         0  stubs.o ABSOLUTE
    _printf_longlong_oct                     0x00000000   Number         0  stubs.o ABSOLUTE
    _printf_ls                               0x00000000   Number         0  stubs.o ABSOLUTE
    _printf_mbtowc                           0x00000000   Number         0  stubs.o ABSOLUTE
    _printf_n                                0x00000000   Number         0  stubs.o ABSOLUTE
    _printf_o                                0x00000000   Number         0  stubs.o ABSOLUTE
    _printf_p                                0x00000000   Number         0  stubs.o ABSOLUTE
    _printf_percent                          0x00000000   Number         0  stubs.o ABSOLUTE
    _printf_pre_padding                      0x00000000   Number         0  stubs.o ABSOLUTE
    _printf_return_value                     0x00000000   Number         0  stubs.o ABSOLUTE
    _printf_s                                0x00000000   Number         0  stubs.o ABSOLUTE
    _printf_sizespec                         0x00000000   Number         0  stubs.o ABSOLUTE
    _printf_str                              0x00000000   Number         0  stubs.o ABSOLUTE
    _printf_truncate_signed                  0x00000000   Number         0  stubs.o ABSOLUTE
    _printf_truncate_unsigned                0x00000000   Number         0  stubs.o ABSOLUTE
    _printf_u                                0x00000000   Number         0  stubs.o ABSOLUTE
    _printf_wc                               0x00000000   Number         0  stubs.o ABSOLUTE
    _printf_wctomb                           0x00000000   Number         0  stubs.o ABSOLUTE
    _printf_widthprec                        0x00000000   Number         0  stubs.o ABSOLUTE
    _printf_x                                0x00000000   Number         0  stubs.o ABSOLUTE
    __cpp_initialize__aeabi_                  - Undefined Weak Reference
    __cxa_finalize                            - Undefined Weak Reference
    __decompress                              - Undefined Weak Reference
    _clock_init                               - Undefined Weak Reference
    _microlib_exit                            - Undefined Weak Reference
    __Vectors_Size                           0x00000200   Number         0  arm_startup_nrf52.o ABSOLUTE
    __Vectors                                0x0001f000   Data           4  arm_startup_nrf52.o(RESET)
    __Vectors_End                            0x0001f200   Data           0  arm_startup_nrf52.o(RESET)
    __main                                   0x0001f201   Thumb Code     0  entry.o(.ARM.Collect$$$$00000000)
    _main_stk                                0x0001f201   Thumb Code     0  entry2.o(.ARM.Collect$$$$00000001)
    _main_scatterload                        0x0001f205   Thumb Code     0  entry5.o(.ARM.Collect$$$$00000004)
    __main_after_scatterload                 0x0001f209   Thumb Code     0  entry5.o(.ARM.Collect$$$$00000004)
    _main_clock                              0x0001f209   Thumb Code     0  entry7b.o(.ARM.Collect$$$$00000008)
    _main_cpp_init                           0x0001f209   Thumb Code     0  entry8b.o(.ARM.Collect$$$$0000000A)
    _main_init                               0x0001f209   Thumb Code     0  entry9a.o(.ARM.Collect$$$$0000000B)
    __rt_final_cpp                           0x0001f211   Thumb Code     0  entry10a.o(.ARM.Collect$$$$0000000D)
    __rt_final_exit                          0x0001f211   Thumb Code     0  entry11a.o(.ARM.Collect$$$$0000000F)
    Reset_Handler                            0x0001f215   Thumb Code     8  arm_startup_nrf52.o(.text)
    NMI_Handler                              0x0001f21d   Thumb Code     2  arm_startup_nrf52.o(.text)
    HardFault_Handler                        0x0001f21f   Thumb Code     2  arm_startup_nrf52.o(.text)
    MemoryManagement_Handler                 0x0001f221   Thumb Code     2  arm_startup_nrf52.o(.text)
    BusFault_Handler                         0x0001f223   Thumb Code     2  arm_startup_nrf52.o(.text)
    UsageFault_Handler                       0x0001f225   Thumb Code     2  arm_startup_nrf52.o(.text)
    SVC_Handler                              0x0001f227   Thumb Code     2  arm_startup_nrf52.o(.text)
    DebugMon_Handler                         0x0001f229   Thumb Code     2  arm_startup_nrf52.o(.text)
    PendSV_Handler                           0x0001f22b   Thumb Code     2  arm_startup_nrf52.o(.text)
    SysTick_Handler                          0x0001f22d   Thumb Code     2  arm_startup_nrf52.o(.text)
    CCM_AAR_IRQHandler                       0x0001f22f   Thumb Code     0  arm_startup_nrf52.o(.text)
    COMP_LPCOMP_IRQHandler                   0x0001f22f   Thumb Code     0  arm_startup_nrf52.o(.text)
    ECB_IRQHandler                           0x0001f22f   Thumb Code     0  arm_startup_nrf52.o(.text)
    FPU_IRQHandler                           0x0001f22f   Thumb Code     0  arm_startup_nrf52.o(.text)
    I2S_IRQHandler                           0x0001f22f   Thumb Code     0  arm_startup_nrf52.o(.text)
    MWU_IRQHandler                           0x0001f22f   Thumb Code     0  arm_startup_nrf52.o(.text)
    NFCT_IRQHandler                          0x0001f22f   Thumb Code     0  arm_startup_nrf52.o(.text)
    PDM_IRQHandler                           0x0001f22f   Thumb Code     0  arm_startup_nrf52.o(.text)
    PWM0_IRQHandler                          0x0001f22f   Thumb Code     0  arm_startup_nrf52.o(.text)
    PWM1_IRQHandler                          0x0001f22f   Thumb Code     0  arm_startup_nrf52.o(.text)
    PWM2_IRQHandler                          0x0001f22f   Thumb Code     0  arm_startup_nrf52.o(.text)
    QDEC_IRQHandler                          0x0001f22f   Thumb Code     0  arm_startup_nrf52.o(.text)
    RADIO_IRQHandler                         0x0001f22f   Thumb Code     0  arm_startup_nrf52.o(.text)
    RNG_IRQHandler                           0x0001f22f   Thumb Code     0  arm_startup_nrf52.o(.text)
    RTC0_IRQHandler                          0x0001f22f   Thumb Code     0  arm_startup_nrf52.o(.text)
    RTC2_IRQHandler                          0x0001f22f   Thumb Code     0  arm_startup_nrf52.o(.text)
    SAADC_IRQHandler                         0x0001f22f   Thumb Code     0  arm_startup_nrf52.o(.text)
    SPIM1_SPIS1_TWIM1_TWIS1_SPI1_TWI1_IRQHandler 0x0001f22f   Thumb Code     0  arm_startup_nrf52.o(.text)
    SPIM2_SPIS2_SPI2_IRQHandler              0x0001f22f   Thumb Code     0  arm_startup_nrf52.o(.text)
    SWI1_EGU1_IRQHandler                     0x0001f22f   Thumb Code     0  arm_startup_nrf52.o(.text)
    SWI3_EGU3_IRQHandler                     0x0001f22f   Thumb Code     0  arm_startup_nrf52.o(.text)
    SWI4_EGU4_IRQHandler                     0x0001f22f   Thumb Code     0  arm_startup_nrf52.o(.text)
    SWI5_EGU5_IRQHandler                     0x0001f22f   Thumb Code     0  arm_startup_nrf52.o(.text)
    TEMP_IRQHandler                          0x0001f22f   Thumb Code     0  arm_startup_nrf52.o(.text)
    TIMER0_IRQHandler                        0x0001f22f   Thumb Code     0  arm_startup_nrf52.o(.text)
    TIMER1_IRQHandler                        0x0001f22f   Thumb Code     0  arm_startup_nrf52.o(.text)
    TIMER2_IRQHandler                        0x0001f22f   Thumb Code     0  arm_startup_nrf52.o(.text)
    TIMER3_IRQHandler                        0x0001f22f   Thumb Code     0  arm_startup_nrf52.o(.text)
    TIMER4_IRQHandler                        0x0001f22f   Thumb Code     0  arm_startup_nrf52.o(.text)
    UARTE0_UART0_IRQHandler                  0x0001f22f   Thumb Code     0  arm_startup_nrf52.o(.text)
    WDT_IRQHandler                           0x0001f22f   Thumb Code     0  arm_startup_nrf52.o(.text)
    __rt_ctype_table                         0x0001f239   Thumb Code     4  ctype_o.o(.text)
    __aeabi_memcpy                           0x0001f241   Thumb Code    36  memcpya.o(.text)
    __aeabi_memcpy4                          0x0001f241   Thumb Code     0  memcpya.o(.text)
    __aeabi_memcpy8                          0x0001f241   Thumb Code     0  memcpya.o(.text)
    __aeabi_memset                           0x0001f265   Thumb Code    14  memseta.o(.text)
    __aeabi_memset4                          0x0001f265   Thumb Code     0  memseta.o(.text)
    __aeabi_memset8                          0x0001f265   Thumb Code     0  memseta.o(.text)
    __aeabi_memclr                           0x0001f273   Thumb Code     4  memseta.o(.text)
    __aeabi_memclr4                          0x0001f273   Thumb Code     0  memseta.o(.text)
    __aeabi_memclr8                          0x0001f273   Thumb Code     0  memseta.o(.text)
    _memset$wrapper                          0x0001f277   Thumb Code    18  memseta.o(.text)
    strlen                                   0x0001f289   Thumb Code    14  strlen.o(.text)
    memcmp                                   0x0001f297   Thumb Code    26  memcmp.o(.text)
    strcpy                                   0x0001f2b1   Thumb Code    18  strcpy.o(.text)
    __aeabi_uldivmod                         0x0001f2c3   Thumb Code    98  uldiv.o(.text)
    __scatterload                            0x0001f325   Thumb Code    28  init.o(.text)
    __scatterload_rt2                        0x0001f325   Thumb Code     0  init.o(.text)
    __aeabi_llsl                             0x0001f349   Thumb Code    30  llshl.o(.text)
    _ll_shift_l                              0x0001f349   Thumb Code     0  llshl.o(.text)
    __aeabi_llsr                             0x0001f367   Thumb Code    32  llushr.o(.text)
    _ll_ushift_r                             0x0001f367   Thumb Code     0  llushr.o(.text)
    GPIOTE_IRQHandler                        0x0001f389   Thumb Code   420  nrf_drv_gpiote.o(i.GPIOTE_IRQHandler)
    POWER_CLOCK_IRQHandler                   0x0001f535   Thumb Code    84  nrf_drv_clock.o(i.POWER_CLOCK_IRQHandler)
    RTC1_IRQHandler                          0x0001f58d   Thumb Code    20  app_timer.o(i.RTC1_IRQHandler)
    SEGGER_RTT_Init                          0x0001f5a5   Thumb Code    14  segger_rtt.o(i.SEGGER_RTT_Init)
    SEGGER_RTT_WriteNoLock                   0x0001f5b9   Thumb Code   102  segger_rtt.o(i.SEGGER_RTT_WriteNoLock)
    SPIM0_SPIS0_TWIM0_TWIS0_SPI0_TWI0_IRQHandler 0x0001f625   Thumb Code     8  nrf_drv_twi.o(i.SPIM0_SPIS0_TWIM0_TWIS0_SPI0_TWI0_IRQHandler)
    SWI0_EGU0_IRQHandler                     0x0001f635   Thumb Code     4  app_timer.o(i.SWI0_EGU0_IRQHandler)
    SWI2_EGU2_IRQHandler                     0x0001f639   Thumb Code    34  softdevice_handler.o(i.SWI2_EGU2_IRQHandler)
    SystemCoreClockUpdate                    0x0001f661   Thumb Code     8  system_nrf52.o(i.SystemCoreClockUpdate)
    SystemInit                               0x0001f671   Thumb Code   402  system_nrf52.o(i.SystemInit)
    __0snprintf$8                            0x0001f955   Thumb Code    44  printf8.o(i.__0snprintf$8)
    __1snprintf$8                            0x0001f955   Thumb Code     0  printf8.o(i.__0snprintf$8)
    __2snprintf                              0x0001f955   Thumb Code     0  printf8.o(i.__0snprintf$8)
    __scatterload_copy                       0x0001fa2f   Thumb Code    14  handlers.o(i.__scatterload_copy)
    __scatterload_null                       0x0001fa3d   Thumb Code     2  handlers.o(i.__scatterload_null)
    __scatterload_zeroinit                   0x0001fa3f   Thumb Code    14  handlers.o(i.__scatterload_zeroinit)
    adv_data_encode                          0x0001fef5   Thumb Code   270  ble_advdata.o(i.adv_data_encode)
    app_error_fault_handler                  0x00020099   Thumb Code    42  app_error_weak.o(i.app_error_fault_handler)
    app_error_handler_bare                   0x000200f9   Thumb Code    22  app_error.o(i.app_error_handler_bare)
    app_timer_init                           0x00020111   Thumb Code    62  app_timer.o(i.app_timer_init)
    app_twi_init                             0x0002015d   Thumb Code    60  app_twi.o(i.app_twi_init)
    app_twi_perform                          0x0002019d   Thumb Code   108  app_twi.o(i.app_twi_perform)
    app_twi_schedule                         0x0002020d   Thumb Code    28  app_twi.o(i.app_twi_schedule)
    app_util_critical_region_enter           0x00020229   Thumb Code    56  app_util_platform.o(i.app_util_critical_region_enter)
    app_util_critical_region_exit            0x0002026d   Thumb Code    40  app_util_platform.o(i.app_util_critical_region_exit)
    ble_advdata_set                          0x000202e5   Thumb Code   106  ble_advdata.o(i.ble_advdata_set)
    bsp_indication_set                       0x0002044d   Thumb Code     4  bsp.o(i.bsp_indication_set)
    intern_softdevice_events_execute         0x000208b9   Thumb Code   116  softdevice_handler.o(i.intern_softdevice_events_execute)
    main                                     0x00020bf1   Thumb Code    46  main.o(i.main)
    nrf_drv_clock_init                       0x00020e99   Thumb Code    70  nrf_drv_clock.o(i.nrf_drv_clock_init)
    nrf_drv_clock_on_sd_enable               0x00020eed   Thumb Code    42  nrf_drv_clock.o(i.nrf_drv_clock_on_sd_enable)
    nrf_drv_clock_on_soc_event               0x00020f1d   Thumb Code    10  nrf_drv_clock.o(i.nrf_drv_clock_on_soc_event)
    nrf_drv_common_irq_enable                0x00020f27   Thumb Code    60  nrf_drv_common.o(i.nrf_drv_common_irq_enable)
    nrf_drv_twi_disable                      0x00020f75   Thumb Code    48  nrf_drv_twi.o(i.nrf_drv_twi_disable)
    nrf_drv_twi_enable                       0x00020fa9   Thumb Code    32  nrf_drv_twi.o(i.nrf_drv_twi_enable)
    nrf_drv_twi_init                         0x00020fcd   Thumb Code   142  nrf_drv_twi.o(i.nrf_drv_twi_init)
    nrf_drv_twi_uninit                       0x00021061   Thumb Code   120  nrf_drv_twi.o(i.nrf_drv_twi_uninit)
    nrf_drv_twi_xfer                         0x000210dd   Thumb Code    34  nrf_drv_twi.o(i.nrf_drv_twi_xfer)
    nrf_log_backend_hexdump_handler_get      0x00021181   Thumb Code     4  nrf_log_backend_serial.o(i.nrf_log_backend_hexdump_handler_get)
    nrf_log_backend_init                     0x00021189   Thumb Code    36  nrf_log_backend_serial.o(i.nrf_log_backend_init)
    nrf_log_backend_std_handler_get          0x00021405   Thumb Code     4  nrf_log_backend_serial.o(i.nrf_log_backend_std_handler_get)
    nrf_log_frontend_hexdump                 0x00021429   Thumb Code    50  nrf_log_frontend.o(i.nrf_log_frontend_hexdump)
    nrf_log_frontend_init                    0x00021461   Thumb Code     4  nrf_log_frontend.o(i.nrf_log_frontend_init)
    nrf_log_frontend_std_0                   0x00021465   Thumb Code     8  nrf_log_frontend.o(i.nrf_log_frontend_std_0)
    nrf_log_frontend_std_1                   0x0002146d   Thumb Code    14  nrf_log_frontend.o(i.nrf_log_frontend_std_1)
    nrf_log_handlers_set                     0x0002147d   Thumb Code     8  nrf_log_frontend.o(i.nrf_log_handlers_set)
    nrf_log_init                             0x00021489   Thumb Code    36  nrf_log_frontend.o(i.nrf_log_init)
    nrf_queue_generic_pop                    0x000214ad   Thumb Code   140  nrf_queue.o(i.nrf_queue_generic_pop)
    nrf_queue_is_empty                       0x00021539   Thumb Code    18  nrf_queue.o(i.nrf_queue_is_empty)
    nrf_queue_is_full                        0x0002154b   Thumb Code    24  nrf_queue.o(i.nrf_queue_is_full)
    nrf_queue_push                           0x00021571   Thumb Code   174  nrf_queue.o(i.nrf_queue_push)
    softdevice_app_ram_start_get             0x0002185d   Thumb Code    16  softdevice_handler.o(i.softdevice_app_ram_start_get)
    softdevice_enable                        0x00021871   Thumb Code    78  softdevice_handler.o(i.softdevice_enable)
    softdevice_fault_handler                 0x0002198d   Thumb Code     4  softdevice_handler.o(i.softdevice_fault_handler)
    softdevice_handler_init                  0x00021991   Thumb Code   104  softdevice_handler.o(i.softdevice_handler_init)
    softdevice_handler_is_enabled            0x00021a05   Thumb Code     6  softdevice_handler.o(i.softdevice_handler_is_enabled)
    twi_slave_tiny_main_unwrap               0x00021edb   Thumb Code    28  twi_slave_tiny_unwrap.o(i.twi_slave_tiny_main_unwrap)
    __ctype_table                            0x00022348   Data         129  ctype_o.o(.constdata)
    Region$$Table$$Base                      0x000223d0   Number         0  anon$$obj.o(Region$$Table)
    Region$$Table$$Limit                     0x000223f0   Number         0  anon$$obj.o(Region$$Table)
    Image$$RW_IRAM1$$Base                    0x20001b38   Number         0  anon$$obj.o ABSOLUTE
    SystemCoreClock                          0x20001b7c   Data           4  system_nrf52.o(.data)
    nrf_nvic_state                           0x20001dc8   Data          12  app_util_platform.o(.bss)
    _SEGGER_RTT                              0x20002200   Data         120  segger_rtt.o(.bss)
    __initial_sp                             0x20004278   Data           0  arm_startup_nrf52.o(STACK)



==============================================================================

Memory Map of the image

  Image Entry point : 0x0001f201

  Load Region LR_IROM1 (Base: 0x0001f000, Size: 0x00003438, Max: 0x00061000, ABSOLUTE)

    Execution Region ER_IROM1 (Exec base: 0x0001f000, Load base: 0x0001f000, Size: 0x000033f0, Max: 0x00061000, ABSOLUTE)

    Exec Addr    Load Addr    Size         Type   Attr      Idx    E Section Name        Object

    0x0001f000   0x0001f000   0x00000200   Data   RO         2721    RESET               arm_startup_nrf52.o
    0x0001f200   0x0001f200   0x00000000   Code   RO         2817  * .ARM.Collect$$$$00000000  mc_w.l(entry.o)
    0x0001f200   0x0001f200   0x00000004   Code   RO         3121    .ARM.Collect$$$$00000001  mc_w.l(entry2.o)
    0x0001f204   0x0001f204   0x00000004   Code   RO         3124    .ARM.Collect$$$$00000004  mc_w.l(entry5.o)
    0x0001f208   0x0001f208   0x00000000   Code   RO         3126    .ARM.Collect$$$$00000008  mc_w.l(entry7b.o)
    0x0001f208   0x0001f208   0x00000000   Code   RO         3128    .ARM.Collect$$$$0000000A  mc_w.l(entry8b.o)
    0x0001f208   0x0001f208   0x00000008   Code   RO         3129    .ARM.Collect$$$$0000000B  mc_w.l(entry9a.o)
    0x0001f210   0x0001f210   0x00000000   Code   RO         3131    .ARM.Collect$$$$0000000D  mc_w.l(entry10a.o)
    0x0001f210   0x0001f210   0x00000000   Code   RO         3133    .ARM.Collect$$$$0000000F  mc_w.l(entry11a.o)
    0x0001f210   0x0001f210   0x00000004   Code   RO         3122    .ARM.Collect$$$$00002712  mc_w.l(entry2.o)
    0x0001f214   0x0001f214   0x00000024   Code   RO         2722    .text               arm_startup_nrf52.o
    0x0001f238   0x0001f238   0x00000008   Code   RO         2820    .text               mc_w.l(ctype_o.o)
    0x0001f240   0x0001f240   0x00000024   Code   RO         2848    .text               mc_w.l(memcpya.o)
    0x0001f264   0x0001f264   0x00000024   Code   RO         2850    .text               mc_w.l(memseta.o)
    0x0001f288   0x0001f288   0x0000000e   Code   RO         2852    .text               mc_w.l(strlen.o)
    0x0001f296   0x0001f296   0x0000001a   Code   RO         2854    .text               mc_w.l(memcmp.o)
    0x0001f2b0   0x0001f2b0   0x00000012   Code   RO         2856    .text               mc_w.l(strcpy.o)
    0x0001f2c2   0x0001f2c2   0x00000062   Code   RO         3140    .text               mc_w.l(uldiv.o)
    0x0001f324   0x0001f324   0x00000024   Code   RO         3153    .text               mc_w.l(init.o)
    0x0001f348   0x0001f348   0x0000001e   Code   RO         3156    .text               mc_w.l(llshl.o)
    0x0001f366   0x0001f366   0x00000020   Code   RO         3158    .text               mc_w.l(llushr.o)
    0x0001f386   0x0001f386   0x00000002   PAD
    0x0001f388   0x0001f388   0x000001ac   Code   RO         1039    i.GPIOTE_IRQHandler  nrf_drv_gpiote.o
    0x0001f534   0x0001f534   0x00000058   Code   RO          807    i.POWER_CLOCK_IRQHandler  nrf_drv_clock.o
    0x0001f58c   0x0001f58c   0x00000018   Code   RO         1660    i.RTC1_IRQHandler   app_timer.o
    0x0001f5a4   0x0001f5a4   0x00000014   Code   RO         2427    i.SEGGER_RTT_Init   segger_rtt.o
    0x0001f5b8   0x0001f5b8   0x0000006c   Code   RO         2436    i.SEGGER_RTT_WriteNoLock  segger_rtt.o
    0x0001f624   0x0001f624   0x00000010   Code   RO         1300    i.SPIM0_SPIS0_TWIM0_TWIS0_SPI0_TWI0_IRQHandler  nrf_drv_twi.o
    0x0001f634   0x0001f634   0x00000004   Code   RO         1661    i.SWI0_EGU0_IRQHandler  app_timer.o
    0x0001f638   0x0001f638   0x00000028   Code   RO         2577    i.SWI2_EGU2_IRQHandler  softdevice_handler.o
    0x0001f660   0x0001f660   0x00000010   Code   RO         2729    i.SystemCoreClockUpdate  system_nrf52.o
    0x0001f670   0x0001f670   0x000001c4   Code   RO         2730    i.SystemInit        system_nrf52.o
    0x0001f834   0x0001f834   0x00000068   Code   RO         2439    i._DoInit           segger_rtt.o
    0x0001f89c   0x0001f89c   0x00000018   Code   RO         2440    i._GetAvailWriteSpace  segger_rtt.o
    0x0001f8b4   0x0001f8b4   0x0000005c   Code   RO         2442    i._WriteBlocking    segger_rtt.o
    0x0001f910   0x0001f910   0x00000044   Code   RO         2443    i._WriteNoCheck     segger_rtt.o
    0x0001f954   0x0001f954   0x00000030   Code   RO         3068    i.__0snprintf$8     mc_w.l(printf8.o)
    0x0001f984   0x0001f984   0x0000001a   Code   RO         1662    i.__NVIC_ClearPendingIRQ  app_timer.o
    0x0001f99e   0x0001f99e   0x00000022   Code   RO         2578    i.__NVIC_DisableIRQ  softdevice_handler.o
    0x0001f9c0   0x0001f9c0   0x0000001a   Code   RO         1663    i.__NVIC_EnableIRQ  app_timer.o
    0x0001f9da   0x0001f9da   0x0000001a   Code   RO         2579    i.__NVIC_EnableIRQ  softdevice_handler.o
    0x0001f9f4   0x0001f9f4   0x0000001a   Code   RO         1664    i.__NVIC_SetPendingIRQ  app_timer.o
    0x0001fa0e   0x0001fa0e   0x00000020   Code   RO         1665    i.__NVIC_SetPriority  app_timer.o
    0x0001fa2e   0x0001fa2e   0x0000000e   Code   RO         3167    i.__scatterload_copy  mc_w.l(handlers.o)
    0x0001fa3c   0x0001fa3c   0x00000002   Code   RO         3168    i.__scatterload_null  mc_w.l(handlers.o)
    0x0001fa3e   0x0001fa3e   0x0000000e   Code   RO         3169    i.__scatterload_zeroinit  mc_w.l(handlers.o)
    0x0001fa4c   0x0001fa4c   0x00000030   Code   RO         2580    i.__sd_nvic_app_accessible_irq  softdevice_handler.o
    0x0001fa7c   0x0001fa7c   0x00000410   Code   RO         3074    i._printf_core      mc_w.l(printf8.o)
    0x0001fe8c   0x0001fe8c   0x00000024   Code   RO         3075    i._printf_post_padding  mc_w.l(printf8.o)
    0x0001feb0   0x0001feb0   0x0000002e   Code   RO         3076    i._printf_pre_padding  mc_w.l(printf8.o)
    0x0001fede   0x0001fede   0x00000016   Code   RO         3077    i._snputc           mc_w.l(printf8.o)
    0x0001fef4   0x0001fef4   0x0000010e   Code   RO          539    i.adv_data_encode   ble_advdata.o
    0x00020002   0x00020002   0x0000000e   Code   RO          540    i.advdata_check     ble_advdata.o
    0x00020010   0x00020010   0x00000060   Code   RO            4    i.advertising_init  main.o
    0x00020070   0x00020070   0x00000028   Code   RO            5    i.advertising_start  main.o
    0x00020098   0x00020098   0x00000060   Code   RO         1576    i.app_error_fault_handler  app_error_weak.o
    0x000200f8   0x000200f8   0x00000016   Code   RO         1534    i.app_error_handler_bare  app_error.o
    0x0002010e   0x0002010e   0x00000002   PAD
    0x00020110   0x00020110   0x0000004c   Code   RO         1669    i.app_timer_init    app_timer.o
    0x0002015c   0x0002015c   0x00000040   Code   RO         2012    i.app_twi_init      app_twi.o
    0x0002019c   0x0002019c   0x00000070   Code   RO         2013    i.app_twi_perform   app_twi.o
    0x0002020c   0x0002020c   0x0000001c   Code   RO         2014    i.app_twi_schedule  app_twi.o
    0x00020228   0x00020228   0x00000044   Code   RO         1866    i.app_util_critical_region_enter  app_util_platform.o
    0x0002026c   0x0002026c   0x00000030   Code   RO         1867    i.app_util_critical_region_exit  app_util_platform.o
    0x0002029c   0x0002029c   0x00000048   Code   RO          541    i.appearance_encode  ble_advdata.o
    0x000202e4   0x000202e4   0x0000006a   Code   RO          542    i.ble_advdata_set   ble_advdata.o
    0x0002034e   0x0002034e   0x00000066   Code   RO          543    i.ble_device_addr_encode  ble_advdata.o
    0x000203b4   0x000203b4   0x00000098   Code   RO            7    i.ble_stack_init    main.o
    0x0002044c   0x0002044c   0x00000004   Code   RO          455    i.bsp_indication_set  bsp.o
    0x00020450   0x00020450   0x00000012   Code   RO         2193    i.buf_len_update    nrf_log_backend_serial.o
    0x00020462   0x00020462   0x0000002a   Code   RO         2194    i.byte2hex          nrf_log_backend_serial.o
    0x0002048c   0x0002048c   0x00000010   Code   RO         1042    i.channel_port_get  nrf_drv_gpiote.o
    0x0002049c   0x0002049c   0x00000028   Code   RO          808    i.clock_clk_started_notify  nrf_drv_clock.o
    0x000204c4   0x000204c4   0x00000078   Code   RO         1675    i.compare_reg_update  app_timer.o
    0x0002053c   0x0002053c   0x00000040   Code   RO          544    i.conn_int_check    ble_advdata.o
    0x0002057c   0x0002057c   0x0000005a   Code   RO          545    i.conn_int_encode   ble_advdata.o
    0x000205d6   0x000205d6   0x00000002   PAD
    0x000205d8   0x000205d8   0x00000040   Code   RO         1676    i.elapsed_ticks_acquire  app_timer.o
    0x00020618   0x00020618   0x0000003c   Code   RO         2731    i.errata_108        system_nrf52.o
    0x00020654   0x00020654   0x0000003c   Code   RO         2732    i.errata_12         system_nrf52.o
    0x00020690   0x00020690   0x0000003c   Code   RO         2733    i.errata_136        system_nrf52.o
    0x000206cc   0x000206cc   0x0000002c   Code   RO         2734    i.errata_16         system_nrf52.o
    0x000206f8   0x000206f8   0x0000001c   Code   RO         2735    i.errata_182        system_nrf52.o
    0x00020714   0x00020714   0x0000003c   Code   RO         2736    i.errata_31         system_nrf52.o
    0x00020750   0x00020750   0x0000002c   Code   RO         2737    i.errata_32         system_nrf52.o
    0x0002077c   0x0002077c   0x0000003c   Code   RO         2738    i.errata_36         system_nrf52.o
    0x000207b8   0x000207b8   0x0000002c   Code   RO         2739    i.errata_37         system_nrf52.o
    0x000207e4   0x000207e4   0x0000002c   Code   RO         2740    i.errata_57         system_nrf52.o
    0x00020810   0x00020810   0x0000002c   Code   RO         2741    i.errata_66         system_nrf52.o
    0x0002083c   0x0002083c   0x00000048   Code   RO         1677    i.expired_timers_handler  app_timer.o
    0x00020884   0x00020884   0x00000032   Code   RO          546    i.flags_encode      ble_advdata.o
    0x000208b6   0x000208b6   0x00000002   PAD
    0x000208b8   0x000208b8   0x00000078   Code   RO         2581    i.intern_softdevice_events_execute  softdevice_handler.o
    0x00020930   0x00020930   0x0000000c   Code   RO         2016    i.internal_transaction_cb  app_twi.o
    0x0002093c   0x0002093c   0x00000196   Code   RO         1301    i.irq_handler_twim  nrf_drv_twi.o
    0x00020ad2   0x00020ad2   0x0000000e   Code   RO          811    i.item_dequeue      nrf_drv_clock.o
    0x00020ae0   0x00020ae0   0x000000f8   Code   RO         1678    i.list_insertions_handler  app_timer.o
    0x00020bd8   0x00020bd8   0x00000016   Code   RO            8    i.log_init          main.o
    0x00020bee   0x00020bee   0x00000002   PAD
    0x00020bf0   0x00020bf0   0x00000060   Code   RO            9    i.main              main.o
    0x00020c50   0x00020c50   0x00000068   Code   RO          547    i.manuf_specific_data_encode  ble_advdata.o
    0x00020cb8   0x00020cb8   0x0000009a   Code   RO          548    i.name_encode       ble_advdata.o
    0x00020d52   0x00020d52   0x00000010   Code   RO         1043    i.nrf_bitmask_bit_is_set  nrf_drv_gpiote.o
    0x00020d62   0x00020d62   0x0000000e   Code   RO          815    i.nrf_clock_event_check  nrf_drv_clock.o
    0x00020d70   0x00020d70   0x00000010   Code   RO          816    i.nrf_clock_event_clear  nrf_drv_clock.o
    0x00020d80   0x00020d80   0x0000008c   Code   RO         1302    i.nrf_delay_us      nrf_drv_twi.o
    0x00020e0c   0x00020e0c   0x0000008c   Code   RO         1679    i.nrf_delay_us      app_timer.o
    0x00020e98   0x00020e98   0x00000054   Code   RO          823    i.nrf_drv_clock_init  nrf_drv_clock.o
    0x00020eec   0x00020eec   0x00000030   Code   RO          830    i.nrf_drv_clock_on_sd_enable  nrf_drv_clock.o
    0x00020f1c   0x00020f1c   0x0000000a   Code   RO          831    i.nrf_drv_clock_on_soc_event  nrf_drv_clock.o
    0x00020f26   0x00020f26   0x0000003c   Code   RO          993    i.nrf_drv_common_irq_enable  nrf_drv_common.o
    0x00020f62   0x00020f62   0x00000010   Code   RO         1303    i.nrf_drv_is_in_RAM  nrf_drv_twi.o
    0x00020f72   0x00020f72   0x00000002   PAD
    0x00020f74   0x00020f74   0x00000034   Code   RO         1305    i.nrf_drv_twi_disable  nrf_drv_twi.o
    0x00020fa8   0x00020fa8   0x00000024   Code   RO         1306    i.nrf_drv_twi_enable  nrf_drv_twi.o
    0x00020fcc   0x00020fcc   0x00000094   Code   RO         1307    i.nrf_drv_twi_init  nrf_drv_twi.o
    0x00021060   0x00021060   0x0000007c   Code   RO         1313    i.nrf_drv_twi_uninit  nrf_drv_twi.o
    0x000210dc   0x000210dc   0x00000028   Code   RO         1314    i.nrf_drv_twi_xfer  nrf_drv_twi.o
    0x00021104   0x00021104   0x0000001e   Code   RO         1069    i.nrf_gpio_cfg_sense_set  nrf_drv_gpiote.o
    0x00021122   0x00021122   0x00000010   Code   RO         1315    i.nrf_gpio_pin_set  nrf_drv_twi.o
    0x00021132   0x00021132   0x00000002   PAD
    0x00021134   0x00021134   0x00000024   Code   RO         1070    i.nrf_gpio_ports_read  nrf_drv_gpiote.o
    0x00021158   0x00021158   0x00000014   Code   RO         1071    i.nrf_gpiote_event_clear  nrf_drv_gpiote.o
    0x0002116c   0x0002116c   0x00000014   Code   RO         1072    i.nrf_gpiote_event_is_set  nrf_drv_gpiote.o
    0x00021180   0x00021180   0x00000008   Code   RO         2196    i.nrf_log_backend_hexdump_handler_get  nrf_log_backend_serial.o
    0x00021188   0x00021188   0x00000028   Code   RO         2197    i.nrf_log_backend_init  nrf_log_backend_serial.o
    0x000211b0   0x000211b0   0x0000011e   Code   RO         2198    i.nrf_log_backend_serial_hexdump_handler  nrf_log_backend_serial.o
    0x000212ce   0x000212ce   0x00000136   Code   RO         2199    i.nrf_log_backend_serial_std_handler  nrf_log_backend_serial.o
    0x00021404   0x00021404   0x00000008   Code   RO         2200    i.nrf_log_backend_std_handler_get  nrf_log_backend_serial.o
    0x0002140c   0x0002140c   0x0000001c   Code   RO         2300    i.nrf_log_direct_feed  nrf_log_frontend.o
    0x00021428   0x00021428   0x00000038   Code   RO         2302    i.nrf_log_frontend_hexdump  nrf_log_frontend.o
    0x00021460   0x00021460   0x00000004   Code   RO         2303    i.nrf_log_frontend_init  nrf_log_frontend.o
    0x00021464   0x00021464   0x00000008   Code   RO         2304    i.nrf_log_frontend_std_0  nrf_log_frontend.o
    0x0002146c   0x0002146c   0x0000000e   Code   RO         2305    i.nrf_log_frontend_std_1  nrf_log_frontend.o
    0x0002147a   0x0002147a   0x00000002   PAD
    0x0002147c   0x0002147c   0x0000000c   Code   RO         2312    i.nrf_log_handlers_set  nrf_log_frontend.o
    0x00021488   0x00021488   0x00000024   Code   RO         2313    i.nrf_log_init      nrf_log_frontend.o
    0x000214ac   0x000214ac   0x0000008c   Code   RO         2084    i.nrf_queue_generic_pop  nrf_queue.o
    0x00021538   0x00021538   0x00000012   Code   RO         2086    i.nrf_queue_is_empty  nrf_queue.o
    0x0002154a   0x0002154a   0x00000018   Code   RO         2087    i.nrf_queue_is_full  nrf_queue.o
    0x00021562   0x00021562   0x0000000e   Code   RO         2089    i.nrf_queue_next_idx  nrf_queue.o
    0x00021570   0x00021570   0x000000ae   Code   RO         2091    i.nrf_queue_push    nrf_queue.o
    0x0002161e   0x0002161e   0x0000000a   Code   RO         1316    i.nrf_twim_event_check  nrf_drv_twi.o
    0x00021628   0x00021628   0x0000000c   Code   RO         1317    i.nrf_twim_event_clear  nrf_drv_twi.o
    0x00021634   0x00021634   0x0000000c   Code   RO           10    i.power_manage      main.o
    0x00021640   0x00021640   0x00000018   Code   RO         2097    i.queue_utilization_get  nrf_queue.o
    0x00021658   0x00021658   0x0000003c   Code   RO          259    i.read_reg          twi_slave_tiny_unwrap.o
    0x00021694   0x00021694   0x00000010   Code   RO         1680    i.rtc1_init         app_timer.o
    0x000216a4   0x000216a4   0x00000034   Code   RO         1681    i.rtc1_start        app_timer.o
    0x000216d8   0x000216d8   0x00000044   Code   RO         1682    i.rtc1_stop         app_timer.o
    0x0002171c   0x0002171c   0x00000080   Code   RO         2582    i.sd_nvic_EnableIRQ  softdevice_handler.o
    0x0002179c   0x0002179c   0x00000004   Code   RO         2202    i.serial_is_busy    nrf_log_backend_serial.o
    0x000217a0   0x000217a0   0x0000002e   Code   RO         2203    i.serial_tx         nrf_log_backend_serial.o
    0x000217ce   0x000217ce   0x0000008c   Code   RO          549    i.service_data_encode  ble_advdata.o
    0x0002185a   0x0002185a   0x00000002   PAD
    0x0002185c   0x0002185c   0x00000014   Code   RO         2583    i.softdevice_app_ram_start_get  softdevice_handler.o
    0x00021870   0x00021870   0x0000011c   Code   RO         2585    i.softdevice_enable  softdevice_handler.o
    0x0002198c   0x0002198c   0x00000004   Code   RO         2586    i.softdevice_fault_handler  softdevice_handler.o
    0x00021990   0x00021990   0x00000074   Code   RO         2587    i.softdevice_handler_init  softdevice_handler.o
    0x00021a04   0x00021a04   0x0000000c   Code   RO         2588    i.softdevice_handler_is_enabled  softdevice_handler.o
    0x00021a10   0x00021a10   0x0000000e   Code   RO          550    i.srdata_check      ble_advdata.o
    0x00021a1e   0x00021a1e   0x00000002   PAD
    0x00021a20   0x00021a20   0x000000a8   Code   RO         2017    i.start_pending_transaction  app_twi.o
    0x00021ac8   0x00021ac8   0x000000ac   Code   RO         2018    i.start_transfer    app_twi.o
    0x00021b74   0x00021b74   0x0000003c   Code   RO          260    i.test_case         twi_slave_tiny_unwrap.o
    0x00021bb0   0x00021bb0   0x00000008   Code   RO         1683    i.timeout_handler_exec  app_timer.o
    0x00021bb8   0x00021bb8   0x00000044   Code   RO         1684    i.timer_list_handler  app_timer.o
    0x00021bfc   0x00021bfc   0x00000006   Code   RO         1685    i.timer_list_handler_sched  app_timer.o
    0x00021c02   0x00021c02   0x00000002   PAD
    0x00021c04   0x00021c04   0x00000048   Code   RO         1686    i.timer_list_insert  app_timer.o
    0x00021c4c   0x00021c4c   0x00000068   Code   RO         1687    i.timer_list_remove  app_timer.o
    0x00021cb4   0x00021cb4   0x0000007c   Code   RO         1690    i.timer_timeouts_check  app_timer.o
    0x00021d30   0x00021d30   0x00000006   Code   RO         1691    i.timer_timeouts_check_sched  app_timer.o
    0x00021d36   0x00021d36   0x00000014   Code   RO           11    i.timers_init       main.o
    0x00021d4a   0x00021d4a   0x00000002   PAD
    0x00021d4c   0x00021d4c   0x00000034   Code   RO         2204    i.timestamp_process  nrf_log_backend_serial.o
    0x00021d80   0x00021d80   0x0000001a   Code   RO         2019    i.transaction_end_signal  app_twi.o
    0x00021d9a   0x00021d9a   0x000000ae   Code   RO         1318    i.twi_clear_bus     nrf_drv_twi.o
    0x00021e48   0x00021e48   0x00000040   Code   RO         2020    i.twi_event_handler  app_twi.o
    0x00021e88   0x00021e88   0x00000034   Code   RO          261    i.twi_init          twi_slave_tiny_unwrap.o
    0x00021ebc   0x00021ebc   0x0000001e   Code   RO         1319    i.twi_process_error  nrf_drv_twi.o
    0x00021eda   0x00021eda   0x0000001c   Code   RO          262    i.twi_slave_tiny_main_unwrap  twi_slave_tiny_unwrap.o
    0x00021ef6   0x00021ef6   0x00000028   Code   RO         1320    i.twim_list_enable_handle  nrf_drv_twi.o
    0x00021f1e   0x00021f1e   0x00000002   PAD
    0x00021f20   0x00021f20   0x00000254   Code   RO         1321    i.twim_xfer         nrf_drv_twi.o
    0x00022174   0x00022174   0x00000032   Code   RO          551    i.tx_power_level_encode  ble_advdata.o
    0x000221a6   0x000221a6   0x0000000a   Code   RO          552    i.uint16_encode     ble_advdata.o
    0x000221b0   0x000221b0   0x00000038   Code   RO          553    i.uuid_list_encode  ble_advdata.o
    0x000221e8   0x000221e8   0x000000a4   Code   RO          554    i.uuid_list_sized_encode  ble_advdata.o
    0x0002228c   0x0002228c   0x00000054   Code   RO          263    i.write_reg         twi_slave_tiny_unwrap.o
    0x000222e0   0x000222e0   0x00000004   Data   RO           13    .constdata          main.o
    0x000222e4   0x000222e4   0x00000014   Data   RO          267    .constdata          twi_slave_tiny_unwrap.o
    0x000222f8   0x000222f8   0x00000038   Data   RO          268    .constdata          twi_slave_tiny_unwrap.o
    0x00022330   0x00022330   0x00000004   Data   RO         1076    .constdata          nrf_drv_gpiote.o
    0x00022334   0x00022334   0x00000014   Data   RO         2021    .constdata          app_twi.o
    0x00022348   0x00022348   0x00000081   Data   RO         2821    .constdata          mc_w.l(ctype_o.o)
    0x000223c9   0x000223c9   0x00000003   PAD
    0x000223cc   0x000223cc   0x00000004   Data   RO         2822    .constdata          mc_w.l(ctype_o.o)
    0x000223d0   0x000223d0   0x00000020   Data   RO         3165    Region$$Table       anon$$obj.o


    Execution Region RW_IRAM1 (Exec base: 0x20001b38, Load base: 0x000223f0, Size: 0x00002740, Max: 0x0000e4c8, ABSOLUTE)

    Exec Addr    Load Addr    Size         Type   Attr      Idx    E Section Name        Object

    0x20001b38   0x000223f0   0x00000017   Data   RW           14    .data               main.o
    0x20001b4f   0x00022407   0x00000001   Data   RW          269    .data               twi_slave_tiny_unwrap.o
    0x20001b50   0x00022408   0x00000014   Data   RW         1695    .data               app_timer.o
    0x20001b64   0x0002241c   0x00000002   Data   RW         2206    .data               nrf_log_backend_serial.o
    0x20001b66   0x0002241e   0x00000002   PAD
    0x20001b68   0x00022420   0x00000014   Data   RW         2594    .data               softdevice_handler.o
    0x20001b7c   0x00022434   0x00000004   Data   RW         2742    .data               system_nrf52.o
    0x20001b80        -       0x00000060   Zero   RW           12    .bss                main.o
    0x20001be0        -       0x0000001c   Zero   RW          264    .bss                twi_slave_tiny_unwrap.o
    0x20001bfc        -       0x0000000c   Zero   RW          265    .bss                twi_slave_tiny_unwrap.o
    0x20001c08        -       0x0000001c   Zero   RW          266    .bss                twi_slave_tiny_unwrap.o
    0x20001c24        -       0x00000014   Zero   RW          833    .bss                nrf_drv_clock.o
    0x20001c38        -       0x00000058   Zero   RW         1075    .bss                nrf_drv_gpiote.o
    0x20001c90        -       0x0000002c   Zero   RW         1322    .bss                nrf_drv_twi.o
    0x20001cbc        -       0x0000010c   Zero   RW         1694    .bss                app_timer.o
    0x20001dc8        -       0x0000000c   Zero   RW         1872    .bss                app_util_platform.o
    0x20001dd4        -       0x0000001c   Zero   RW         2315    .bss                nrf_log_frontend.o
    0x20001df0        -       0x00000488   Zero   RW         2444    .bss                segger_rtt.o
    0x20002278        -       0x00002000   Zero   RW         2719    STACK               arm_startup_nrf52.o


==============================================================================

Image component sizes


      Code (inc. data)   RO Data    RW Data    ZI Data      Debug   Object Name

        22          0          0          0          0       2257   app_error.o
        96         54          0          0          0      30645   app_error_weak.o
         0          0          0          0          0      20768   app_scheduler.o
      1382        110          0         20        268      49509   app_timer.o
       646         14         20          0          0      10316   app_twi.o
       116         20          0          0         12      10106   app_util_platform.o
        36          8        512          0       8192        932   arm_startup_nrf52.o
      1460          0          0          0          0      39332   ble_advdata.o
         4          0          0          0          0        677   bsp.o
       438         74          4         23         96     111299   main.o
       314         28          0          0         20      13320   nrf_drv_clock.o
        60          0          0          0          0      30751   nrf_drv_common.o
       566         28          4          0         88      21368   nrf_drv_gpiote.o
      1856         46          0          0         44      62788   nrf_drv_twi.o
       814         28          0          2          0      11087   nrf_log_backend_serial.o
       158         16          0          0         28       8319   nrf_log_frontend.o
       394          0          0          0          0       5942   nrf_queue.o
       416         40          0          0       1160       8325   segger_rtt.o
       832        248          0         20          0      45490   softdevice_handler.o
      1016         98          0          4          0       8771   system_nrf52.o
       284         36         76          1         68      18309   twi_slave_tiny_unwrap.o

    ----------------------------------------------------------------------
     10934        848        648         72       9976     510311   Object Totals
         0          0         32          0          0          0   (incl. Generated)
        24          0          0          2          0          0   (incl. Padding)

    ----------------------------------------------------------------------

      Code (inc. data)   RO Data    RW Data    ZI Data      Debug   Library Member Name

         8          4        133          0          0         68   ctype_o.o
         0          0          0          0          0          0   entry.o
         0          0          0          0          0          0   entry10a.o
         0          0          0          0          0          0   entry11a.o
         8          4          0          0          0          0   entry2.o
         4          0          0          0          0          0   entry5.o
         0          0          0          0          0          0   entry7b.o
         0          0          0          0          0          0   entry8b.o
         8          4          0          0          0          0   entry9a.o
        30          0          0          0          0          0   handlers.o
        36          8          0          0          0         68   init.o
        30          0          0          0          0         68   llshl.o
        32          0          0          0          0         68   llushr.o
        26          0          0          0          0         80   memcmp.o
        36          0          0          0          0         68   memcpya.o
        36          0          0          0          0        108   memseta.o
      1192         48          0          0          0        420   printf8.o
        18          0          0          0          0         68   strcpy.o
        14          0          0          0          0         68   strlen.o
        98          0          0          0          0         92   uldiv.o

    ----------------------------------------------------------------------
      1578         68        136          0          0       1176   Library Totals
         2          0          3          0          0          0   (incl. Padding)

    ----------------------------------------------------------------------

      Code (inc. data)   RO Data    RW Data    ZI Data      Debug   Library Name

      1576         68        133          0          0       1176   mc_w.l

    ----------------------------------------------------------------------
      1578         68        136          0          0       1176   Library Totals

    ----------------------------------------------------------------------

==============================================================================


      Code (inc. data)   RO Data    RW Data    ZI Data      Debug   

     12512        916        784         72       9976     496871   Grand Totals
     12512        916        784         72       9976     496871   ELF Image Totals
     12512        916        784         72          0          0   ROM Totals

==============================================================================

    Total RO  Size (Code + RO Data)                13296 (  12.98kB)
    Total RW  Size (RW Data + ZI Data)             10048 (   9.81kB)
    Total ROM Size (Code + RO Data + RW Data)      13368 (  13.05kB)

==============================================================================

